:10000000544649530001000084EB02002F222A5A73
:1000100017130106200730174D353143171301011F
:10002000200730174D3531431713020020073017D2
:100030004D353143030000000000000000000000C7
:10004000544643530020000054B602000000000054
:100050000080011001210000252100004131020033
:10006000292100002B2100002D2100003D2100004E
:100070003D2100003D2100003D2100002F21000016
:10008000312100003D21000033210000416D0000BE
:100090000B710000372100003D2100004157001086
:1000A0003721000051500000555000003B70000007
:1000B000372100007F690000716000005950000086
:1000C0003967000037210000372100008D5B0000F8
:1000D0000000000000000000000000000000000020
:1000E0000000000000000000000000000000000010
:1000F0000000000000000000000000000000000000
:1001000000000000000000000000000000000000EF
:1001100000000000000000000000000000000000DF
:1001200000000000000000000000000000000000CF
:1001300000000000000000000000000000000000BF
:1001400000000000000000000000000000000000AF
:1001500000F003F800F020F8FEE70D480168890878
:100160008900002001C101C101C101C17047000027
:100170005C600010FEE7FEE7FEE7FEE7FEE7FEE755
:10018000FEE7FEE7FEE703480047FEE7FEE7000064
:10019000202100003D21000000F002F800F068F886
:1001A0000AA090E8000C82448344AAF10107DA45D2
:1001B00001D100F05DF8AFF2090EBAE80F0013F0BC
:1001C000010F18BFFB1A43F0010318473052020019
:1001D000905202000A444FF0000C10F8013B13F05B
:1001E000070408BF10F8014B1D1108BF10F8015B90
:1001F000641E05D010F8016B641E01F8016BF9D183
:1002000013F0080F1EBF10F8014BAD1C0C1B09D1D9
:100210006D1E58BF01F801CBFAD505E014F8016B4B
:1002200001F8016B6D1EF9D59142D6D370470000DD
:10023000103A24BF78C878C1FAD8520724BF30C812
:1002400030C144BF04680C607047000000230024E4
:1002500000250026103A28BF78C1FBD8520728BFD6
:1002600030C148BF0B6070471FB51FBD10B510BD32
:10027000DFF80CD0FFF7F8FF07F038F920F07BFF2C
:100280000080011003B4FFF7F1FF03BC20F07AFFF8
:1002900008B500200346024600900121022000F02C
:1002A0005EFB08BD38B5FF4D0024FF48AC81EC81F2
:1002B0002C8240698047E861FF202872FB480023B8
:1002C0001A46046044608460C4600461012068725E
:1002D0002C70AC70EC7001460220009400F03FFBE3
:1002E000012038BD38B5EF4D02282C7A22460DD0BA
:1002F000052810D0A24208BF38BD002003460246A0
:100300002146009000F02BFB2C7238BD022914BF4F
:1003100001240224EEE7022914BF04240824E9E79B
:1003200008B5009313460A460146012000F017FB6A
:1003300008BD08B50346009103220221012000F008
:100340000EFB08BD38B500240EF072FB002818BF64
:10035000012412F0D2FF002818BF0224D1480178EE
:10036000A14208BF38BD047000200346022100905E
:100370002246084600F0F3FA38BD38B5C94D0446A8
:100380006878A04208BF38BD07F0CAF86C70002C2E
:100390000CBF0521062100200346024600900220E2
:1003A00000F0DDFA38BD08B500210B460246009189
:1003B0000721022000F0D3FA08BD08B500210B4642
:1003C000024600910821022000F0C9FA08BD08B5D4
:1003D00000210091002814BF0122002200230321E4
:1003E000022000F0BCFA08BD08B500200346024612
:1003F00000900421022000F0B2FA08BDA94B0028A9
:10040000DA7814BF01210021D9708A4208BF7047F1
:10041000021C18BF012208B50020034600900A21E3
:10042000022000F09CFA08BD9E4B00289A7814BF69
:100430000121002199708A4208BF7047021C18BF31
:10044000012208B50020034600900921022000F097
:1004500086FA08BD93488078002818BF01207047AD
:1004600001209049087170478E48007970478D4986
:100470000020087170472DE9F0410446012700254E
:1004800003F00700874E8846012804BF0020308211
:1004900048D0022846D1308A834904280BD200284C
:1004A00018BFB06902D148688047B06110F8011BDD
:1004B0002170B0612FE0062809D288688047318A10
:1004C00080B2C1F10501C900C840207023E00828AE
:1004D00008D208698047318AC1F10701C900C840C4
:1004E000207018E00C2808D248698047318AC1F191
:1004F0000B01C900C84020700DE00E2808D28869A1
:100500008047318AC1F10D01C900C840207002E066
:10051000FF2020700027308A401C80B230820E28D5
:1005200028BF012588F800503846BDE8F08130B476
:1005300003F007000024DFF86CC1012804BFACF809
:100540000C40ACF810401BD013F0070F18D1554BDE
:10055000BCF810009B89022805D2120242EA13223D
:10056000ACF80C2009E003449D1EB5F5806F04DA59
:10057000DCF81C502B4403F8022C401CACF8100093
:100580000C7030BC00207047F0B40746002003F028
:100590000704444D0646012C04BF2E826E6125D00F
:1005A000DFF800C1022CBCF80EC003D013F0070F17
:1005B0000DD01BE02A8A0CEB0203B3F5806F15D235
:1005C000E869C05C3870501C288201200EE01202DD
:1005D00042EA1C22EA816B69012B05D1B2F5806FDA
:1005E00024BF40F2FF32EA815A1C6A610E70F0BCEF
:1005F000704738B503F0070000240D46012809D1E3
:10060000284800231A460482848119460220009457
:1006100000F0A5F92C70002038BD2DE9F04182B022
:1006200017460C0005464FF0000800F003812678BD
:100630001F49012E18BF022E05D0032E5BD0002EBD
:1006400000F0F880BEE06078421E05EB001000F874
:10065000102C607805EB001000F80F6C08686288B9
:10066000438DC08C5A4392FBF0F0627805EB021286
:1006700022F80E0C0868A288018D808C514391FBF2
:10068000F0F0617805EB011121F80C0C6178A0798C
:1006900005EB011121F80A0C6178207A05EB0111B4
:1006A00008E0000000840010A4720200908900108D
:1006B000C888001021F8080C6178607A05EB0111F8
:1006C00021F8060C6178A07B05EB011121F8040CE0
:1006D000E0790528607805EB001010F8021C0CBFCB
:1006E00041F0010121F0010100F8021C002E69D146
:1006F00002B0BDE8F0816078421E05EB001000F802
:10070000102C6278032005EB021202F80F0C086827
:100710006288438DC08C5A4392FBF0F0627805EBFF
:10072000021222F80E0C0868A288018D808C5143B9
:1007300091FBF0F0617805EB011121F80C0C06F04B
:10074000EFFE052821D107B36178B87905EB0111D7
:1007500021F80A0C6178387A05EB011121F8080CB0
:100760006178787A05EB011121F8060CF8790528F3
:10077000607805EB001010F8021C0CBF41F001017D
:1007800021F0010100F8021C17E0607805EB001071
:1007900020F80A8C607805EB001020F8088C60784F
:1007A00005EB001020F8068C607805EB001010F8BF
:1007B000021C21F0010100F8021C607805EB00101A
:1007C00020F8048C012E18BF032E06D00DF0F4FE85
:1007D000002804BF02B0BDE8F08106F0A1FE0528A4
:1007E0001CBF02B0BDE8F081012E04BFC0208DF80F
:1007F000000005D0022E0CBFC220C1208DF80000E1
:1008000060788DF8010060880123000A8DF80200ED
:10081000A0788DF80300A0880622000A8DF8040055
:1008200020798DF805006946072011F0C2FB02B05F
:10083000BDE8F08185F8008085F80180A5F8028088
:10084000A5F80480A5F80680A5F80880A5F80A8018
:10085000A5F80C80A87B20F00100A87302B0BDE8C9
:10086000F081444900204871704742484079704700
:10087000002818BF01203F49887170473D488079A2
:100880007047002818BF01203A49C871704739489D
:10089000C07970473749488170473648408970476A
:1008A0003449012048717047334B03EB80004254B8
:1008B000704730B585B001788DF8001042788DF81A
:1008C000012082788DF80220C2788DF80320027909
:1008D0008DF8042042798DF8052080798DF8060086
:1008E00000200125234C8DF8070002900390522927
:1008F00005D1A07988B9A57106F0C3F860819DF88B
:100900000000462801BF9DF801000128E079002879
:1009100003D1E57106F0B5F8608106F039FF0128D2
:100920000CD10DF097FB012801BF9DF8000046286F
:100930009DF80100012804BF05B030BD68460DF0E8
:100940008EFB05B030BD70470A49002818BF012052
:10095000487270470748407A70470848704708B5A2
:10096000DDF808C0CDF800C0DFF814C0DCF800C026
:10097000E04708BD0084001090890010386802002C
:10098000A47202007047F648D0F8500300F001004E
:10099000704770B5F24D04000AD002F077FA38B90A
:1009A000D5F8500310F0010F1CBF0020A86005D13E
:1009B0000120A860002C08BF00202DD0D5F86003CE
:1009C00010F0010F0BD1D5F8600340F00100C5F81D
:1009D0006003D5F8600320F00100C5F86003E1482A
:1009E000016811F0010F07D1016841F001010160B8
:1009F000016821F00101016004F05EFA00281CBFCB
:100A0000D5F8500310F0010F05D004F04FFA00287C
:100A100018BF04F05DFA0120286270BDD048006A5A
:100A2000002818BF01207047C00000F1804000F589
:100A3000A04041637047C00000F1804000F5A04035
:100A4000006B00F4807070471021C00000F18040FE
:100A500000F5A0404163704730B48209C24B00F0FA
:100A60000F0000EB400053F822404FF4847505EB73
:100A70008015D1F800C044F805C053F822204FF487
:100A8000867303EB80104968115030BC70478209AF
:100A9000B54850F82200D0F8402161F30D22C0F88B
:100AA00040217047B049800951F82000D0F840013A
:100AB000C0F305207047AA49D1F8402160F31742DE
:100AC000C1F840217047A648D0F84001C0F3074064
:100AD00070474FF4A072C0F3011302EB8312DFF8EA
:100AE00088C200F00F03800903EB43035CF8200089
:100AF000002900EB8310815814BF41F0010121F05F
:100B0000010181507047984A810952F8212000F074
:100B10000F0101EB410102EB8111C0F301104FF411
:100B2000A07202EB8010085800F0010070478E4A56
:100B3000810952F82110D1F8E01100F00F000122D4
:100B400001F0070102FA00F0084018BF01207047C9
:100B50004FF4A072C0F3011302EB8312DFF808C256
:100B600000F00F03800903EB43035CF82000002929
:100B700000EB8310815814BF41F0020121F0020103
:100B800081507047784A810952F8212000F00F0106
:100B900001EB410102EB8111C0F301104FF4A0728F
:100BA00002EB80100858C0F34000704781096F4A7B
:100BB00001EB410102EBC10100F00F0201EBC201A8
:100BC000C0F3011051F820007047684982091CD019
:100BD0000122B2EB901F18BF704765480068C0F350
:100BE0000800886163480268C2F308420A6200682C
:100BF000C0F30800486260480268C2F308428A6293
:100C00000068C0F30800C86270475548D0F8242136
:100C1000C2F308020A60D0F8E421C2F308428A60F5
:100C2000D0F8E421C2F30802CA60D0F8A422C2F3CB
:100C300008420A61D0F8A402C0F308004861704776
:100C40002DE9F0030122830900F00F01C0F3011C1C
:100C5000C0F3011622EA0C0C00290BBF02254D1E21
:100C600000224FEA0C124FF0080404EBCC043F4F73
:100C700003EB430C07EBCC0C0CEBC101DFF8E88075
:100C800051F826604FF4587C58F823100CEBC5053A
:100C900051F805C000F00F001CF0010F00EB400000
:100CA0004FF4927C0CEB801C40F2FF1729D02C48AB
:100CB000D0F844034FF032090005000D06FB09F699
:100CC0000EBF0120B6FBF0F0401CFF2888BFFF20BC
:100CD0004E594FF0FF0909FA04F9C0B226EA090695
:100CE000A0403043485158F8230050F80C3007FA20
:100CF00002F123EA0102114340F80C10BDE8F003B1
:100D0000704751F80C0007FA02F39843C6F3080342
:100D100003FA02F2104341F80C00BDE8F0037047FB
:100D200010B50020FFF78CFF0120FFF789FF11208D
:100D3000FFF786FF0220FFF783FF1220FFF780FFF7
:100D40004020FFF77DFF4120FFF77AFF5120FFF79A
:100D500077FF4220FFF774FFBDE8104052206FE795
:100D600000500040605B004054680200448A00105C
:100D700024590040E4590040A45A00402DE9F047AE
:100D800007464FEA9016FF480D0050F826404FF0F6
:100D900000002062C4F84001C4F80002C4F8400218
:100DA000C4F8C002C4F8000308BFBDE8F087286893
:100DB00020606868606061680120002908BF606089
:100DC000F1490860A868A060E868E0602869A0614F
:100DD0006869E061E8696062286AE0622120606316
:100DE000E063686A2064A86A6064E86AA064286BAB
:100DF000E064686B2066A86BA066E86B6067286C8F
:100E0000A067686CE067A86CC4F88000E86CC4F860
:100E10008400286DC4F88800686DC4F88C00A86D43
:100E2000C4F89000E86DC4F8A400286EC4F8A800C7
:100E3000686EC4F8AC00A86EC4F8B000E86EC4F8E0
:100E4000B400286FC4F8B800686FC4F8BC004FF055
:100E5000FF30C4F8E400A86FC4F8F000E86FC4F8ED
:100E6000F400D5F88000C4F8FC004FF4107205F1CE
:100E7000840104F580700DF0F7F8D5F8C40220F471
:100E80008030C4F84003D5F8C802C4F84C03D5F844
:100E9000CC02C4F85003D5F8D002C4F85403D5F8F6
:100EA000D402C4F85803D5F8D802C4F85C03002073
:100EB00005EBC002D2F8DC3204EBC001C1F86033AC
:100EC000D2F8E022C1F86423401C0328F0DBD5F8F7
:100ED000F402C4F87803D5F8F802C4F87C03D5F816
:100EE000FC02C4F80004D5F80003C4F80404D5F8E3
:100EF0000403C4F80804D5F80803C4F80C04D5F8B2
:100F00000C03C4F810040022002104EBC20805EB16
:100F1000C20000EB8103D3F8109308EB810CCCF8EE
:100F20003094D3F83893CCF85894D3F86033CCF895
:100F30008034491C0229ECDB05EB8200D0F88833B1
:100F400004EB8201C1F8A834D0F89C33C1F8BC345A
:100F5000D0F8B003C1F8D004521C052AD4DB002E0F
:100F600014BF8A488A48006830F0FF0105D1D4F8E0
:100F7000901060F30301C4F89010D4F8500320F0EF
:100F80000100C4F85003D4F8600320F00100C4F855
:100F90006003D4F8680320F00100C4F86803D4F8B3
:100FA000700320F00100C4F870033846BDE8F04734
:100FB0000BE6784800787047764840787047754966
:100FC000887070477348807870477349D1F854230C
:100FD00060F30902C1F8542370476F48D0F85403F6
:100FE000C0F3090070476B49486070476948406822
:100FF00070476849886070476648806870476648EF
:10100000D0F8440340F25712C0F30B0153003C20C8
:10101000A1F2571CBCF1000F4CBF521A6246A1F25C
:10102000AE2CBCF1000F4CBF591AA1F2AE21914277
:10103000B8BF1E2070475749C86070472DE9F05F60
:1010400004460027384614F4803F18BF012014F4EA
:10105000003F18BF40F0040014F4802F18BF40F088
:10106000020014F4002F18BF40F0100014F4001F09
:1010700018BF40F0400014F4800F18BF40F0080083
:1010800014F4000F18BF40F02000DFF80881DFF8EB
:10109000089198F8021010EA0105D9F8400320F4ED
:1010A0008030C9F8400336D0D8F80C60D9F848032E
:1010B000002740F00100C9F84803D9F8480320F0A0
:1010C0000100C9F84803D9F8400340F48030C9F85A
:1010D00040034FF0630ADFF8C4B016E004F033F8C1
:1010E0005046D9F8481311F0010F0AD0D9F844033B
:1010F0000005000D1CBFBBFBF0F0C8F8080001277D
:1011000003E0011EA0F10100EBDC301EA6F1010698
:1011100001DD002FE2D0D9F8500320F00100C9F81A
:101120005003D9F8600320F00100C9F86003D9F832
:10113000680320F00100C9F86803D9F8700320F0B3
:101140000100C9F87003164A106820F00100106011
:101150001448016821F00101016013490B6823F074
:1011600001030B60EFB315F0010F05D0D9F8503330
:1011700043F00103C9F8503315F0040F1AD0D9F821
:10118000703313E05468020004580040F0FE04007D
:10119000E0FE0400208400100050004080F0FA02BD
:1011A000605B0040685B0040705B004043F00103FF
:1011B000C9F8703315F0020F05D0D9F8603343F049
:1011C0000103C9F8603315F0100F05D0D9F8683362
:1011D00043F00103C9F8683315F0400F05D00B68E0
:1011E00000E01CE043F001030B6015F0080F03D092
:1011F000116841F00101116015F0200F03D0016862
:1012000041F00101016088F80150012088F80000D8
:10121000D9F8400340F48030C9F8400321E00020B1
:1012200088F80100ADB1022088F80000D9F8400329
:1012300040F48030C9F84003D9F8480340F0010079
:10124000C9F84803D9F8480320F00100C9F8480359
:1012500007E0D9F8401321F48031C9F8401388F829
:101260000000D9F8400114F0010F20F00D0018BF64
:1012700040F0010014F0040F18BF40F0040014F017
:10128000020F18BF40F00800C9F84001D9F8000269
:1012900014F0100F14BF40F0010020F00100C9F855
:1012A0000002D9F8400214F0200F14BF40F00100F2
:1012B00020F00100C9F84002D9F8C00214F0400F34
:1012C00014BF40F0010020F00100C9F8C002D9F8B5
:1012D000000314F0800F14BF40F0010020F0010063
:1012E000C9F80003FF4814F4805F016814BF41F09F
:1012F000010121F001010160FB4814F4005F016865
:1013000014BF41F0010121F001010160F74814F41C
:10131000804F016814BF41F0010121F0010101601B
:10132000F34814F4004F016814BF41F0010121F0AB
:1013300001010160EF49086814F4807F20F00D007E
:1013400018BF40F0010014F4806F18BF40F0040093
:1013500014F4007F18BF40F0080008600020FFF779
:101360006FFC0120FFF76CFC1120FFF769FC0220E5
:10137000FFF766FC1220FFF763FC4020FFF760FCDC
:101380004120FFF75DFC5120FFF75AFC4220FFF798
:1013900057FCBDE8F05F522052E42DE9F04F84097C
:1013A00000F00F0343EA8411D34D4FEA911CC1F3BF
:1013B000011855F82C6003EB430C06EB8C174FF427
:1013C000A07606EB8818024657F80870002017F040
:1013D000010F10D141F010018F09C1F3011155F82F
:1013E000277006EB811107EB8C17795811F0010F6C
:1013F00008BFBDE8F08F55F82410CF6907F0080842
:1014000001EB8C17D7F80011DFF8F0A204EB440CC5
:101410000AEBCC0C1FFA81F902F00F05002103EB57
:1014200043060CEBC505C2F3011A43EA011242EA76
:101430008412DFF8C4C2C2F3811B5CF82BC0C2F374
:10144000011B4FF4A0720CEB861C02EB8B125CF8B4
:10145000022012F0010F1AD007EB811C55F82A2048
:10146000DCF844B1B8F1000FCBF3080B0EBF4FF01E
:10147000000CDCF844C1CCF3023C02EBC20E0EEBD4
:10148000021200EB42000BFA0CF202FB0900491CAD
:101490000229CAD3BDE8F08F2DE9F0418509AA01E0
:1014A00095489309002450F82300D0F8401111F01A
:1014B000010F34D0914E03EB430306EBC30302F05C
:1014C0000F0603EBC603C2F3011211F0040F53F829
:1014D0002220D0F8003101F0080C9EB2D0F844313F
:1014E000C3F3080318BFC1F30744C769C1F305215B
:1014F00017F0080F1ABFD0F84401C0F302300020E3
:10150000BCF1000F18BF491C03FA00F001FB0040BA
:1015100002EBC201704301EB021100EB4104012018
:1015200040EA8510FFF739FF0646022040EA8510A1
:10153000FFF733FFA1190844BDE8F08110B5002082
:10154000FFF7AAFF4FF47A7148434CF25031B0FBD9
:10155000F1F010BD6A484068C0F30C00704770B5E8
:1015600004460020FFF798FF05464020FFF794FF50
:1015700035B3634BB0B141F288310844A84211D968
:10158000421B186800F01F0104FB01F000EBC00CC7
:101590000CEB0010B2EB400F04D932204843B2FBF1
:1015A000F0F0441CB4F5005F28BF41F6FF7402D28E
:1015B000002C08BF0124586864F30C00586070BD0B
:1015C000B4F5005F28BF41F6FF7402D2002C08BFBB
:1015D00001244C48016864F30C01016070BD2DE9E1
:1015E000F041474F0646386810F01F0508BF012537
:1015F0000020FFF751FFDFF810810446002E18BFCE
:10160000002C3FD0414900204A68002A08BF01222F
:101610003309B3FBF2F1D7F850C31CF0010F1BD014
:10162000B3EB420F1DD33A49B1FBF2F3B6FBF2F133
:101630000A09B3FBF4F1102928BF0F218A4298BF91
:10164000114639B1012984BF01FB1430B0FBF1F020
:1016500007D908E0012109E0B8FBF6F2A24288BFF1
:10166000101B0029F6D0102988BF0F21D7F85C2362
:1016700061F30302C7F85C2332216943B0FBF1F048
:10168000FFF76DFF7868C0F30C00684300EBC00102
:1016900001EB001004EB4000B8FBF0F0BDE8F08176
:1016A00070B5174D0024D5F8500310F0010F08D085
:1016B0001648D5F85C13406801F00F014843040157
:1016C0002EE00020FFF7E8FE02462868696800F077
:1016D0001F00C1F30C01414301EBC10000EB0110FD
:1016E00018E00000005A0040405A0040C05A004034
:1016F000005B00404059004054680200448A0010DA
:1017000000500040045800400008AF2F2084001013
:1017100080F0FA0212EB40001CBFFD49B1FBF0F46F
:10172000204670BD002818BF0120FA49D1F85C237B
:1017300060F30302C1F85C237047F648D0F85C03FD
:1017400000F00F0070478109F34A00F00F0000EB32
:10175000400052F821104FF4807202EB80100858BC
:10176000EE4980B2B1FBF0F0401C400870472DE913
:10177000F041E94B8209DFF8A4C353F8223000F0AE
:101780000F0731B1BCFBF1F1491C4A08B2F5004F1B
:1017900001D347F6FF72BCFBF2F1491C4D08D3F8A8
:1017A00080104FEA520C01F00704D3F88010DA4B96
:1017B0004FEA9018C1F3031600F00F0153F82830D8
:1017C00001EB410103EB81112FB3D1F80431F61C79
:1017D00074439BB2A2EB4404D1F8006124F00104ED
:1017E00062F30F06C1F80061D1F800216CF31F42CB
:1017F000C1F80021D1F8042163F30F02C1F80421DC
:10180000D1F8182164F30F02C1F8182101F0C9F8CA
:101810002846BDE8F081F61CACF10E037443A3EB3F
:101820004404D9E710B48309BB4C10F00F0F00F04B
:101830000F0054F8233000EB40004FF4807404EBA9
:10184000801018584FEA10401CBF10BC7047D3F8E6
:1018500080C00CF00704D3F880C0401AD3F80411FC
:10186000CCF3031C60F30F01C3F80411012A1CBF61
:1018700010BC70470CF103016143A0EB4100D3F8A9
:10188000181120F0010060F30F01C3F8181110BC0B
:1018900070478109A04A00F00F0000EB400052F8A9
:1018A00021104FF4807202EB80100858000C704732
:1018B000830910F00F02984850F8230002EB42030E
:1018C00000EB8313D3F800C161F31F4CC3F800C1D0
:1018D00018BF7047D0F8802002F00703D0F88020AE
:1018E000C2F30312D21C5A430E39A1EB4202D0F8C4
:1018F000043122F0010261F30F03C0F80431D0F883
:10190000181162F30F01C0F818117047824A81095B
:1019100052F8212000F00F0101EB410102EB81118F
:10192000C0F301104FF4A27202EB80100858C0F30C
:1019300008007047F0B4784B840900F00F0C53F89E
:1019400024300CEB4C0503EB8516C0F30112D6F8DE
:101950001C5106EB82164D1BD6F8447161F3080743
:10196000C6F844714CEA021141EA841101F00F02F9
:10197000C1F3011101EB4201694A03F5C07352F84A
:1019800021104A08C90753F822C0C90E40F2FF14BB
:101990008C402CEA040CAD1EC5F3080404FA01F1D6
:1019A0004CEA010143F82210F0BC00F0FABF8309B1
:1019B00000F00F01C0F30112574850F82300C3692B
:1019C00001EB410100EB811013F0100FD0F828114A
:1019D00000EB8210C9B2D0F84401C0F3080008BF80
:1019E0000021401A0004000C08BF012070470309C1
:1019F0001B0203EB810101F1405101F500310007A9
:101A0000C00E0B6802FA00F0184308607047020924
:101A1000120202EB810101F1405101F50031000792
:101A20000968C00E21FA00F000F00300704770B49E
:101A3000DFF8E4C0820900F00F035CF8225003EBEA
:101A40004303C0F301104FF4A87605EB831506EBB2
:101A500080160C68AC515CF82220496802EB8312B6
:101A60004FF4AA7303EB8010115070BC704730B470
:101A7000DFF8A4C0820900F00F035CF8224003EBFA
:101A80004303C0F301104FF4A87504EB831405EB76
:101A9000801564590C605CF8222002EB83124FF42D
:101AA000AA7303EB80101058486030BC70471A4985
:101AB00010B4820983B051F8222000F00F0101EB2D
:101AC000410102EB8111C0F301104FF4A87202EB47
:101AD00080128A5800924FF4AA7202EB80100858C4
:101AE0000190002001466A4601234FEA511C01F093
:101AF0001F0452F82CC003FA04F41CEA040F18BFA8
:101B0000401C491C2629F0D303B010BC70470000CC
:101B10000008AF2F0050004054680200A08601006A
:101B20005C68020030B4002210F00F0F06D000F005
:101B30000F02C0F3011303EB4202521EFE4B800959
:101B40004FF4866553F8204005EBC205D1F800C07C
:101B500044F805C053F8200040F2344303EBC202BE
:101B60004968815030BC704710B4002210F00F0F4C
:101B700006D000F00F02C0F3011303EB4202521E25
:101B8000ED4B80094FF4866453F820C004EBC20487
:101B90005CF804C0C1F800C053F8200040F23443A0
:101BA00003EBC2028058486010BC7047E348C0682D
:101BB00070470022E049830951F82310CB6913F0E4
:101BC000080F0ED000F00F0202EB420201EB82116F
:101BD000C0F301104FF4A27202EB80100858C0F35A
:101BE000023210467047DFF850C310B482095CF827
:101BF0002230DC6944F00804DC615CF8223000F03B
:101C00000F0202EB420203EB8212C0F301134FF406
:101C1000A27000EB8310135861F30E33135010BC05
:101C200070470022C449830951F82310CB6913F08F
:101C3000080F0ED000F00F0202EB420201EB8211FE
:101C4000C0F301104FF4A47202EB80100858C0F3E7
:101C5000024210467047B84A830952F8233000F018
:101C60000F0202EB420203EB8212C0F301134FF4A6
:101C7000A47000EB8310135861F3124313507047A4
:101C8000042988BF70472DE9F0030027DFF8A882F8
:101C9000840958F82430DA69C0F3011C12F0080FE7
:101CA0004FF4A27202EB8C1C00F00F0202EB420216
:101CB00005D003EB821555F80C50C5F30237DD69EA
:101CC000002615F0080F4FF4A475C0F3011005EBC2
:101CD000801504D003EB82104059C0F30246C91BA3
:101CE0007018042803DD081A011D042003E00028F1
:101CF000BCBF014400207E18D96941F00801D961B8
:101D000058F8241001EB821151F80C3066F30E33B1
:101D100041F80C3058F8241001EB82114A5960F355
:101D200012424A51BDE8F0037047834A80090029F6
:101D300052F82000816914BF41F0080121F0080128
:101D4000816170477C49800951F820008069C0F3A7
:101D5000C0007047784A8009002952F82000816944
:101D600014BF41F0020121F0020181617047724904
:101D7000800951F820008069C0F3400070476E4B25
:101D8000820953F8223000F00F0202EB420203EB0B
:101D90008212C0F301104FF4A67303EB80101150B0
:101DA0007047654A810952F8212000F00F0101EBCC
:101DB000410102EB8111C0F301104FF4A67202EB56
:101DC0008010085870475D4A10B4D2F8400110F0F6
:101DD000010F0BD0D2F84C01D2F844110028C1F306
:101DE00002311EBF0029C043C2F84C01012300206C
:101DF00003EB43018C0104EB801101F1804101F5FB
:101E0000A041D1F8402112F0010F0CD0D1F84C21A3
:101E1000D1F844C1002ACCF3023C1EBFBCF1000F34
:101E2000D243C1F84C21401C0228E4D35B1C032B95
:101E3000DDD310BC704700223F49830951F82310BD
:101E4000CB6913F0080F0ED000F00F0202EB420234
:101E500001EB8211C0F301104FF4A47202EB801069
:101E60000858C0F3005210467047012070472DE912
:101E7000F04F82B0022ADDE90B49DDF8348026BF3D
:101E8000921E4FEA520C4FF0000C022B26BF9A1EF6
:101E9000530800232A4AA2FB04421709B8F1000F95
:101EA00014BF012200220192B9F1020F16BF5FEAAE
:101EB00009024FF0010B4FF0000B82091E4C00F09D
:101EC0000F0606EB460554F822404FF4B27E04EBB1
:101ED000851AC0F301140EEB841ECDF800A05AF849
:101EE0000EA061F35C6A6BF3186A05D167F3174AB9
:101EF00063F3CA1A6CF3C60A019969F3420A61F3E3
:101F0000000A0099DFF8309041F80EA059F822201D
:101F10004FF4B471C0F3011A01EB8A1102EB851280
:101F2000B8F1000F555814BF45F0800525F0800525
:101F30005550012506E000005468020000500040A2
:101F4000CDCCCCCCB5EB901F1CBF02B0BDE8F08F60
:101F500004EB4600FC4951F82020183111F820808C
:101F600006EB4600800100EB841000F1804000F594
:101F7000A040D0F85049F549FF26A1FB029149083D
:101F8000A1EB81094A44D2009640FFB297404FEA44
:101F90008802002003F00F0393400CF00F0C4FF069
:101FA0000F090CFA02FC09FA02F24FEA810805FA5D
:101FB00000F1214222D008EBC00101F1804101F57E
:101FC000A041D1F8809C29EA060949EA0709C1F82D
:101FD000809C810001F1804101F5A041D1F8A89CCD
:101FE00029EA020949EA0309C1F8A89CD1F8BC9C76
:101FF00029EA020949EA0C09C1F8BC9C401C0528E1
:10200000D5D302B0BDE8F08F2DE9F04F84B0DDE903
:102010000EA8DDF834C0B8F1000F14BF012400246D
:102020000294BAF1020F16BF5FEA0A044FF0010BE7
:102030004FF0000B8409C64D00F00F0707EB470671
:1020400055F824504FF4B27E05EB8619C0F3011504
:102050000EEB851ECDE9009E59F80E9061F35C6988
:102060006BF318697ED002996AF3420961F30009A3
:10207000DDE9001BDFF8D8A241F80B904FF4B471F2
:102080005AF82440C0F3011901EB891104EB8614BE
:10209000B8F1000F665814BF46F0800626F080069F
:1020A00066500126B6EB901F1CBF04B0BDE8F08F50
:1020B00005EB4700A449A74C51F8201054F82040E4
:1020C00007EB4700800100EB851000F1804000F530
:1020D000A040D0F850099D4DFF26A5FB01756D0865
:1020E000A5EB850739444FEAC109009006FA09FEBD
:1020F00000200F21A400A1404FEA850B012505FA1D
:1021000000F6009D2E4241D01568022D26BFAD1E5F
:102110006D080025121D1E68022E26BFB61E760809
:1021200000265CF8048B8C4FA7FB08874FEA075802
:102130000BEBC00707F1804707F5A047D7F880AC45
:102140004FEA18682AEA0E0A08FA09F84AEA080863
:10215000C7F8808C870007F1804707F5A047D7F8BC
:10216000A88C00E018E006F00F0628EA0108A64057
:1021700048EA0606C7F8A86CD7F8BC6C05F00F054E
:102180008E43A5403543C7F8BC5C1B1D401C052889
:10219000B4D304B0BDE8F08F1168022926BF891EB0
:1021A00049080021D3F800B0BBF1020F26BFABF104
:1021B000020B4FEA5B0B4FF0000BCDF80CB0DFF8D1
:1021C00098B1DCF800E0ABFB0EEB4FEA1B1B6BF3A6
:1021D0001749DDF80CB06BF3CA1961F3C60942E781
:1021E0002DE9F00F5A4D84094FF4B27955F8244087
:1021F00000F00F0505EB450604EB8614C0F301164D
:1022000009EB8619DDE9098754F80940DDF820C09B
:10221000C4F3436BC4F3410904F0010A002918BF59
:10222000C1F800B0B8F1000F18BFC8F80090002F37
:1022300018BFC7F800A081094FF001085BD0B8EBC8
:10224000901F1CBFBDE8F00F704706EB45003E49EC
:10225000404C51F8201054F820B005EB45008001A7
:1022600000EB861000F1804000F5A040D0F850A9A6
:10227000364C0020A4FB015464084FEA8409A4EB07
:1022800084042144CF004FEA8B0508FA00F111EADB
:102290000A0F2AD009EBC00101F1804101F5A041EC
:1022A000D1F8801CF940840004F1804404F5A04476
:1022B000C9B2D4F8A86CD4F8BC4CEE4006F00F06B6
:1022C000EC4004F00F041AB16400A41C42F8044B63
:1022D0001BB17400A41C43F8044BBCF1000F04D0E4
:1022E00001EB810189004CF8041B401C0528CCD36C
:1022F000BDE8F00F7047C4F30740C4F3C311C4F343
:10230000C30412B16400A41C146013B14900891CF9
:102310001960BCF1000F04BFBDE8F00F704700EB7F
:1023200080008000CCF80000BDE8F00F7047084A3C
:102330008009002952F82000C16914BF41F0200132
:1023400021F02001C161704774680200ABAAAAAAFB
:10235000546802008C680200CDCCCCCCF7498009CF
:1023600051F82000C069C0F34010704730B490B0FD
:1023700000224FF48045EC466C1001E0082A05D29B
:10238000531C03EB8303B5FBF3F304E0D31F03EB10
:102390008303B4FBF3F35B1A48BF5B424CF8223073
:1023A000521C102AEAD30023009C01215CF8212052
:1023B000A242BCBF14460B46491C1029F6D300F0BC
:1023C0000F0202EB42014FEA8111C0F3011C01EB45
:1023D0008C1101F18041840901F5A0412AD001242A
:1023E000B4EB901F1EBF10B030BC70470CEB420026
:1023F000D1F850C9D24A12F820200F2591000020B0
:102400008D4003F00F028A4004FA00F111EA0C0F2C
:102410000AD0810001F1804101F5A041D1F8D03C02
:10242000AB431343C1F8D03C401C0528ECD310B09B
:1024300030BC7047D1F8680163F30300C1F868014C
:1024400010B030BC704781091CBF0020704700F0FD
:102450000F0101EB41018901C0F3011001EB801074
:1024600000F1804000F5A040D0F8680100F00F00B6
:10247000082834BF401CC01F00EB800034BF4FF45D
:1024800080414FF40051B1FBF0F070472DE9F007A7
:102490004FF0010991B0B9EB901F1EBF11B0BDE81C
:1024A000F007704700F00F02C0F3011000EB420389
:1024B00002EB4202920102EB8010DFF884C200F1CD
:1024C000804000F5A0405CF82330D0F850A90F20E0
:1024D0004FEA83084FF0000C4FF480466C4600FA38
:1024E00008F709FA0CF010EA0A0F36D051F8043B4D
:1024F00000204FF4005501E0082805D2421C02EBF1
:102500008202B6FBF2F204E0C21F02EB8202B5FBCC
:10251000F2F2D21A48BF524244F82020401C102840
:10252000EAD30025009B012054F820209A42BCBF2A
:1025300013460546401C1028F6D34FEA8C0000F1E4
:10254000804000F5A040D0F8D02C05F00F03BA432E
:1025500003FA08F31A43C0F8D02C0CF1010CBCF1BB
:10256000050FBED311B0BDE8F007704770B4012469
:10257000B4EB901F1CBF70BC704700F00F02C0F39B
:10258000011000EB420302EB42029201DFF8B0C1FE
:1025900002EB801000F1804000F5A0405CF8233091
:1025A000D0F850C900209B004FF480456E1004FA0B
:1025B00000F212EA0C0F16D0820002F1804202F5FE
:1025C000A042D2F8D02CDA4002F00F02082A34BF21
:1025D000521CD21F02EB820234BFB5FBF2F2B6FBF3
:1025E000F2F241F8042B401C0528E0D370BC704780
:1025F00000F00F02C0F3011303EB4202504B8009BD
:10260000A3F1380C53F822205CF8200001230029A4
:10261000D0F8101403FA02F214BF11439143C0F82A
:102620001014704700F00F01C0F3011303EB4101D8
:10263000434B0022800913F82110383B53F8200047
:10264000D0F81004012303FA01F1084218BF012257
:102650001046704770B410F0300F14BF01230023F0
:102660008609DFF8D8C000F00F024FEA90104FF44F
:102670009A7502EB42025CF820004FF0010405EB72
:10268000821214D085584FEA430C5B420CEB430393
:102690009B1C04FA03F35B1E03FA0CF4194025EAB1
:1026A000040401FA0CF12143815070BC70470029E9
:1026B000815804FA03F31ABF194381509943F3D0A8
:1026C00070BC704730B410F0300118BF012184098C
:1026D0004FEA9013194D00F00F0000EB40004FF44B
:1026E0009A7202EB801255F823004FF0010C0CD0C7
:1026F00082584800C240494200EB4100801C0CFA5D
:1027000000F0401E30BC1040704780580CFA01F1B8
:10271000084018BF012030BC7047084B800953F8AF
:1027200020C0CCF8741053F820C01168CCF8781091
:1027300053F820005168C1677047000054680200D8
:102740008C680200C0490028D1F8AC0014BF40F0EA
:10275000020020F00200C1F8AC007047BA4900281E
:10276000D1F8AC0014BF40F0010020F00100C1F826
:10277000AC007047B448D0F8E000B4490968084399
:102780007047B149C1F8E400B14908607047AE48EC
:10279000D0F89800AF49096840EA4100704770B42A
:1027A0004FEA0075860900F00F044FEAD565C0F3C3
:1027B0000110A5F1020502F0010C05444FEA8C332B
:1027C0004FEA520012D001EB41017CB305EB450208
:1027D000D20002EB8C3202EB810101EB800000F1B0
:1027E000405000F5C030406A70BC704701EB4102B8
:1027F00002EB01117CB198226A4302EB8C3202EBAE
:10280000810101EB800000F1405000F58030D0F8EC
:102810008C0E70BC704703EB810101EB800000F16E
:10282000405000F58030006870BC7047FFE703EB54
:10283000810101EB800000F1405000F5C0300068DC
:1028400070BC7047F0B44FEA0076870900F00F04BF
:102850004FEAD666C0F30110A6F1020602F0010CA1
:1028600006444FEA8C354FEA520012D001EB410189
:102870007CB306EB4602D20002EB8C3202EB810104
:1028800001EB800000F1405000F5C0304362F0BC25
:10289000704701EB410202EB01117CB198227243B7
:1028A00002EB8C3202EB810101EB800000F1405021
:1028B00000F58030C0F88C3EF0BC704705EB81011C
:1028C00001EB800000F1405000F580300360F0BC67
:1028D0007047FFE705EB810101EB800000F14050FC
:1028E00000F5C0300360F0BC7047830900F00F02B0
:1028F000C0F301100CD0002A08BF574805D0012AA8
:1029000017D000280CBF5548554800EB8130704760
:10291000002A08BF4FF04050F7D0012A04D0002809
:102920000CBF50485048F0E7002814BF4F485048AB
:10293000EBE7002814BF4F484F48E6E710B44FEAD2
:10294000007C840900F00F034FEADC6CC0F3011037
:10295000ACF1020C604410D0002B08BF47481CD0DB
:1029600000EB4000C00000EB813002EB420100EBC5
:102970008100434910BC08447047002B08BF414800
:102980000BD09823584300EB813002EB420101EB5E
:10299000021100EB81003C49ECE710BC00EB8130F8
:1029A00070472DE9F0074FEA901C00F00F043748FC
:1029B00004EB440150F82C0000F5C07300EB8110CB
:1029C000D0F800014FF47A7280B2B2FBF0F100FB54
:1029D0001120002818BF01200D182D4F002040F2B3
:1029E000FF1644EA001141EA8C1101F00F02C1F315
:1029F000011101EB420157F821104A08C90753F8A9
:102A00002280C90E03EB820228FA01F8D2F80CA04A
:102A1000A8EB050906FA01F8C9F308092AEA080A29
:102A200009FA01F14AEA0109C2F80C90D2F81890AB
:102A300029EA080848EA01019161401C0228D0D324
:102A4000BDE8F0077047000000500040E05800402B
:102A5000E45800409858004000800030E481003085
:102A6000248300304C1800304C1D0030CC0E003058
:102A7000CC090030648100302480003000800130B7
:102A800024800130000001308C0E013054680200B7
:102A90005C680200FDF7C2BF10B5FDF7BFFF01285B
:102AA00018BF10BD0020FDF774FF21210020FDF7A5
:102AB000BBFF2121BDE810400120FDF7B5BF10B5D7
:102AC000FDF760FFFDF7AAFF01280AD10020FDF7FE
:102AD00060FF21210020FDF7A7FF21210120FDF744
:102AE000A3FF0121052001F022FD0121052001F0B5
:102AF0001EFDFF490020487110BD10B54FF406605F
:102B000001F06BFDBDE810404FF4066001F056BDCA
:102B1000F74A0146D078002818BF0120002918BFC5
:102B20000121D170002111717047F14A516A506240
:102B300008467047EE490020887048707047EC499D
:102B4000002088704870704770B50007C00E0D46B1
:102B5000801E00EB400101EB0014E6484FF4987230
:102B600000EBC40029460BF07FFAE34805F59871A5
:102B700000EBC400BDE870404FF498720BF074BADB
:102B8000DFF878C348B14A424FF4806300EB81011B
:102B900003EB820260460BF067BA4FF48061604637
:102BA0000BF067BA2DE9F04105460020FDF77AFFEA
:102BB000D34FDFF850830446EDB14C2004FB00F204
:102BC0001646294638460BF04FFA324605F5E461C1
:102BD00040460BF049FA04EB440000EB041407EB09
:102BE00084004C210BF045FA08EB8400BDE8F0416D
:102BF0004C210BF03EBA4C21401C41430C46384658
:102C00000BF037FA21464046BDE8F0410BF031BAEF
:102C100010B5B74CE061FEF711FAFEF7CAF9616929
:102C20006269C1F307216FF30F0262616369C2B287
:102C300043EA02226261022803D1626942F0010282
:102C4000626181421ABFA269002A10BD012918BF22
:102C50000021012818BF0020814208BF10BDBDE837
:102C6000104010474FF04020816941F0020181611E
:102C7000016941F00301016100F0E7BE2DE9F04177
:102C80004FF04022054690690C4640F002009061EA
:102C9000116941F00300106100F0D7FE0027002CFD
:102CA0007DD00020FDF775FE00202168FEF766F854
:102CB00040206168FEF762F82846FFF7A9FF002070
:102CC000FDF721FF0126002832D0A068FFF76AFF38
:102CD0008A48636953B1E169B202C1F1000C02EBA9
:102CE0008C0203EB81010BF0BFF91AE0864D4FF423
:102CF00080610BF0BEF90020295600290EDB0A097D
:102D0000120202EB800202F1405202F50032090782
:102D1000C90E136806FA01F119431160401C2628F8
:102D2000EAD37A48A16969B14FF400720BF09CF9BB
:102D3000E068A0B30120FDF7E6FEDFF8B8816E4E33
:102D400028B108E04FF400710BF093F9F0E711207F
:102D5000FDF7D9FE68B1E56840464FF49872294600
:102D60000BF082F930464FF4987205F598710BF02C
:102D70007BF90220FDF7C7FE18B91220FDF7C3FE4C
:102D800068B1E46862484FF4987221460BF06CF920
:102D900060484FF4987204F598710BF065F9544847
:102DA000877047704762C1780021C17007714FF486
:102DB000066001F012FCBDE8F0414FF4066001F03E
:102DC000FDBB10B50020FDF7E4FD00F02EFE4848E5
:102DD000806B002808BF10BD4FF04020016921F032
:102DE00003010161816921F00201816110BD4FF48D
:102DF000066001F0E8BB10B54FF4066001F0E3FB9C
:102E0000FDF70CFE01280AD10020FDF7C2FD2121AB
:102E10000020FDF709FE21210120FDF705FE3E48B7
:102E2000D0F8401321F48031C0F840130020FDF7A2
:102E3000B0FD00F0FAFD2E48806B002808BF10BDE1
:102E40004FF04020016921F003010161816921F007
:102E50000201816110BD10B501F0BAFB10F06000F5
:102E600018BF012010BD224A916990610846704741
:102E70001F48C06970471E484069704772B61C49B8
:102E80004A6922EA0000486162B670471848007833
:102E9000002818BF0120704770B5FDF7BFFD00285E
:102EA00018BF70BD0024124DAC706C7021212046FB
:102EB000FDF7BAFD21210120FDF7B6FD2C70BDE81C
:102EC00070400120FDF765BD70B50446FDF7A6FD15
:102ED000002818BF70BD0021054DA970697021211F
:102EE0000020FDF7A1FD21210120FDF79DFD15E04A
:102EF000308400108C0E01308C4E01300000023006
:102F00000000013000400130748A0010004002309F
:102F1000BC0F0130BC4F013000500040022C3CBFC0
:102F20000120FDF791FD012028702C62BDE8704062
:102F3000FDF72FBD10B5FDF771FD002818BF10BDBE
:102F40000020F84CA07060702121FDF76DFD21215B
:102F50000120FDF769FD0120FDF776FD01202070BD
:102F60002062BDE81040FDF714BD0020FDF711BD43
:102F700010B5EC4C0020A07060702121FDF754FDCD
:102F800021210120FDF750FD207800281CBF0120E1
:102F9000FDF75AFD0120BDE81040FDF7FABCE149FC
:102FA00088627047DF48806A7047DE49C8627047B0
:102FB000DC48C06A7047DB4A00F00F00D16A21F09C
:102FC0000F010843D0627047D64890F82C0000F0FB
:102FD0000F007047D34948637047D248406B704731
:102FE000D04908637047CF48006B704770B5CD4C2F
:102FF0000546A06A421CA262E16A11F0800F14BF6C
:10300000C1F3021101F00F0139B1B2FBF1F001FB84
:103010001020002808BFFEF7D6FE207850B1206AA5
:1030200010B1206A401E2062206A002804BF0020E0
:10303000FDF7AFFC20212846FDF7F6FCFDF7BCFFAD
:1030400010F0010F07D0FDF7DAFF216B091A18BF46
:10305000012161632063616A00291CBF28468847FB
:10306000FDF7A7FF022815D1AF48D0F8481311F09B
:10307000010F0FD0D0F8481341F00101C0F84813F8
:10308000D0F8481321F00101C0F84813606940F0FE
:1030900002006061A548016841F02001016070BD37
:1030A0000020A3E70120A1E710B5FFF763FB04466A
:1030B000FFF767FB9E48044208BF10BD994841696D
:1030C00041F0040141610E2101EAD43104F0010212
:1030D0000A43416962F31F4141619448016841F02C
:1030E0002001016010BD002818BF01208D498863B0
:1030F000704790487047904870478A48C06B704747
:1031000088488179027A914214BF006C406C704704
:103110008448406C70472DE9F04F0025DFF8149289
:103120008DB009F14C04AC466F1E09F8057004F827
:1031300005C06D1C262DF8DB0025002805DD565D39
:1031400009F805606D1CA842F9DC00220126CDF8C3
:1031500004C06D46CDF800C0002821DD19F902B089
:10316000BBF1000F19DBBBF1140FA8BFABF1140BBF
:1031700004DABBF10A0FA8BF0BF1120BBBF1260F4B
:103180000BD24FEA5B180BF01F0B55F828A006FA7C
:103190000BFB4AEA0B0A45F828A0521C8242DDDBF1
:1031A000002292460DF108084FEA521B02F01F0E52
:1031B00055F82BB006FA0EFE1BEA0E0F1ABF08F8E0
:1031C00002A00AF1010A08F80270521C262AEBDB61
:1031D0004FF0000A002816DD19F90A20002A0EDB3C
:1031E000142AA8BF143A02DA0A2AA8BF1232262AE1
:1031F0003ABF18F8022004F80A2004F80A700AF10D
:10320000010A8245E8DBDFF81C9100220028C9F89A
:103210003CC009DD14F902A0924502D0C9F83C4037
:1032200002E0521C8242F5DB444A0020A2F1720403
:10323000A2F1260A27540AF800C002F800C0401C78
:103240002628F7DB0020002906DD13F800B004F87B
:1032500000B0401C8142F8DC0020CDF804C0CDF85D
:1032600000C0002913DD2356002B0DDB262B0BD2CB
:103270004FEA531B03F01F0355F82BE006FA03F344
:103280004EEA030345F82B30401C8842EBDB00205C
:1032900003464FEA501B00F01F0E55F82BB006FAFC
:1032A0000EFE1BEA0E0F1ABF08F800305B1C08F870
:1032B0000070401C2628ECDB002000290ADD235684
:1032C000002B04DB262B3CBF18F803301354401CA2
:1032D0008842F4DB0020C9F844C0002908DD1356F9
:1032E000834202D0C9F8442002E0401C8842F6DB49
:1032F00011F0010F18BF252024D0420900F01F0350
:1033000055F8222006FA03F31A4219D1420900F0B7
:103310001F0055F8223006FA00F0184345F8220045
:1033200010E0000030840010005000407C84001049
:1033300001000700748A00109A8A00100C8B00109C
:10334000401EDAD500200246430900F01F0B55F855
:10335000233006FA0BFB13EA0B0F1ABF08F8002004
:10336000521C08F80070401C2628EDDB00200029C4
:103370000BDD2256002A05DB262A3CBF18F8022066
:103380000AF80020401C8842F3DB0020C9F840C046
:103390000029DCBF0DB0BDE8F08F1AF90020824291
:1033A00004D0C9F840A00DB0BDE8F08F401C8842A1
:1033B000F3DB0DB0BDE8F08F40F2DB114843FE496E
:1033C00001EB80007047FD49C0EB001001EBC0002D
:1033D0007047DFF8ECC3012B8CF806008CF807105F
:1033E00003D9401C20F0010011468CF808008CF82D
:1033F000091000FB01F24FF6FF7101EA4202ACF83E
:10340000102001EA4000ACF812007047EC48407A06
:103410007047EB48007A7047E94A9072D172704762
:10342000E748C07A7047E648807A7047E54A1070EE
:1034300051707047E349085C70472DE9F047DFF8A9
:103440008093044699F80300002804BF99F801000E
:103450000AF014FE0AF0FFFC28B9002301227F21A4
:1034600007200EF019FD99F80400002808BFBDE8F8
:10347000F0870027D9F81C003E463D46B84610F0BC
:10348000070F1CBFCC4F10F0020F05D0B9F8101079
:10349000C94A21F001018E1810F0F00F18BFC74D76
:1034A000D9F828002060FDF787FD10F0010F06D045
:1034B000FEF743F9022828BF99F8020000D2002045
:1034C000C4F81480C4E90107C4E903650120BDE81C
:1034D000F087BB4900200871704770B50546002091
:1034E000FDF7E0FA4C2100FB01F21446B6492846EC
:1034F0000AF0BAFD224605F5E460BDE87040B34924
:103500000AF0B2BDF0B583B00020FDF7CBFA044657
:1035100069460020FEF7ABFA0022002C2AD96E463D
:103520004FF0010C4FF6F07502EB4200002100EB6A
:1035300002104B0901F01F0756F823300CFA07F769
:103540003B4211D0CB075B0C03EB80034F0803EB2E
:10355000870303F1405303F580331B889BB2AB42D2
:1035600002D903B00020F0BD491C2629E1D3521C2A
:10357000A242D9D303B00120F0BD70B50007C00E40
:103580000D46801E00EB400101EB001490484FF403
:10359000987200EBC40128460AF066FD8D484FF48E
:1035A000987200EBC40105F59870BDE870400AF010
:1035B0005BBD2DE9F04F07460007C00E83B0801EAB
:1035C000002527F03F0BE9464FF001084FF6F07653
:1035D0000290384665F31F1040EA0B0000F0FF0A26
:1035E0005046FDF790FA00283DD05046FEF7E1FA2C
:1035F00008FA00F4022C88BF022469465046FEF700
:1036000036FA0022002C2ED902989821284400FB7B
:1036100001FA02EB4200002100EB021C480901F014
:103620001F0359F8200008FA03F3184215D001F0DF
:1036300001000AEB803000EB8C004B0800EB8300AC
:1036400000F1405000F58030B0F88C0E80B2B042EE
:1036500003D903B00020BDE8F08F491C2629DDD333
:10366000521CA242D5D36D1C022DB2D303B001204F
:10367000BDE8F08F2DE9F0410026514D00280C46A1
:1036800045D000F00F01C0F3011001290EBF002149
:103690000229BDE8F081022828BFBDE8F0810F189B
:1036A000FDF7BCF95FEA00081CBF0020FDF771F9C7
:1036B00000239820474303EB4300002200EB031C48
:1036C00002F0010007EB8030510800EB8C0000EBAA
:1036D000810000F1405000F58030521CC0F88C4E43
:1036E000262AEDD35B1C022BE5D3B8F1000F08BFEF
:1036F000BDE8F081AE706E7021210020FDF794F9D5
:1037000021210120FDF790F92878A0B330E0FDF7E2
:1037100085F907001CBF0020FDF73BF9002303EBF0
:103720004300002200EB0310D107490C4FEA520C72
:1037300001EB800101EB8C0C0CF1405C0CF5803C42
:10374000521CCCF80040262AEED35B1C312BE6D36A
:10375000002F08BFBDE8F081AE706E7021210020FF
:10376000FDF762F921210120FDF75EF9287810B1FB
:103770000120FDF769F9BDE8F0410120FDF709B925
:1037800010B5FEF714F90E49C88110BD0C4B10B4EA
:10379000E02101EA102CDB89C1B2C0F30422994276
:1037A00088BF194664246143B1FBF3F102EBC20305
:1037B00003EB021210E0000074160110E01D01106E
:1037C000308400103C8400100000013000400130C3
:1037D0008C0E01308C4E013001EB82014FF47A7275
:1037E0003D4B0CFB02F2A3FB02329208521C520822
:1037F00010F4803F08BF494210F4003F14BF8818FE
:10380000881A00B210BC704710B5344C4FF4806178
:1038100033480AF02EFC002001232156002910DB3A
:103820000A09120202EB800202F1405202F5003254
:103830000907C90ED2F800C003FA01F14CEA0101F0
:103840001160401C2628E8D310BD10B5234C4FF45E
:10385000806123480AF00DFC002001232156002935
:1038600010DB0A09120202EB800202F1405202F55B
:1038700000320907C90ED2F800C003FA01F14CEA80
:1038800001011160401C2628E8D341F2EC011548E3
:103890000AF0EFFBBDE8104041F2EC0112480AF0DB
:1038A000E8BB124810B5C06911490840FFF7B0F9EC
:1038B0004FF480610A480AF0DCFB40F68C6109484D
:1038C0000AF0D7FB40F68C6107480AF0D2FBBDE84E
:1038D00010400020FDF743BEABAAAAAA748A0010CC
:1038E0000000023000000130004001303084001040
:1038F0000100FF0082B04FF4FA62009013E000BFB5
:1039000000BF00BF00BF00BF00BF00BF00BF00BFBF
:1039100000BF00BF00BF00BF00BF00BF00BF0198D5
:10392000411E0191EBD20098411E009128BF0192E7
:10393000F5D202B070472DE9F0410027634D012612
:10394000002808BF2E701FD001282F7018BF6F707D
:103950001AD04FF04028D8F8100040F00400C8F802
:10396000100029785A4C002914BF49F608305948EC
:10397000E06014BF58484FF0BB70A0605748006823
:1039800030F0FF0206D101E06E70E2E7E26860F31A
:103990000302E26089B1A06840F01800A060012035
:1039A000FFF7A8FFA06840F48050A0600120FFF757
:1039B000A1FFA06840F40070A0600120FFF79AFF0B
:1039C000687870B1E06840F02000E060A06820F402
:1039D0000070A0600120FFF78DFFE06840F010004C
:1039E000E060D4F8B00040F00100C4F8B00001205D
:1039F000FFF780FFE6674FF4E0602061C4F888704D
:103A00002878002818BFC4F89460E06820F03000DF
:103A1000E060A06820F49050A060D8F8100020F07A
:103A20000400C8F81000BDE8F0812948C16821F001
:103A30003001C160816821F4905181604FF04020D5
:103A4000016921F00401016170474FF040200169D4
:103A500041F0040101611D491D480A783AB18268AC
:103A600042F018028260826842F490528260497883
:103A700019B1C16841F03001C160D0F8B01041F017
:103A80000101C0F8B0107047B0F5007F28BF40F2C8
:103A9000FF10C0F30800124941EA00200C490864F5
:103AA00070470B494FF0204008647047084A116C7A
:103AB0004FF020401064506C11F0FF0FC0F308204D
:103AC0001CBF41F020411164704700007884001051
:103AD0000060004005F4010020009B00D0FE0400BF
:103AE000130000A04FF04020002101630222426336
:103AF000826B02F03C0242F001028263026922F012
:103B000003020261026A22F001020262424A136861
:103B100043F0010313603C2282612822C2613F48C6
:103B200001603F4801603F4850F88C2F42F48052BA
:103B300002603D4A481E10603C480160704710B565
:103B400001F0F9FA39480468002C08BF30BFFAD0F8
:103B50000021016001F0F3FA204610BD10B501F01C
:103B6000EAFA324B00204FF0402101221C6824B1B8
:103B7000186001F0E4FA204610BD72B6D1F838C0E2
:103B80000CF03C0CC1F838C00A6320BF0863D1F8C0
:103B900038C00CF03C0C4CF0010CC1F838C062B6D7
:103BA000BFF36F8FBFF34F8FE0E710B504460F20D0
:103BB00000F0F8FC0F2000F0DDFC1D490A6842EA25
:103BC0000400086010BD1A490A6822EA0000086073
:103BD0007047164A516850600846704770B51448DF
:103BE000006814490968114D00EA01046968002958
:103BF0001CBF2046884714F0100F05D0094850F824
:103C00008C1F41F48051016007480460286840F42B
:103C10000040286070BD000000480040244800407B
:103C20001048004000300040144800407C840010E0
:103C30001C48004018480040704770470022B2EB13
:103C4000D10F26D20368B3F1FF3F04BF4368B3F13D
:103C5000FF3F17D18368B3F1FF3F04BFC368B3F1DF
:103C6000FF3F0FD10369B3F1FF3F04BF4369B3F1D5
:103C7000FF3F07D18369B3F1FF3F04BFC369B3F1CD
:103C8000FF3F01D0002070472030521CB2EBD10F13
:103C9000D8D30120704710B40023B3EBD20F30D239
:103CA000D0F800C00C68A44522D1D0F804C04C68FC
:103CB000A4451DD1D0F808C08C68A44518D1D0F80F
:103CC0000CC0CC68A44513D1D0F810C00C69A44531
:103CD0000ED1D0F814C04C69A44509D1D0F818C051
:103CE0008C69A44504D1D0F81CC0CC69A44502D08D
:103CF00010BC00207047203020315B1CB3EBD20F8A
:103D0000CED310BC012070472DE9F041054601F0EB
:103D10001AFA002021264FF4825784464FF4E022FD
:103D20001660C5F800C0116841F004011160116807
:103D300011F0040FFBD1176080232C460021D4F82A
:103D40000080B8F1FF3F04BFD4F80480B8F1FF3F12
:103D50001DD1D4F80880B8F1FF3F04BFD4F80C801F
:103D6000B8F1FF3F13D1D4F81080B8F1FF3F04BF82
:103D7000D4F81480B8F1FF3F09D1D4F81880B8F115
:103D8000FF3F04BFD4F81C80B8F1FF3F08D0C2F851
:103D900000C0401CC0B20828C2D30220BDE8F08198
:103DA000491C2034B1EBD30FC9D3C2F800C00120A5
:103DB000BDE8F0812DE9F041054601F0C4F900208D
:103DC000092684464FF4E0231E60C5F800C0196838
:103DD00041F004011960196811F0040FFBD12C4661
:103DE0004FF4806200212768B7F1FF3F04BF676886
:103DF000B7F1FF3F17D1A768B7F1FF3F04BFE768EE
:103E0000B7F1FF3F0FD12769B7F1FF3F04BF6769E3
:103E1000B7F1FF3F07D1A769B7F1FF3F04BFE769DB
:103E2000B7F1FF3F08D0C3F800C0401CC0B2032860
:103E3000CAD30220BDE8F081491C2034B1EBD20F77
:103E4000D1D3C3F800C00120BDE8F0812DE9F05FB7
:103E50008846814604274FF07F0A4FF0020B4FF44B
:103E6000E02601F070F94946424653464FF0060CF1
:103E7000C6F800B052F8040B41F8040BC6F800C0B5
:103E8000306810F0040FFBD15B1EF1D200203060CF
:103E90004C4645461F20D4E900C3D4E90221D5F899
:103EA00000E0E64504BFD5F804C09C4505D1AB68E9
:103EB000934204BFEA688A4208D07F1E03D3484673
:103EC000FFF722FFCDE70220BDE8F09F1034103548
:103ED000401EE0D20120BDE8F09F70B50D460446BB
:103EE00001F031F94FF40072214628460AF0BCF87F
:103EF000012070BD2DE9F0410546C005ADF5007DFE
:103F000014460E46C00D25D0A8466FF308086F462C
:103F100001F019F94FF40072414638460AF0A4F84E
:103F2000C5F30800C0F50077A74288BF274668445C
:103F30003A4631460AF0A7F84046FFF7E5FE022868
:103F400044D069464046FFF781FF022843D03D44F4
:103F50003E44E41BB4F5007F19D34FF400723146A0
:103F600068460AF090F82846FFF7CEFE02282DD0CA
:103F700069462846FFF76AFF02282CD0A4F5007492
:103F800005F5007506F50076B4F5007FE5D2C4B1FD
:103F90006F4601F0D8F84FF40072294638460AF00F
:103FA00063F82246314668460AF06DF82846FFF766
:103FB000ABFE02280AD069462846FFF747FF0228D1
:103FC00009D00DF5007D0120BDE8F0810DF5007DE3
:103FD0000A20BDE8F0810DF5007D0B20BDE8F081E1
:103FE00030B4354D2A68002101244FF0030C04FA47
:103FF00001F3034204D04B000CFA03F39A431A4333
:10400000491C0C29F3DB2A6030BC7047F0B42A4D00
:104010002A68002101244FF0030C022604FA01F360
:10402000034206D04B000CFA03F7BA4306FA03F337
:104030001A43491C0C29F1DB2A60F0BC70472DE9BA
:10404000F001002201251D4C0F2605FA02F3034260
:1040500017D0D31702EB537C4FEAEC0304EB830336
:104060001F682CF0070CA2EB0C0C4FEA8C0C06FA24
:104070000CF827EA080701FA0CFC47EA0C0CC3F815
:1040800000C0521C0C2AE0DB0B498A6A22EA0000BD
:104090008862BDE8F001704707498A6A1043886268
:1040A00070470548416821F080014160416821F472
:1040B0000071416070470000001000402010004077
:1040C000704772B64FF04020816941F04001816134
:1040D000C16941F04001C16162B6016A41F001016C
:1040E000016270474FF04020016A21F00101016236
:1040F00072B6C16921F04001C161816921F04001BE
:10410000816162B6704710B572B64FF04024A06965
:1041100040F04000A061E06940F04000E06162B61C
:10412000206A40F001002062D94843F63F71C16027
:10413000002181638164C0F8D01003210A2000F0BF
:10414000F6F90A2000F016FA206A20F00100206239
:1041500072B6E06920F04000E061A06920F0400004
:10416000A06162B610BDCA4A1060516048439060B9
:104170007047C74A10605160484310F0010F18BFE4
:10418000401C90607047C249C1F8D0007047C049D8
:10419000002818BF012088647047BD498863C8683B
:1041A00040F00200C8607047DFF8E4C2CCF820009D
:1041B000CCF82410CCF82820CCF82C300120CCF8F6
:1041C0003000DCF8340010F0010F05D020BFDCF81F
:1041D000340010F0010FF9D110F0020018BF4FF0B9
:1041E000FF307047AA48C16821F00201C1607047E2
:1041F000A748C16841F00101C1607047A44B186233
:1042000059629A6201201864586C10F0010F04D0B2
:1042100020BF586C10F0010FFAD110F0060018BF43
:104220004FF0FF3070479A48C16821F00101C1602A
:1042300070479748C16841F00401C1607047944AD3
:104240008189116701685162416891628168D16218
:1042500001211165516D11F0010F04D020BF516D86
:1042600011F0010FFAD1536F0361936F1B14838216
:10427000936FC3F30523C382936F03F03F0303835C
:10428000D36F1B144383D36FC3F305238383D36F8F
:1042900003F03F03C383D2F88030C3F309430384A0
:1042A000D2F88020C2F30902428411F0020018BF44
:1042B0004FF0FF3070477648C16821F00401C160BB
:1042C00070477348C16841F00401C1607047027CC7
:1042D000017B02F03F0241EA02416D4A91650168AB
:1042E0005162416891628168D16201211165516D0D
:1042F00011F0010F04D020BF516D11F0010FFAD160
:10430000D36D8382D36D1B0CC382136E0383136E34
:104310001B0C4383536E8383526EC2F30E42C283DF
:1043200011F0020018BF4FF0FF3070475848C168C5
:1043300021F00401C16070475548C16841F008018F
:10434000C1607047DFF848C1CCF89820CCF8200055
:10435000CCF82430CCF828100120CCF89000DCF800
:10436000940010F0010F05D020BFDCF8940010F08D
:10437000010FF9D110F0060018BF4FF0FF30704761
:104380004348C16821F00801C160704701684FEAE5
:1043900031423F49C1F8BC204068C1F8C000C8683C
:1043A00040F02000C860704701684FEA3142384948
:1043B000C1F8BC204268C1F8C020027A407A02F0FD
:1043C000010262F35F00C1F8C400C86840F0200039
:1043D000C86070472E4B18625A6299620120C3F878
:1043E000B400D3F8B80010F0010F05D020BFD3F807
:1043F000B80010F0010FF9D110F0060018BF4FF00F
:10440000FF307047224A106251620120C2F8B000AA
:10441000D2F8B80010F0010F05D020BFD2F8B800D4
:1044200010F0010FF9D110F0060018BF4FF0FF3067
:1044300070471748C16821F02001C16070471448D7
:10444000C16841F01001C1607047A3F1050C104B29
:10445000C3F8A8C018625A6299620120C3F8A0008C
:10446000D3F8A40010F0010F05D020BFD3F8A400AA
:1044700010F0010FF9D110F0060018BF4FF0FF3017
:1044800070470348C16821F01001C1607047000007
:1044900000900040234810B5022140F8501F012130
:1044A00001611021416241F20601416100218161F7
:1044B0000421816390214163416B41F0010141631B
:1044C000C16B21F40021C163C16B41F40051C16390
:1044D000C16B21F00101C163C16B41F00101C163F6
:1044E0004FF4817101610161032000F043F8002164
:1044F000032000F01CF8002010BD10B5032000F0D0
:1045000045F808484FF480710166002101661021CA
:10451000816702214165002010BD03490020087019
:10452000704700000030004084840010704700F0A5
:104530000303DA004FF0FF0C0CFA02F24FF0050C07
:104540000CEBC30301FA03F300F00C0101F1E021CD
:10455000002807DAD1F8140D90431A401043C1F82F
:10456000140D7047D1F8000490431A401043C1F86D
:104570000004704700F01F01012202FA01F1400916
:10458000800000F1E020C0F80011704700F01F012A
:10459000012202FA01F14009800000F1E020C0F898
:1045A0008011704700F01F01012202FA01F1400959
:1045B000800000F1E020C0F8801270474FF0E02149
:1045C000C1F8000170474FF0E021C1F88001704749
:1045D0004FF0E020D0F8000170474FF0E021C1F823
:1045E00080027047084800687047074A11681060E9
:1045F00008467047044A126800F1100352F823007D
:1046000042F823107047000008ED00E002210C2062
:10461000FFF78DBF72B64FF04020816941F48051A1
:104620008161C16941F48051C16162B6704772B65F
:104630004FF04020816921F480518161C16921F4EA
:104640008051C16162B67047AA4881B0016F11F410
:10465000007FFBD1816E11F0010F1CBFD0F88410D8
:10466000009104D0D0F88410009A9142FAD0016FE2
:1046700011F4007F04BF4CF27101016642F2413136
:10468000816601B070479B4981B04FF40D528A6634
:104690000A6FCA66012898BF012005D9401EB0F5EF
:1046A000803F28BF4FF6FF7082B24FF05C5040EA67
:1046B000022048664FF01140C1F88000086F10F4E6
:1046C000007FFBD1886E10F0010F1CBFD1F8840071
:1046D000009004D0D1F88400009A9042FAD0086F7C
:1046E00010F4007F04BF4CF27100086642F24130C2
:1046F000886601B070477F4881B0016F11F4007F78
:10470000FBD1816E11F0010F1CBFD0F88410009115
:1047100004D0D0F88410009A9142FAD04FF40D5191
:10472000816601B070474FF04020806910F48050DE
:1047300008BF70476F48806E00F0010070476D48F9
:10474000406EC0F30F2070476A48D0F8840070476D
:1047500010B50C20FFF726FF0C20FFF70BFF654973
:104760000220486710BD634910B5032088670C20FC
:10477000FFF70CFFBDE810400C20FFF713BF5E4AA7
:1047800011681060084670475A4810B5016FC1663D
:1047900059480068002818BF80475848016841F40C
:1047A0008051016010BD54484068704710B572B622
:1047B0004FF04020816941F480518161C16941F429
:1047C0008051C16162B603204A4988670C20FFF717
:1047D000DDFE0C20FFF7E6FE00F03CF9484B04201C
:1047E000C3F888004FF6FF70C3F88C0072B66033D0
:1047F000FFF749FF4FF40070186062B610BDF8B5BE
:1048000072B63C48016F11F4007FFBD1816E11F04C
:10481000010F1CBFD0F88410009104D0D0F8841090
:10482000009A9142FAD04FF40D51816634494FF409
:1048300000320A6662B6D1F804124FF04025002912
:1048400046D02D4C4FF6FF73591AA1602A6BD5F84C
:1048500034C002F00F020CF00F0C6244121D01FA7A
:1048600002F2A2F54341DFF89CC0513961452FD2D5
:10487000D0F88400191AE160B1F5803F28D2224BAC
:104880004FF0000CA1FB03070CFB037301FB0C3181
:10489000634609F0FDFB401C40082061B0F57A7FBB
:1048A00038BF4FF47A70194B9968002908BF986097
:1048B0005A681A609968C3E901108A4215D9824280
:1048C00005D9814201D9616002E0606000E0626068
:1048D00000F0D0F872B6A86920F48050A861E869A9
:1048E00020F48050E86162B6F8BD8242EFD8814280
:1048F000EBD8E8E700C00040888400107C840010FA
:1049000000A000404F62250000E1F505348B001047
:104910004FF04020816941F0040181610C48016839
:1049200041F404710160001F016821F0040101607D
:10493000016841F010010160704706490860704746
:10494000BFF34F8F054904480860BFF34F8FFEE760
:1049500014ED00E008ED00E00400FA050CED00E0C5
:104960004FF04020816941F0040181610B480168EA
:1049700041F0010101600B490948C1F8C4007047CA
:104980000948006842F2700108407047084807492A
:104990000160084981600021C1607047144C0040EB
:1049A00001005FA00060004000440040A0C00E0075
:1049B00000100040508A5900022824BF0020704790
:1049C000DC4B53F8202043F820101046704770B598
:1049D000D94C206FD74D10F0010F05D00120E066B3
:1049E0002868002818BF8047206F10F0020F08BF0A
:1049F00070BD0220E0666868002808BF70BDBDE891
:104A00007040004710B572B64FF04020816941F008
:104A100080018161C16941F08001C16162B60222F9
:104A2000C5490A6501230B660323CB664A6572B646
:104A3000816921F080018161C16921F08001C1613A
:104A400062B60920FFF796FD0221BDE8104009205B
:104A5000FFF76DBD72B64FF04020816941F08001D3
:104A60008161C16941F08001C16162B60220B24931
:104A700008657047B0490220486572B64FF0402083
:104A8000816921F080018161C16921F08001C161EA
:104A900062B670474FF040208069C0F3C010704785
:104AA000A548016F11F4007F14BF4FF440714FF41B
:104AB00080710166704710B59F4CE06F10F0020FD7
:104AC0004FF0010018BF0320606700F06DF94FF050
:104AD00040210A6B496B02F00F02D04001F00F0138
:104AE000C8400521B0FBF1F04FF405710009C4F88E
:104AF00080109249A1FB00104009C4F88400206F87
:104B000010F4007F14BF4FF440704FF480702066A3
:104B100010BD8948016F11F4807F14BF4FF44071BC
:104B20004FF4007101667047834B30B4DA6F12F0B6
:104B3000010F14BF032202225A6700EB4005C5EBA8
:104B4000C010C1EBC0004FF4FA744C43C0EB00102E
:104B500000EB40007A4904EBC000A1FB00104FF0CD
:104B6000402100220C6B4FF0020CC008496B04F08E
:104B70000F0401F00F012144C8400521B0FBF1F002
:104B8000B0F5803F05D3511C4008CAB2B0F5803F54
:104B9000F9D242EA0C2141F01001C3F88810C3F8A1
:104BA0008C00186F10F4807F14BF4FF440704FF4E6
:104BB0000070186630BC70475F48016F11F4003F09
:104BC00014BF4FF440314FF48031016670475A48AA
:104BD000016F11F4803F14BF4FF440314FF40031A6
:104BE000016670475448006FC0F300207047524878
:104BF000006FC0F3402070474FF040218969C1F336
:104C0000C011002904BF002070474B4900280CBF89
:104C1000D1F80002D1F8040270474FF040239A699E
:104C2000C2F3C012002A04BF00207047424A002885
:104C30000CBFD2F88000D2F88800C0F30A200CBF65
:104C4000D2F88020D2F8882002F00F02D3F830C0CA
:104C50005B6B0CF00F0C03F00F0363441A4491409C
:104C6000012202EB400048433449A1FB0010000937
:104C70007047344901200870704770B432224FF0F9
:104C8000402351431A6BD3F834C002F00F020CF0EA
:104C90000F0C6244121DD14008BF012104D0B1F5B0
:104CA000803F28BF4FF6FF719A69C2F3C012002AF5
:104CB0001CBF70BC704772B69A6942F080029A615C
:104CC000DA6942F08002DA6162B602241A4A146597
:104CD000250415664FF0040CC2F888C0C2F88C1089
:104CE000DFF864C0C2F86CC05467184902283CBFA2
:104CF000104E46F820100021124801704FF4007148
:104D00001166017819B920BF01780029FBD015661A
:104D1000C2F878C0C2F86CC0546572B6986920F0C9
:104D200080009861D86920F08000D86162B670BCBC
:104D300070470000A084001000A000401F85EB51C8
:104D4000CDCCCCCC9C84001002000202236C00006D
:104D50004FF0E021002088610861274948607047D2
:104D600010B54FF0E02460610020A0610221401ED8
:104D7000FFF7DDFB07202061BDE8104008F088BF89
:104D800010B508F089FF4FF0E0210020086110BD48
:104D900010B508F081FF4FF0E021002008611648AF
:104DA0000188491C018010BD1348806870472DE9B7
:104DB000F041114C002705462780A0684FF47A7116
:104DC000B0FBF1F04FF0E026401E7061B7610221A8
:104DD000C81EFFF7ACFB0720306108F059FF21889F
:104DE000A942FCD308F058FF3761BDE8F0810349C0
:104DF0004843014988607047A884001040420F0072
:104E00004FF04020816921F400518161C16921F492
:104E10000051C1617047A8490A78824218BF06282C
:104E200028BF7047A54AA64B52F830C0C3F808C047
:104E300002EBC0025268DA60087070474FF0402001
:104E4000816941F400518161C16941F40051C1613E
:104E5000704710B501210720FFF769FB4FF0402094
:104E6000816941F400518161C16941F40051C1611E
:104E7000934A0021116093495160DFF83CC2002140
:104E80009CF800303BB10CF110031C6894605B6827
:104E9000D3608CF800108C491161816921F40051B4
:104EA0008161C16921F40051C16110BD824840682F
:104EB00070478348806970474FF04020806910F444
:104EC000005008BF70477E48006900F0010070473D
:104ED0004FF04020806910F4005F04D0784B1869CF
:104EE00010F0010F01D10020704710B472494FF645
:104EF000FE7000248A684AB19A69D1F808C06245F8
:104F000004D08C604C6010BC0120704700BF00BF13
:104F100000BF00BF00BF00BF00BF00BF00BF00BF99
:104F200000BF00BF00BF00BF00BF00BF00BF00BF89
:104F300000BF00BF00BF00BF00BF00BF401E002871
:104F4000D8DC8C604C6010BC002070475A498860E7
:104F500070475948806870475948016941F001011C
:104F6000016155490120486070475548016921F0A9
:104F7000010101615049002048607047002100286C
:104F800008BF4FF0006103D0022808BF4FF08061D6
:104F90004B48026922F04062114301617047484961
:104FA0000120096901F04061B1F1806F04BF022066
:104FB0007047B1F1006F08BF00207047404840695A
:104FC00070473D48007870474FF04020806910F4EA
:104FD000005F38D03A4A106910F0010F33D03648DC
:104FE000406801282FD090696FF07F43984238BF06
:104FF00000EB400C27D25169B1EB9C0F01D301208B
:10500000704700BF00BF00BF00BF00BF00BF00BFB0
:1050100000BF00BF00BF00BF00BF00BF00BF00BF98
:1050200000BF00BF00BF00BF00BF00BF00BF00BF88
:1050300000BF00BF00BF00BF00BF00BF00BF00BF78
:1050400000BF9842D7D30020704710B50720FFF764
:10505000A9FA0720FFF78EFA1948016941F01001FB
:10506000016110BD164810B5016921F01001016100
:105070000720FFF78BFABDE810400720FFF792BA30
:105080000D4AD168D0600846704738B50C4CE069CD
:10509000E061094910F0020F1CBFA2698A60C9686B
:1050A00000291CBF00018847E0690090074801689B
:1050B00041F08001016038BDB4840010C484001048
:1050C00000D00040D0121300660F00157C84001041
:1050D000704770B505464FF40D500406A0660320D6
:1050E000E066264860664CF2710020662448C4F8E9
:1050F000800042F24630A06602210020FFF717FA36
:105100000020FFF737FA002D08BF70BDA06E42F2F5
:1051100041310843A06670BD012110B58807816741
:105120004FF40D5181660020FFF730FABDE81040C2
:105130000020FFF737BA0120810748677047012038
:105140008107886770474CF27100810708667047D5
:105150000C4A11681060084670470A4808B5006894
:1051600018B18047002818BF08BD4CF271018807AC
:105170000166016FC166006F009008BD075E5F3772
:1051800000AF2F91F4840010FE4900208871704711
:10519000FC488079704770B5FA4C00254FF4E46103
:1051A0002570E570F84808F064FF4FF4E461F748B3
:1051B00008F05FFFA56025714C21F54808F059FF04
:1051C0004C21F44808F055FF65717421F24808F04D
:1051D00050FF7421F14808F04CFFE56070BDE948CC
:1051E0000079002818BF01207047E6484079002860
:1051F00018BF01207047E348C078002818BF01207D
:105200007047E548704770B5E54DE64E04460146E7
:105210002A783078E04B10444200184608F033FFFB
:105220002A783078DD4B104442002146184608F0B9
:105230002AFFD44801214171817941F00401817133
:1052400070BDD048C0687047CF4870472DE9F04125
:10525000CC4F80463878002814BFD348D34805780F
:1052600014BFD348D348047805FB04F6FEF729FFA2
:1052700021462846FEF777FFC3494346C34A0846FE
:10528000FEF792FFFEF72EFF72004146BF4808F07E
:10529000FAFE0120F870B87940F00100B8710120E1
:1052A000BDE8F0812DE9F047B64D04460146287867
:1052B000DFF8D4C2DFF8F082DFF8F092BC4EBD4FC9
:1052C000002815BF98F8002099F8002033783B7823
:1052D00002FB03F04FEA4002604608F0D4FE287853
:1052E000DFF8A8C22146002815BF98F8002099F8D9
:1052F000002033783B7802FB03F04FEA400260461F
:1053000008F0C1FE0120E870A87940F00100A87102
:10531000BDE8F0879B488068704770B5A64C05468D
:10532000014622789A48520008F0ADFE22782946BC
:105330005200984808F0A7FE924801210171817936
:1053400041F00201817170BD2DE9F04FADF25C7D3D
:10535000DFF830820120CDF8400798F80300CDF83F
:105360003C0798F80400CDF83807002498F805B0F9
:1053700002F0D6F80546FDF78DFBCDF85407FDF792
:1053800085FDCDF85007FCF7E5F8CDF84C07FBF7A5
:1053900013FE0646FBF70DFE0746FDF77DFB98F86A
:1053A0000100002804BF0420C8F814000BD0022D0F
:1053B00018BF642411D002F0CBF8062808BF0F24D0
:1053C000002088F80100FBF7F7FD10F0010F14D062
:1053D00002F033FA3C280AD00FE016F0D8F948F270
:1053E0000211084214BF4FF4FA74FA24E3E7FFF7FE
:1053F00063FD002818BFFFF7E7FD4FF00109022FFA
:105400000AD1022D08BF4FF47A7403D0052D08BFCE
:10541000322401D188F80190002CD8BFD8F81400AC
:105420000EDD16F0010F27D002F007FAF8B1604345
:105430004FF47A7100F5FA70B0FBF1F0C8F814007F
:105440000228BCBF0220C8F8140098F80100B8F880
:105450001410000240EA014040F0010200239121B3
:1054600007200CF019FD16F0010F37D110E0052DC3
:1054700014BF78203C20DAE7FCF760F84FF47A712B
:10548000614300F5967001EB5001B1FBF0F0D5E7F8
:10549000022D23D00020FCF762F8FDF74BFD00251C
:1054A000AA4607F0C7FA01281ED00DF5E460FDF703
:1054B000C4FF002800F0C5810DF5E46008F00FFA84
:1054C000D8F81400C01EA842ACBF01260026DDF8A3
:1054D0002C0748B3DDF8380750B144E0FDF7DCFC99
:1054E0000020CDF84007DAE74FF0010A00F093B949
:1054F0006846DDF82C1708F0D0FD0746AEB12E4CFB
:10550000394620784200224808F0BDFD207839460F
:105510004200204808F0B7FD88F8049098F806008B
:1055200040F0020088F806001DE0FEF7CAFD224C9C
:1055300001212078FEF717FE164A3B46A2F14C01E6
:105540000846FEF731FEFEF7CDFD207839464200D1
:10555000104808F098FD88F8049098F8060040F08C
:10556000020088F80600DDF8280700287DD0DDF865
:105570003C07002879D198F80000DDF82847D8BB0F
:105580001CE00000F8840010D01E0110408B0010B9
:10559000A0A00010ECA00010F025011038A1001010
:1055A0005D8500105E8500105B8500105885001039
:1055B0005C850010598500105F850010D8F80870D0
:1055C00037B3FD480078CDF84807FC480078CDF89F
:1055D0004407FEF776FDDDF84417DDF84807FEF7CF
:1055E000C8FD21463A460846FEF708FEFEF77AFD5A
:1055F000F3480078022800E020E004BF384607F0B6
:1056000044FEEF480078092804BF204607F03DFE1D
:10561000EC480078012811D9E94F3878042804BFF4
:10562000204607F032FE2146684608F03BFD04465E
:105630003878052804BF204607F027FE8EB3E248DD
:1056400098F800202146002A0CBFE04ADA4A127876
:1056500014BFDA4BDE4B1B7802FB03F24FEA420227
:1056600008F011FDDB4B214600E052E098F8000005
:10567000002814BFD048D548007814BFCF4AD44A78
:10568000127800FB02F04FEA4002184608F0FBFCDB
:1056900088F8039098F8060040F0010088F80600AA
:1056A00030E0FFE7CDF8444798F80000002814BF29
:1056B000C148C648077814BFC048C548047807FBEE
:1056C00004F0CDF84807FEF7FCFC21463846FEF70B
:1056D0004AFDBD49BF4A0846DDF84437FEF764FD80
:1056E000FEF700FDDDF84807DDF844174200B94831
:1056F00008F0C9FC88F8039098F8060040F0010013
:1057000088F80600AE480078032804BFAE4807F0CA
:10571000BCFDDDF83007002873D0BBF1000F70D15D
:10572000044698F8000038BBD8F80C7027B3AA4894
:105730000178AA4800780844401C400801900220E3
:105740000090FEF7BEFCDDE90010FEF712FD2146D9
:105750003A460846FEF752FDFEF7C4FCA048007822
:10576000022804BF384607F04EFF9D4800780928FC
:1057700004BF204607F047FFD6B19A48964E974F90
:10578000214633783A781A44520008F07CFC32788B
:105790003B7895481A442146520008F074FC88F87A
:1057A000059098F8060040F0040088F8060021E013
:1057B000894826460178894800780C18FEF781FC54
:1057C000601C40080221FEF7CEFC86493346864A1B
:1057D0000846FEF7E9FCFEF785FC62003146824888
:1057E00008F051FC88F8059098F8060040F0040095
:1057F00088F806007A480078032804BF794807F043
:1058000002FFFDF766FED8F814006D1CA84211DCFB
:10581000D8F8100070B1FDF73FF9DDF84C07FBF741
:105820009EFEDDF8540788B1DDF8500760B1FDF742
:1058300081FB0BE0DDF84007002818BFFDF77AFB7D
:105840002FE601F0C8FE2CE6FDF726FBBAF1000FAB
:1058500004BF0420C8F8140009D0DDF83C0788F81C
:105860000300DDF8380788F8040088F805B04FEA2F
:105870000A2040EA05420023912107200CF00CFB8E
:105880000DF25C7D5046BDE8F08F10B50024FDF7A9
:10589000EFFA564910F0070F0AD0CA78002A08BF5D
:1058A000012410F0020F03D00A79002A08BF012456
:1058B00010F0F00F03D04879002808BF0124002021
:1058C000002C08BF10BD00200870BDE810403BE56B
:1058D00008B540F20F3101F0DDFF012804D1FFF7D8
:1058E000D4FF009002F075F94048C17800291CBF30
:1058F0004179002904D0007900281CBF012008BD8F
:10590000002008BD08B540F20F3101F0C3FF0128A7
:1059100004D1FFF7BAFF009002F05BF93348C17879
:1059200000291CBF4179002904D0007900281CBF40
:10593000012008BD002008BD70472C4910B5002289
:10594000CA700A714A7100281CBF012048700DF00E
:10595000C2FBBDE81040FAF747BD10B54FF4E46153
:10596000194808F086FBBDE810404FF4E46119487F
:1059700008F07FBB1E48704714480178144800782F
:10598000484341001A4808F074BB70B506460F48FA
:1059900004780F480578FEF794FB29462046FEF769
:1059A000E8FB094A31461248FEF728FCFEF79AFB4D
:1059B0000348007815281DE05B8500105C85001009
:1059C000DD8500105A850010D01E0110588500108A
:1059D00059850010408B00105D8500105E85001019
:1059E000E3850010F025011038A10010F8840010A4
:1059F0006092001018BF70BDF948BDE8704007F014
:105A000044BC70B50446F7480578F7480678FEF7B9
:105A100058FB31462846FEF7ACFB2246F3491046B8
:105A2000FEF7ECFBFEF75EFBF1480078162804BF9A
:105A3000204607F02AFC204670BD002818BF012030
:105A4000EC49C870704710B5EA4C002804BFA0604C
:105A500010BDDFF8A4C3E9490B78E9490A7801468B
:105A60005A435200604608F00EFBE348A06010BDA8
:105A700010B54C21E34808F0FCFABDE810404C2179
:105A8000E14808F0F6BADF487047002818BF012047
:105A9000D8490871704710B57421DC4808F0E9FA5C
:105AA000BDE810407421DA4808F0E3BA002818BFB6
:105AB0000120D0494871704710B5CE4C002804BF72
:105AC000E06010BD74220146D24808F0DCFAD148EB
:105AD000E06010BD70B5C74D00210446E970297122
:105AE00069710DF0F8FAFAF77FFC002C14BF012061
:105AF00000202870BDE8704026E42DE9F04F89B001
:105B00004FF4E461BC4808F0B4FA7421C14808F0CD
:105B1000B0FAFDF7ADF90446FCF7BCFF0890FDF7BD
:105B2000B5F90790FBF716FD0690FCF7B5FFFBF7FC
:105B300043FA10F0010F0BD001F07FFE3C2807D193
:105B4000FFF7BAF920B10420FFF765F9FFF73CFA37
:105B50000020FBF704FDFDF7EDF900252E4606F0C9
:105B600069FF012853D06846FDF767FC00285ED026
:105B7000684607F0B4FE14F0070F1CD09F48DFF80A
:105B800078B2DDF8089090F800809D48DA460778F2
:105B9000FEF797FA0120FEF7FAFA39464046FEF77B
:105BA000E8FA524649465846FEF728FB0020FEF721
:105BB000EEFAFEF797FA14F0F00F20D09648DFF8CF
:105BC00054B2022701789548DA46DDF81090007843
:105BD0000844401C4FEA5008FEF773FA0120FEF714
:105BE000D6FA39464046FEF7C4FA52464946584668
:105BF000FEF704FB0020FEF7CAFAFEF773FAFDF782
:105C000068FC6D1C102D03D2FDF794F9A7E701265F
:105C10000520FFF700F9FCF73FFF0698FBF79FFC14
:105C2000089848B1079828B1FDF784F904E001F01D
:105C3000D2FC94E7FDF730F9DEBB6E4F14F0070F8E
:105C40001BD06E48DFF8B0C101786D48E04600789F
:105C500001FB00F210200021002A88BF03460AD968
:105C600038F9115005EB5005B5FBF3F52CF8115040
:105C7000491C8A42F4D86048B86014F0F00F18D07C
:105C80006548644B017865481C4600780A184FF057
:105C900010014FF000000AD034F9105005EB510507
:105CA000B5FBF1FC23F810C0401C8242F4D85948DF
:105CB000F86009B03046BDE8F08F012070474FF41E
:105CC0007B3070474FF47B300068704703460020FC
:105CD0009A682C2A88BF2C220021B1EB920F28BF92
:105CE000704753F821C0491C6044B1EB920FF8D3C0
:105CF00070474B4A0168914214D14168B1F5807FE9
:105D000010D9836800222C2B88BF2C230021B1EBF3
:105D1000930F09D250F821C0491C6244B1EB930F94
:105D2000F8D30AB100207047012070474FF47B314F
:105D30003B4B0A689A423ED191F827300022012B52
:105D400008BF0122052804BF91F82300704713DC27
:105D5000012804BF087F7047022804BF91F8200083
:105D60007047032804BF91F821007047042804BF3E
:105D700091F82200704731E0142808D015280CD083
:105D8000162811D0172804BF1846704726E0002AAD
:105D90001CBF91F82400704704E0002A1CBF91F852
:105DA000250070472D207047002A1CBF91F826005F
:105DB000704728207047052834D007DC01280DD013
:105DC00002281CBF032804282CD007E0142818BF81
:105DD0001528E7D01628ECD0172823D0FF207047CD
:105DE000609200105885001059850010D01E0110D7
:105DF000DD850010F8840010809900105B8500108C
:105E00005C850010A0A00010ECA00010F02501108F
:105E100038A10010ACA100105D8500105E85001057
:105E20004353494D002070472DE9F047ADF5007D03
:105E300000244FF40071684608F01BF9FF20A046CB
:105E400060F307082D20254660F3070560F30F2552
:105E5000282060F317454FF47B37F74E64F31F6536
:105E60004FF481794FF02C0AFF224FF400716846FD
:105E700008F01DF9CDE902A4CDE9064805940A947D
:105E8000CDE900690494CDE908453846FDF73CFFAB
:105E900069463846FDF7DAFF012818BF00200DF5E6
:105EA000007DBDE8F0872DE9F047ADF50C7D894612
:105EB00005461F4690464FF0000A4FF400716846B1
:105EC000949E08F0D6F84FF0000CCDF800C24FF4C5
:105ED0007B34CDF804C2CDF808C2CDF80CC2CDF8A1
:105EE00010C2CDF814C2CDF818C2CDF81CC2CDF83E
:105EF00020C2CDF824C2CDF828C2CF4920688842FC
:105F000006D0FFF791FF0DF50C7D5046BDE8F087F8
:105F1000D4E901120DF5007AE3688AE80F0004F174
:105F200010010DF5047A0FC98AE80F00D4E90801C1
:105F3000A26A8A92CDE9880184988DF820928DF822
:105F40002182401C8DF822728DF81C528DF823623C
:105F50008490002D14BF8698859800F1010014BF2D
:105F60008690859080AB82980021CDF80CC22C28B9
:105F700094BF02462C220020B0EB920F06D253F8B9
:105F800020C0401C6144B0EB920FF8D3484283908C
:105F9000FF224FF40071684608F089F880AC94E85D
:105FA0000F008DE80F0084AC94E80F0004AC84E887
:105FB0000F00DDE988018A9A4FF47B34CDE90801AE
:105FC0000A922046FDF7A0FE69462046FDF73EFFF7
:105FD000012818BF00200DF50C7DBDE8F0872DE9E4
:105FE000F041ADF50C7D0F46804616464FF400712A
:105FF000684608F03EF8002580954FF47B34819583
:1060000082958395849585958695879588958995BC
:106010008A9589492068884218D16068B0F5807FE8
:1060200014D9A06821464FF0000C2C2888BF2C20E2
:106030000023B3EB900F11D251F823205B1C944442
:10604000B3EB900FF8D3BCF1000F07D0FFF7ECFED5
:10605000002804BF0DF50C7DBDE8F0810FCC0DF5D7
:10606000007C8CE80F000FCC0DF5047C8CE80F0051
:10607000D4E90001A2688A92CDE988018DF82482D2
:106080008DF825728DF8266201208DF827028298FE
:10609000002180AB83952C2894BF02462C2200203F
:1060A000B0EB920F06D253F820C0401C6144B0EB15
:1060B000920FF8D348428390FF224FF40071684654
:1060C00007F0F5FF80AC94E80F008DE80F0084AC7A
:1060D00094E80F0004AC84E80F00DDE988018A9A97
:1060E0004FF47B34CDE908010A922046FDF70CFEFF
:1060F00069462046FDF7AAFE012818BF00200DF5CD
:106100000C7DBDE8F0812DE9F04F4C4D4FF00008BB
:1061100085B06C42474646461720FFF707FE4FF40E
:106120007B32844644491068884217D15068B0F5E4
:10613000807F13D9936800212C2B88BF2C2300204B
:10614000B0EB930F80F0FE8052F82090401C494441
:10615000B0EB930FF8D3002900F0F480FFF764FE52
:10616000002804BF05B0BDE8F08F1420FFF7DEFD66
:1061700002901520FFF7DAFD00901620FFF7D6FDFC
:1061800040B201901620FFF7D1FD404240B203908B
:10619000FCF76EFEDFF8A8908246002089F8030025
:1061A00089F8040089F805000CF095FFFAF71CF94E
:1061B000002089F80000FFF7C7F81AF0F00F05D0AB
:1061C00007F07AFF012808BF48F001081AF0070F0E
:1061D0007DD01C481D4A002690F800E01A4803783C
:1061E00099F80200A3EB000984468145C4BFAEEBD9
:1061F0000C01A1F1010B1CDD61468B4516DD01F19F
:10620000010A01FB03070AFB030A32F8177032F890
:106210001AA0A7EB0A073FB2002FB8BF7F423FB2D8
:10622000B742C8BFBEB2491C8B45E8DC401C814563
:10623000E2DC009800280BE04353494DF1D8FFFF02
:10624000F88400105985001058850010D01E0110E8
:1062500018BF864288BF48F002080027E246AEEB2E
:106260000A0000905045C8BFA9F1010B1BDD604634
:10627000834513DD0AFB030132F811E002EB410113
:106280004988AEEB010109B20029B8BF494209B201
:10629000B942C8BF8FB2401C8345EBDC00980AF1BD
:1062A000010A5045E3DC0298002818BF874288BFE6
:1062B00048F00408E2460098504516DD61468945DD
:1062C0000EDD0AFB031032F91000A84200E016E0D0
:1062D000C8BF0546A042B8BF0446491C8945F0DC4A
:1062E00000980AF1010A5045E8DC0198002806DD13
:1062F000854202DC0398844201DA48F00808FF2F47
:1063000088BFFF27FF2E88BFFF267F2DC8BF7F25B0
:1063100004DC15F1800FB8BF6FF07F057F2CC8BF7C
:106320007F2404DC14F1800FB8BF6FF07F04E0B26B
:106330000090EBB2F2B2F9B24046FFF7B4FD05B0FF
:10634000BDE8F08FBCF1000F18BFBCF1010F3FF4A6
:106350000CAF03E7FE4900208862704740B2FC4959
:1063600010F1050FBCBF00228A6288707047F848A0
:1063700090F902007047F64800787047F44840787A
:106380007047F3480021C17141718172C17201737C
:1063900041727047EE4920F07E4008627047EC4839
:1063A000006A7047EA48408A7047E948808A704727
:1063B000E748B0F916007047E548B0F91800704793
:1063C000E348B0F91A007047E148407B7047E04865
:1063D000C078002818BF0120704710B54FF4E46161
:1063E000DC4807F046FEDA490020C87010BD2DE9F0
:1063F000F74F90B00025D848019502950395049574
:1064000005950695079508950995006817460C4669
:10641000052A08BFB0F97A600AD0062F08BFB0F984
:10642000786005D00A2F0CBF1E26B0F976600FD019
:10643000B0F97400DFF82083B04209DA15F0A7F94B
:10644000C64908421CBFD8F80000B0F8746036B2E4
:10645000324601A9109807F034FE059800B220805A
:10646000BDF826106182BDF81E106181BDF82010B4
:10647000A181BDF82210E181BDF824102182BDF870
:106480001810A180BDF81A10E180BDF81C10218100
:106490000028B8BF25808DF82850B148B149007850
:1064A0008DF82A008DF8295009788DF82B1071424B
:1064B000ADF82E10ADF8300080B2ADF82C60ADF81C
:1064C0000000DDE90A232146109800F08BFD052F1E
:1064D00011D0E582A5822583A088002804BF4FF44F
:1064E0000040A0806089002804BF47F6FF706081EB
:1064F00013B0BDE8F08FFEF7A7FE002107F0E6FD20
:10650000002800F0F180DDF828C0DDE90B0ACCF3AB
:10651000072310994FEA1C62ADF80050ADF83450D3
:1065200099469A4269D91FFA8AF50CF0FF0603FBD7
:10653000056E1FFA8EF80E9531F91880BDF80060CF
:10654000BDF834500FFA80FBD845C4BF761CB6B2F4
:106550004FEA204BD845BCBF6D1CADB2ADF8006012
:106560000EF101081FFA88F8ADF8345031F918809F
:106570000FFA80FBD845C4BF761CB6B24FEA204B59
:10658000D845BCBF6D1CADB2ADF80060DDF83880F9
:10659000CCF3074B03FB08BEAEF102081FFA88F8E4
:1065A000ADF8345031F918800FFA80FBD845C4BFDC
:1065B000761CB6B24FEA204BD845BCBF6D1CADB2BD
:1065C000ADF80060AEF101081FFA88F8ADF834505C
:1065D00031F918800FFA80FBD845C4BF761CB6B2DB
:1065E0004FEA204BD845BCBF6D1CADB2ADF8006082
:1065F0005B1CADF834509A4295D80CF0FF03CCF3F5
:10660000074E9E456CD91FFA8AF609FB063C1FFA15
:106610008CF8BDF800C031F918800FFA80FBADB2DC
:10662000D845C4BF0CF1010C1FFA8CFC4FEA204B7B
:10663000D845BCBF6D1CADB2ADF800C009F1010872
:1066400008FB06381FFA88F8ADF8345031F9188085
:106650000FFA80FBD845C4BF0CF1010C1FFA8CFC6B
:106660004FEA204BD845BCBF6D1CADB2ADF800C0A1
:10667000A2F1020808FB06381FFA88F8ADF834507A
:1066800031F918800FFA80FBD845C4BF0CF1010C1A
:106690001FFA8CFC4FEA204BD845BCBF6D1CADB235
:1066A000ADF800C0A2F1010808FB0636B6B2ADF89D
:1066B000345031F916600FFA80F84645C4BF0CF12A
:1066C000010C1FFA8CFC4FEA20484645BCBF6D1CEC
:1066D000ADB2ADF800C05B1CADF834509E4592D809
:1066E000E582BDF80000A082DDF830900A9E109D82
:1066F0004FF0000C052F50D01748062F006803BF3D
:10670000B0F8781002273846B0F876101CBF012781
:106710000020B4F90230B4F90020934244D18A42F7
:1067200042DDC6F307210144C0EB166A8A4531D920
:10673000C6F30742F0B2D21B3844A2F101088045EB
:1067400025D91FFA89F201FB020292B20CE0000087
:106750001085001020A20010BC86001002810100EC
:10676000588500105985001035F9123005EB4202AA
:10677000B2F90220B3EB020B48BFA2EB030B0FFAF6
:106780008BF26245C8BF9446401C8045D9D8491C4D
:106790008A45CDD8A4F818C09EE6FE4802270068B6
:1067A000B0F87A103846B4E7228395E6084318BF5C
:1067B0007047F948016A11F0807F08BF7047F549BA
:1067C0000968096F11F4003F08BF7047002111707C
:1067D000182101827047F048006B70472DE9FF5F78
:1067E000EE480027DDF83CA005780E98119E8B46F8
:1067F000B9463C4650452CD006FB050E10983BF997
:106800001EC006FB05093BF91900BCEB000148BF9F
:10681000A0EB0C0106FB05A83BF91840B4EB000CFB
:1068200048BFA0EB040C01EB0C0004B232F91EC00F
:1068300032F91900BCEB000148BFA0EB0C0132F9A2
:1068400018C0BCEB000248BFA0EB0C0288180FFA7E
:1068500080F9D148006B012818BF012B37D04FF0C9
:10686000010807F038FCCE49002C0A7807DD1099A2
:1068700006FB05113BF911101431282909D800999C
:10688000B1F914103C2904DC0099B1F916103C2927
:1068900026DD0E9902EB0A0C11448C4520D9129B7F
:1068A000139D13442A448B421CBF8D1A15F1020F0D
:1068B00030F9115000EB4106B6F90260A5EB060570
:1068C00008D01E353C2D08D94FF0000808E0A1453E
:1068D0000CDD0AE00A35142DF6D8491C8C45E2D8A7
:1068E000A14503DDB8F1000F00D0012704B0384600
:1068F000BDE8F09F7047A848B0F90E007047A64960
:106900000020C88170470021018041804FF400427F
:106910008280C1800181521E42818181C1810182B8
:1069200041828182C182018370479B48C06A70475F
:10693000002818BF01209849C86270470022964974
:10694000022802D080208A6288708A62704770B5FF
:10695000914E04460D46306B844206D044EA05222F
:1069600000236B2107200BF097FA34B90020022D89
:1069700002D08021B062B170B062346370BD8648CD
:1069800090F9020010F1800F18BF10F1050FACBF95
:106990000020012070472DE9F0418846054614F09B
:1069A000DEFE044614F0D7FE04FB00F17A4E2218F6
:1069B000002496F9020009B210F1800F274618BF93
:1069C00010F1050F1BDAB6F91A006439814211DAA9
:1069D0000124B8F1000F12D10021002A0FD935F996
:1069E0001100B0F5487F01DA002403E0491C914210
:1069F000F5D324B911F0B9FD012808BF0124306B8B
:106A0000012808BF002C16D1B06A4EF6C421884276
:106A10000BD200F08BFD0021022819D0042808BFFA
:106A20004FF4FA71B06A0844B0624EF660218142B8
:106A300028BF012400D2B762306B844206D044F4F0
:106A4000807200236B2107200BF026FA54B906E070
:106A50000CF03EFB002814BF11210821E2E7802042
:106A6000B762B0703463BDE8F081002818BF012020
:106A70004949486370474848406B70474649888396
:106A800070474548808B70474348406A7047424989
:106A90004862F9F7C9BC4049886370472DE9F04F57
:106AA000404987B002240A783C49A2F1020C521EE8
:106AB00091F8008000210091A8F10101CDE9011CAD
:106AC00000212546A8F102090B46BCF1020F84BF44
:106AD000A9F1010CCDF80CC06BD94FF0000CCDF82A
:106AE00014C0CDF810C0AC464D4551D2039F04FBF5
:106AF00008C6BC450FD230F9167000EB4606B6F951
:106B00000260B7EB060E48BFA6EB070EBEF1320FD0
:106B100001D9E34608E00CF1010CE145E6D8DDF8C7
:106B200014C0BCF1000F1BD0A9F1010CAC4517D368
:106B300004FB08C665450FD230F9167000EB460617
:106B400036F9026CB7EB060E48BFA6EB070EBEF196
:106B5000320F01D9E24608E0ACF1010CAC45E7D2B6
:106B6000DDF810C0BCF1000F12D04FF0010CCDF8D1
:106B700000C0DDF804C0DC4588BFCDF804B0514545
:106B800038BF5146A24288BF2246A34238BF23469F
:106B9000641C0AE0BC8600101085001058850010A7
:106BA0005E8500105985001003E0DDF808C06445DB
:106BB00093D3FE48DDF800C0846B644518BFC0F86D
:106BC00038C0019807B0BDE8F04F15F0A1BD2DE920
:106BD000FF4F8BB00025DDE918A90090F3480E4661
:106BE000057045700CF088FA002840F03F8100F0F5
:106BF00097FC052868D0DFF8B483EE4998F80D00BB
:106C00000290EB480978006890F886400191B0F94D
:106C10008470E949B8F91800322891F800B0B8F842
:106C2000120005DA002804BF6006040E05D100E05A
:106C300018B998F80400012844D10CF0A5FA0028EE
:106C400040D1B9F1010F3DD0BAF1010F03D1B8F82D
:106C50001400C82836D8B8F81400002804BFB8F8C3
:106C6000120000282ED00CF033FA012809D014F0BD
:106C700075F878B114F03CFE60B114F0FBFD082803
:106C800008D0CB48006890F88740029801280CBFD4
:106C900041273C273088A8F80E000199002011EB0D
:106CA0000B030BD036F91010B8F90E209142C8BF73
:106CB000A8F80E10401C80B28342F3D8B8F90E0039
:106CC000B84202DD88F80B501DE0D8F8200010F41F
:106CD000803F18D0B6480068006F10F4803F12D093
:106CE00098F80B00401CC0B288F80B00A0420AD9EB
:106CF0004FF0FF3000901020A8F81000012088F815
:106D0000080088F80B5011F030FCB8B100F00EFC10
:106D1000042813D1A54890F8201011F0800F0DD051
:106D2000A349096891F8701011F0800F06D007216F
:106D300001824FF0FF3100910121017214F0D8FD62
:106D400050B114F097FD082806D04B4652466946CC
:106D5000304600F017FA89E00CF0BAF9012856D154
:106D60004B4652466946304600F00CFA914804966C
:106D70004FF0000A007807908F48B9F1010F90F8A2
:106D800000B08B480068089090F8870009903CD0CC
:106D90004FEA5B000590079840080390002001909F
:106DA0008146029006EB4B000690002632463146A3
:106DB000B9F1000F06BF5B46049CDDE906430020E5
:106DC000002B88BFA3F1010E22D934F91070642F73
:106DD000D8BF002214DD70450DD204EB400CBCF985
:106DE00002C0B7EB0C0848BFACEB07080FFA88FCF1
:106DF000D445A8BFE246491C002A04BF0122761CE4
:106E0000401C8342E1D8012E02D9684805732DE069
:106E1000B9F1000F0CBF0191029109F10109B9F11B
:106E2000020FC2D305990198884284BFDDE90201AF
:106E30008842EAD9BAF1320FE7DC5C49087B401C92
:106E4000C0B208730A6A12F4801F0FD0089A126F3A
:106E500012F4801F1CBF099A904207D94FF0FF30EF
:106E6000009014200882012008720D7314F08FFC2A
:106E700010F4014F24D000F053FB022820D1012749
:106E800007F02EF9064614F06AFC044614F063FC81
:106E900000220021002C08D901FB002336F9133011
:106EA0000F2B0DDB491CA142F6D34FB1521C012A16
:106EB000EFD92FB14FF0FF303C490090012008720C
:106EC0000FF0EFFA032824D1384801950295017C90
:106ED0008DF80410BDF80410009A62F30F21ADF88C
:106EE0000410C279BDF8061062F30301427962F31F
:106EF0000711027A62F30821827962F34921ADF821
:106F00000610C089ADF808000222062101A80FF082
:106F1000CBFA06F08BFC254C217A4170A279827065
:106F2000E279C27062790271227C4271009A8271A8
:106F3000B2F1FF3F1AD101291CBF0FB0BDE8F08F9D
:106F40000D98FEF722FD2572012060704FF4E46178
:106F50001A4807F08EF8E5700D98002818BFFEF764
:106F6000A1F90E98002818BFFEF74DF900980028E7
:106F700007BFA07901280FB0BDE8F08FFEF7FCFC39
:106F8000A571012020704FF4E4610C4807F071F8FE
:106F9000E57000F0CBFA04280D9817D0002818BF30
:106FA000FEF780F90E9800280AE000001085001016
:106FB000BC8600105D8500105E85001020A20010C8
:106FC00018BFFEF720F90FB0BDE8F08F002818BFFA
:106FD000FEF73CF90E98002818BF07F086F80FB0AE
:106FE000BDE8F08F2DE9F8070023DDF820C0C2F3DB
:106FF0000724ADF80030160E2546D3B21FFA8CFCDC
:10700000C2F30747A64259D904FB0C381FFA88F28D
:1070100030F9129000EB4202B2F902A0B9EB0A0279
:1070200048BFAAEB090212B2BDF900909145B8BF62
:10703000ADF8002008F1010292B230F9129000EB95
:107040004202B2F90280B9EB080248BFA8EB09027C
:1070500012B2BDF900809045B8BFADF8002004FB26
:107060000C78A8F1030292B230F9129000EB4202C0
:10707000B2F902A0B9EB0A0248BFAAEB090212B2A8
:10708000BDF900909145B8BFADF80020A8F102020B
:1070900092B230F9128000EB4202B2F90290B8EBE2
:1070A000090248BFA9EB080212B2BDF90080904561
:1070B000B8BFADF80020641CA642A5D8A7F101080E
:1070C000984559D96F1CB41E761E05FB0C3292B23E
:1070D00030F9129000EB4202B2F902A0B9EB0A02B9
:1070E00048BFAAEB090212B2BDF900909145B8BFA2
:1070F000ADF8002007FB0C3292B230F9129000EB91
:107100004202B2F902A0B9EB0A0248BFAAEB090297
:1071100012B2BDF900909145B8BFADF8002004FB54
:107120000C3292B230F9129000EB4202B2F902A096
:10713000B9EB0A0248BFAAEB090212B2BDF90090EE
:107140009145B8BFADF8002006FB0C3292B230F981
:10715000129000EB4202B2F902A0B9EB0A0248BF5A
:10716000AAEB090212B2BDF900909145B8BFADF883
:1071700000205B1C9845A8D8BDF800004880BDE8F9
:10718000F8077047D44830B400680025D34C90F815
:1071900088C0002A1ADC012B18D0226A12F4003FA2
:1071A0001CBF006F10F4003F0DD0A07A401CC0B28D
:1071B000A072604507D94FF0FF300860112020828F
:1071C00001202072A57230BC00207047A57230BC2F
:1071D000002070472DE9FF4FDFF8FCB2044689B06C
:1071E000DBF800001D461646B0F878A013F0B6FD97
:1071F000012804BF4FF6FF7000EA4A0A14F0C7FAEC
:10720000B74F384207D0B5F9141001232046169A1B
:1072100006F070FF04E0012220461699FFF7E7F818
:10722000DFF8B8820024254688F80440DDF828906D
:10723000FEF70AF8009401940294039404940594D0
:10724000069407940894A44C69462068B0F8762008
:10725000484606F036FF2168BDF91A00B1F97610EC
:1072600049428842B8BF0125BDF82000B0F5E17F52
:1072700088BF01259948057114F089FA9849084298
:107280000DD11698B0F91200002808DC0BF020FF91
:10729000012804D091480079012840F0E78014F0DB
:1072A00076FADFF83CB210EA0B0F00F0D7808D4879
:1072B00047F6FF79179C90F800808B4807780020EC
:1072C0000546019014F063FA10EA0B0F0FBF504609
:1072D00081480068B0F8740000B2009014F057FACA
:1072E00010EA0B0F1FBF7C480068B0F874004042E2
:1072F00008BFCAF1000000B2039014F048FA10F47D
:10730000807F1CBF4FF0010A4FF0220C34D04FF0A9
:10731000000B009848457DDA5A46B8F1000F7AD93B
:10732000ACF101000690A8F101000590ACF102005B
:1073300004905046E2453CBF11B202916FD202FB6D
:10734000070399B236F911100029B4BFC1F1000941
:107350008946DDF800E0F14537DD714527DDB4F9F8
:107360000490494503DDA180E080029921810199C3
:10737000491C09B2019128E010F4004F07D04FF0EA
:10738000000A4FF0260CD3464FF00508C1E710F471
:10739000803F04BF4FF0000ABC46B8D04FF01C0A33
:1073A0004FF0260C4FF0000B4FF01108B1E7DDF85D
:1073B0000C90894509DDB4F90A90894503DD6181A6
:1073C000A0810299E181691C0DB2069988421FD201
:1073D00006EB430136F91390B1F90230B9EB030122
:1073E00048BFA3EB090109B25A451CBF059B9A424D
:1073F00004D050451CBF049B984204D1B4F902301C
:107400008B42B8BF6180B4F900308B42B8BF218095
:10741000401C02E007E01DE001E060458FD3521CF4
:10742000424586D316E0B8F1000F13D95346E24522
:107430000CD20BFB073080B236F910100398814252
:10744000BCBF681C05B25B1C6345F2D30BF1010B9A
:10745000C345EBD301982082658204E006223046C2
:107460001799FEF7C4FF1999012008701798B0F911
:107470001000002808DC1798B0F91200002803DC7F
:1074800016480079012814D114F081F914490842F2
:1074900007D0052347F6FF71189A0A9806F02AFECE
:1074A00004E0052218990A98FEF7A1FF1A99012015
:1074B00008701698418A094841821699098A818282
:1074C00016994989C1821699898801831899098A70
:1074D00041830DB0BDE8F08FBC8600101085001010
:1074E00002810100598500105885001010B50BF07D
:1074F000D9FB0BF0C9FC002010BD0000FE49C8708C
:107500007047FD48C0787047FB4908717047FA48DA
:1075100000797047401E022894BF01200020704768
:10752000F54800787047F44880787047F248007852
:10753000022805D005281CBF0020704707F027B897
:107540000BF0A6BDEC4908707047EB4948707047D6
:10755000E9484078704770B5E74E04460D463078EC
:10756000A04212D002281ED0052814BF002007F028
:107570000EF844EA05213278002341EA024141EA4B
:107580000062612107200AF087FC3078844218BF2E
:107590007070B570072C28BF70BDDFE804F01A07C3
:1075A0000B13170F1A000BF073FDE2E7284600F0EB
:1075B00023FB0EE028460BF01FFE0AE0284606F0EB
:1075C000D7FF06E028460AF061FD02E0284606F0F3
:1075D0008EFF347070BDC94900200968B1F8B01041
:1075E00011F4807F08BF7047FCF7A9BAC349002097
:1075F0000968B1F8B01011F4807F08BF7047FCF73C
:10760000ADBABE4900200968B1F8B01011F4007F8E
:1076100008BF704706F073BDB749487900281CBF02
:10762000401E4871704770B5B5480068B24C10F004
:10763000130F0FD010F0100F05D0B24951F88C2F56
:1076400042F480520A60B04908606079002804BFA3
:10765000012060714FF040208069A84D10F0020FAA
:10766000296806D1A948006810F0010F01D060799F
:1076700040B1B1F8B010002011F4807F18BFFCF7C2
:107680006DFA07E0B1F8B010002011F4806F18BF58
:1076900006F03AFD9E49084208BF70BD2968D1F83E
:1076A000B010090C617170BD10B572B6FDF734FDF4
:1076B000BDE81040FDF744B910B5012802D00228FA
:1076C00005D007E04FF47F30FCF71EFB02E0924943
:1076D0009048086072B6FDF71FFDBDE81040FDF749
:1076E0002FB9854900288A7918BF01208871C0B256
:1076F000824208BF70470022002818BF01220023E1
:10770000012102200AF0C8BB7B488079002818BFFD
:1077100001207047784AD179814208BF70471072C2
:107720000120507270477448007A7047724948725D
:1077300070477148407A704770B56F4C0028E57902
:1077400018BF0120E071C0B2F8F72DFEE079854244
:1077500014BF002870BD207802281CBF052870BD0A
:107760000221BDE87040F6E610B514F010F86B4940
:1077700008421CBF002010BD5F48C079002818BF18
:10778000012010BD00285C4918BF01208872704795
:1077900010B513F0FCFF614908421CBF002010BD6A
:1077A0005548807A002818BF012010BD5248C07A81
:1077B00070472DE9F041504D00281CBF0020E872B1
:1077C00004D1E87A002818BFBDE8F081544E37682C
:1077D0003020FCF71BFC06213020FCF730FCF06A5F
:1077E00040F03000F0624F4C4FF07F0811E0FDF7A1
:1077F000AAFCF06A10F0100F03D0E87A40F07E0087
:10780000E872F06A10F0200F03D0E87A40F001002F
:10781000E872201EA4F1010403DDE87A38EA0000D2
:10782000E5D13020FCF738FC3760BDE8F081324804
:10783000C06970473048806970472F4880690028C8
:1078400018BFC07A70472C49086270472A48006AFE
:1078500070472949486270472748406A704727485F
:10786000026802F5C873118A508A02F5A872FBF704
:1078700052BC10B507F0CDFB002818BFC07A10BD70
:1078800010B507F0C6FB00280CBF4FF0FF3090F991
:10789000240010BD2DE9F04FDFF85CA099B00D4633
:1078A000CAF81C0007F0B5FBCAF81800002800F061
:1078B000E58090F800C08AF80CC041788AF80D1075
:1078C000837804460CF101008AF80E3000F0FE00C7
:1078D0008AF80F00E2788AF8102020798AF81100DF
:1078E00060798AF812000AF114004FF0000B80F85A
:1078F00000B080F801B017E04C850010BC86001085
:10790000184800400030004014480040144C00402B
:1079100008001300AD2007B0304C00400281010088
:10792000001000408038010020788AF8130060467B
:10793000FBF74FFD9AF812109AF81100FBF76CFD57
:107940006946204607F083FBE089DAF820600028CA
:107950001CBF7043060BB4F81280DAF82490B8F11B
:10796000000F08BF4FF48058E78A002F08BF4FF47C
:1079700080574FF480501890002015F0040F18BF66
:10798000052015F0080F18BF40F0020015F0020F97
:1079900018BF40F0F00015F0010F18BF40F4774019
:1079A00015F4807F18BF40F4803015F4007F18BFB5
:1079B00040F47E00E16901EA000504F029FF012896
:1079C00008BF25F0F00500981090059812900798D0
:1079D000CDF844B0CDE9130B01981590A07A17901B
:1079E0000398169010A92846FBF748F915F0070FE1
:1079F00074D00020F9F756F89AF8101088421AD07F
:107A00000020F9F744F89AF8100000EB400101EB70
:107A10000010754901EB80004C2106F02AFB9AF812
:107A2000100000EB400101EB0010704901EB8000F9
:107A30004C2106F01EFB06F0CAFF18B101460020DB
:107A4000F9F795FE06F0DAFF7043060B06F0F6FF35
:107A500009FB00F0000B4030C2090A20012101FAA5
:107A600000F3134201D1401EF9D5A0F10509207B96
:107A7000002818BFA0F1010B11D10CE05C48006890
:107A8000B0F8B00010F4807F18BFFCF767F8002052
:107A900019B0BDE8F08F0020FAF78BF88346607BC1
:107AA000002814BF401EFAF7BCF80BEB09010529AA
:107AB00005DDA9EB010101F10509052104E000291B
:107AC000BCBFA9EB010900218144B9F1050F06DD16
:107AD000A9F10500C6404FF0050908E00EE0B9F134
:107AE000000F04DAC9F1000086404FF000090020C1
:107AF000FAF779F849460020FAF7ADF815F0F00FDB
:107B000043D0207C70B115F0100F03D0411E01202E
:107B1000FAF769F815F0400F04D0207C411E0220CE
:107B2000FAF761F8207D70B115F0200F03D0411EE7
:107B30001120FAF758F815F0800F04D0207D411E6F
:107B40001220FAF750F8607C70B115F0100F03D0D6
:107B5000411E0120FAF77FF815F0400F04D0607C39
:107B6000411E0220FAF777F8607D70B115F0200F02
:107B700003D0411E1120FAF76EF815F0800F04D0E3
:107B8000607D411E1220FAF766F8E07A00281CBFDB
:107B90000001F9F724FD029806F09DF9049830B130
:107BA00033469AF80D209AF80C1006F0B2FA3A46CD
:107BB00041463046189B06F0B1FA0698FDF743FFA0
:107BC0000898FDF779FF0BF0E9FB19B00120BDE83B
:107BD000F08F10B5FBF70FF906F085F90549002085
:107BE0008861012010BD000000000130004001301C
:107BF000BC8600104C850010FE4908707047FD4897
:107C000000787047FC4810B4FC4A016891421CD1CE
:107C10004168B1F5987F18D8D0F808C00146BCF586
:107C2000007F12D800220B461146B2EB9C0F24BFF6
:107C300010BC704753F82140491C2244B1EB9C0F03
:107C4000F8D3002A04BF10BC7047002010BC704756
:107C5000E948FCF759B8E7490120087070472DE959
:107C6000F04117460E4605461024FFF7E3FD15F0D8
:107C7000070F18BF062403D115F0F00F18BF082412
:107C80003246102C28BFBDE8F081002A08BFBDE8AD
:107C9000F08120443B4690F920102046BDE8F04199
:107CA00007F0FDB9F0B5ADF6446D0446FFF7C2FD2F
:107CB000054614F0070F0CD06F4605263846FBF733
:107CC0000CFC95F925104FF464633A46304607F0F2
:107CD000E6F914F0F00F04BF0DF6446DF0BD072473
:107CE0006E46FBF7C5F810F0300F0CBF02200120E4
:107CF0006946FBF742FC95F927104FF4187332469A
:107D0000204607F0CCF90DF6446DF0BD2DE9F34F98
:107D100089B000200690087803904868049088682D
:107D200005900D7B487B0190887B8A8AD1E9088B7E
:107D3000C0F5807602EA00070998B1F91090B1F910
:107D400012A0896910F0010F07914FF0000044D094
:107D500000900198002840F2D7800098012101FA94
:107D600000F20798104018BF01200024029061091A
:107D700004A804F01F0250F8211001209040014295
:107D800000F0B7803BF9020B0299A0EB0A00002932
:107D90000CBFA9EB000509EB000538F9020BA0EBBD
:107DA0000A0014BF4844A9EB0000002DB4BF69428B
:107DB00029460028B8BF4042884278D92246009917
:107DC0000398FAF7ECFC0246C0F30420D1B212F497
:107DD000803F6FD0002D6FDB70E0FAF746F800901F
:107DE00001980321684301EB400020F00302414663
:107DF000584606F048F90098FAF737F801984FF01E
:107E0000000B002852D90121079801FA0BF210400B
:107E100018BF012000250290690904A805F01F027F
:107E200050F8211001209040014237D038F9020B60
:107E30000299A0EB0A0000290CBFA9EB000409EB92
:107E400000042A4659460398FAF7A9FCC0F3042116
:107E5000C2B210F4803F02D0002C02DB03E0002C01
:107E600001DD941B00E09419BC4205DD1F293ABFD7
:107E70000024491C3C4606E0002C04DA0029C6BF59
:107E80003C46491E002400F4783040EA012040EAD4
:107E900004032A4659460398FAF7D4FC6D1C262D94
:107EA000BAD301980BF1010B8345ACD32CE020E051
:107EB00000E001E0002D01DD8D1900E08D1BBD42C9
:107EC00005DD1F283ABF0025401C3D4606E0002D79
:107ED00004DA0028C6BF3D46401E002502F4783172
:107EE00041EA002040EA0503224600990398FAF788
:107EF000A9FC641C262CFFF43AAF00980199401CA1
:107F000000908842FFF429AF0998032826BF01207A
:107F1000069006980BB0BDE8F08F2DE9F04F8BB0BE
:107F2000002205920A7800924A6802928A680392B7
:107F30004D7B8A7B0492B1F91080B1F9122007922F
:107F40000C6A8A690892898A049AC0F1080A01EACF
:107F5000020600283BD0BAF1000F7DDB4FF0000B8A
:107F6000002D7AD9012000FA0AF00690AAF101004A
:107F7000012101FA00F009900121089801FA0BF2A1
:107F8000104018BF012000270190790902A807F0CE
:107F90001F0250F821100120904001427DD034F999
:107FA000021B0798081A019900290CBFA8EB0009C9
:107FB00008EB00093A4659460098FAF7F0FB0346E9
:107FC00010F4803F7BD0B9F1000F7DDA7AE04FF0FA
:107FD000000B002D41D90121089801FA0BF2104045
:107FE00018BF012000270190790902A850F821103C
:107FF00006E000007485001000EE03005443524672
:1080000007F01F0201209040014250D034F9021BBA
:108010000798081A019900290CBFA8EB000908EB82
:1080200000093A4659460098FAF7B9FBFE49014063
:1080300011F4803F18D0B9F1000F2ADA11F4F85189
:108040001CBFA1F5807141F4803122D110F4604F42
:108050001FD04FF4D05101E050E048E0A0F50050AF
:1080600010F4003F15D012E0B9F1000F11DD11F44A
:10807000F85118BFA1F580710BD110F4604F08D0F2
:10808000A0F500504FF4D05110F4003F01D04FF450
:108090008D3100F43830084302E01FE00FE013E0B8
:1080A00040F080033A4659460098FAF7CBFB7F1C14
:1080B000262F99D30BF1010BAB458CD317E0B9F107
:1080C000000F01DD06988343BAF1000FC4BF099881
:1080D00003433A4659460098FAF7B4FB7F1C262F13
:1080E000FFF453AF0BF1010BAB45FFF445AFBAF111
:1080F000000FC2BF05980BB0BDE8F08F0027002D20
:108100002ED904980DF1080A4FF0010BC0F58079C3
:1081100040F480780024600904F01F015AF8200020
:108120000BFA01F1084215D0224639460098FAF7B9
:1081300036FBC1B201EB590101EA0801B14288BF27
:10814000314620F0FF0040EA0103224639460098FC
:10815000FAF778FB641C262CDDD37F1CAF42D9D301
:10816000012005900BB0BDE8F08F2DE9F04F89B0EC
:10817000002204920A7800924A6802928A68039266
:108180004A7B0192B1F91060B1F912B00C6A8969A9
:10819000C0F105080591002837D0B8F1000F70DB59
:1081A0004FF00009002A6BD908F10800012101FAFB
:1081B00000FA401E01FA00F006900121059801FA2C
:1081C00009F2104018BF012000250790690902A894
:1081D00005F01F0250F821100120904001425FD0AD
:1081E00034F9020B0799A0EB0B0000290CBF371ADA
:1081F00037182A4649460098FAF7D1FA034610F490
:10820000803F3FD0002F41DA3EE00027002A4FD9BF
:108210000120059900FA07F20A4214BF4FF0010A43
:108220004FF0000A0025690902A805F01F0250F866
:1082300021100120904001421BD034F9020BBAF109
:10824000000FA0EB0B000CBFA6EB000906EB00092A
:108250002A4639460098FAF7A2FAB9F1000FC8BFCA
:1082600040F4803040F480532A4639460098FAF7AB
:10827000E9FA6D1C262DD6D301987F1C8742C7D3FF
:1082800016E01AE0002F01DD23EA0A03B8F1000F1F
:10829000C4BF069803432A4649460098FAF7D2FA23
:1082A0006D1C262D92D3019809F10109814584D3D3
:1082B000B8F1000F04BF01200490049809B0BDE894
:1082C000F08F2DE9F04F89B0002204920A780092D5
:1082D0004A6802928A6803924A7B0192B1F910605F
:1082E000B1F912B00C6A8969059150490969421ABD
:1082F000C2F10308814277D83DD101984FF00007C1
:10830000002871D90120059900FA07F20A4214BF2A
:108310004FF0010A4FF0000A0025690902A805F094
:108320001F0250F821100120904001421BD034F967
:10833000020BBAF1000FA0EB0B000CBFA6EB00097B
:1083400006EB00092A4639460098FAF728FAB9F1EF
:10835000000FC8BF40F4003040F400432A463946BD
:108360000098FAF76FFA6D1C262DD6D301987F1C62
:108370008742C7D34FE0B8F1000F51DB01984FF0AF
:108380000009002847D908F10D00012101FA00FA7F
:10839000401E01FA00F006900121059801FA09F249
:1083A000104018BF012000250790690902A805F0B8
:1083B0001F0250F8211001209040014223D034F9CF
:1083C000020B0799A0EB0B0000290CBF371A3718D6
:1083D0002A4649460098FAF7E2F9034610F4003FAE
:1083E00003D0002F05DA02E015E0002F01DD23EABB
:1083F0000A03B8F1000FC4BF069803432A46494652
:108400000098FAF71FFA6D1C262DCED3019809F1BA
:1084100001098145C0D3B8F1000F04BF01200490C9
:10842000049809B0BDE8F08F001F010074850010AA
:108430002DE9F14FADF54E7D0020C090BF9072B692
:10844000FAF716FD0746FCF725FB48B1FCF7CAFB17
:10845000C090FCF7B1FBFCF7CAFBBF90FCF7B7FB81
:10846000FAF700FCFAF716FBC590FAF70FFDC49077
:10847000FAF712FBFAF7A8FDBC900020FAF79BFD73
:108480000120F9F78EFCC8901120F9F78AFCC990F9
:108490000220F9F786FCCA901220F9F782FCCB90F3
:1084A000FCF741F9C390FCF726F94FF49350FCF721
:1084B00094F862B60020F9F745FCC2900121002033
:1084C000F9F733FC0020F9F752FC0021C19008466F
:1084D000F9F740FC0120F9F7C8FCCC900020FAF72E
:1084E00024FBC7900020FAF713FBC690F9F732F887
:1084F000CD900020F9F733F8002006469EAD45F8F0
:108500002060401C0C28FAD317F0070F4FF001042D
:108510000AD040F68C61FE489E9405F0AAFD40F614
:108520008C61FC4805F0A5FD17F0F00F47D0012045
:10853000F8F7E9FA38B19821F74805F09AFD982143
:10854000F64805F096FD1120F8F7DDFA38B19821CC
:10855000F34805F08EFD9821F24805F08AFD0220CF
:10856000F8F7D1FA38B19821EF4805F082FD98214B
:10857000EE4805F07EFD1220F8F7C5FA38B19821D3
:10858000EB4805F076FD9821EA4805F072FD0120E0
:10859000F8F7B9FA002818BFA0941120F8F7B3FA39
:1085A000002818BFA1940220F8F7ADFA002818BFE0
:1085B000A2941220F8F7A7FA002818BFA3944FF04E
:1085C000405ADFF874B3DFF874939E984FF0FF08B9
:1085D00058B330468DF8006001A9F9F748FA9DF8C4
:1085E0000000F9F764FA8DF80C009DF80000F8F728
:1085F00059FA8DF80D009DF80000F9F71CFC0028D1
:108600000CBF4FF0FF31002106918DF80E80B9F8B4
:108610000200ADF81000ADF812609DF80000F9F707
:10862000C6F9ADF81400CDE908AB9F986F4640B38A
:108630008DF8286007F12C013046F9F718FA9DF8FB
:108640002800F9F734FA8DF834008DF8354010968B
:108650008DF83680B9F80200ADF83800ADF83A6010
:108660009DF82800F9F7A3F9ADF83C009DF80C003F
:108670009DF80D1048430AEB40010BEB4000CDE99B
:108680001210A0984FF4806A02264FF0AA3BE0B384
:108690008DF8504007F154012046F9F7E8F99DF8AC
:1086A0005000F9F704FA8DF85C009DF85000F9F7D6
:1086B00080FA04FA00F08DF85D009DF85000F9F79B
:1086C00070FB1A908DF85E80B9F80400ADF8600078
:1086D000ADF862A09DF85000F9F769F9ADF86400B3
:1086E00097481C9097481D909DF85D00022809D975
:1086F0009DF85C10801E48431C9901EB40001C90C3
:108700008DF85D601A9800B100E007E09DF8500018
:108710004FF0AA31F9F733FBCDF868B0A198E0B378
:10872000112007F17C018DF87800F9F7A0F99DF888
:108730007800F9F7BCF98DF884009DF87800F9F716
:1087400038FA04FA00F08DF885009DF87800F9F702
:1087500028FB24908DF88680B9F80600ADF88800D3
:10876000ADF88AA09DF87800F9F721F9ADF88C00F2
:1087700075482690754827909DF88500022809D9EC
:108780009DF88410801E4843269901EB40002690F6
:108790008DF88560249800B100E007E09DF878002E
:1087A0004FF0AA31F9F7EBFACDF890B0A298E0B308
:1087B00007F1A40130468DF8A060F9F758F99DF84B
:1087C000A000F9F774F98DF8AC009DF8A000F9F756
:1087D000F0F904FA00F08DF8AD009DF8A000F9F76B
:1087E000E0FA2E908DF8AE80B9F80800ADF8B00030
:1087F000ADF8B2A09DF8A000F9F7D9F8ADF8B40033
:1088000053483090534831909DF8AD00022809D963
:108810009DF8AC10801E4843309901EB4000309029
:108820008DF8AD602E9800B100E007E09DF8A00043
:108830004FF0AA31F9F7A3FACDF8B8B0A398E0B396
:10884000122007F1CC018DF8C800F9F710F99DF856
:10885000C800F9F72CF98DF8D4009DF8C800F9F795
:10886000A8F904FA00F08DF8D5009DF8C800F9F7D2
:1088700098FA38908DF8D680B9F80A00ADF8D8008B
:10888000ADF8DAA09DF8C800F9F791F8ADF8DC0072
:1088900031483A9031483B909DF8D500022809D9DB
:1088A0009DF8D410801E48433A9901EB40003A905D
:1088B0008DF8D560389800B100E007E09DF8C80059
:1088C0004FF0AA31F9F75BFACDF8E0B0F8F774FB96
:1088D00010F0010F0BD0FEF7B0FF3C2807D1FCF7DA
:1088E000EBFA20B10420FCF796FAFCF76DFBFAF7DF
:1088F00021FB4FF00008C346C2464646C14604F07D
:1089000099F801287DD0BBF1800F7AD8AAA827E07A
:1089100000000130004001308C0E01308C4E0130DF
:10892000240F0130244F0130BC0F0130BC4F013007
:108930005410013054500130004000307485001054
:10894000CC090030CC490030CC0E0030CC4E003089
:108950004C1800304C5800304C1D00304C5D00303D
:10896000FAF76BFD00286ED0AAA804F0B8FFBC98F7
:10897000002818BF00273BD09EA850F82700A0B3BE
:1089800007EB8701684600EBC104207810F00F0F59
:108990002BD0F9F706FA10F0010F26D0216A257BBB
:1089A00001F0030000EB8502D21C22F0030221F04B
:1089B0000301CDE9BD1278A90C1878A8BD9905F07E
:1089C00062FB0020002D0BD9411934F8102034F837
:1089D000113024F81030401C24F811208542F3D8BF
:1089E00078A9BE9ABD9805F04EFB7F1C0C2FC3D30F
:1089F0001AF1010A7DD04FF0000A5046B0AD0127B0
:108A000000E077E00BF1010B45F82070401C0C28CA
:108A1000FAD3052E6ED2DFE806F003172A3D500088
:108A200000249EA850F8240048B104EB8401684655
:108A300000EBC1014846FFF744FC45F82400641CE4
:108A40000C2CEED33BE068E000249EA850F82400F4
:108A500048B104EB8401684600EBC1014846FFF7CA
:108A600084FB45F82400641C0C2CEED327E0002482
:108A70009EA850F8240048B104EB8401684600EB3E
:108A8000C1014846FFF749FA45F82400641C0C2C44
:108A9000EED314E000249EA850F8240048B104EB63
:108AA0008401684600EBC1014846FFF72FF945F8FD
:108AB0002400641C0C2CEED301E04FF001080121CE
:108AC000002055F82020CAB1401C0C28F9D3A9B1C8
:108AD0001F2E0DD2761CCE9807FA06F1014207D15F
:108AE000761C042E04D8CE9807FA06F10142F7D07E
:108AF00001E005E017E04FF0000901E009F101098C
:108B0000FAF7E7FCB8F1000F0DD1BC98002818BFA8
:108B1000F9F759F9FAF70EFAF1E6FEF767FDB8F141
:108B2000000F3FF4ECAEFAF7D4FCF9F7B5FF0520DF
:108B3000FCF771F90120C899F9F721F91120C999B9
:108B4000F9F71DF90220CA99F9F719F91220CB9902
:108B5000F9F715F9BC98FAF72EFA0020C199F9F740
:108B6000F9F80020C299F9F7E0F8CC98F9F77DF907
:108B7000C798F9F7DAFFC698F9F7CAFFCD98F8F762
:108B8000EEFCC59830B1C49810B1FAF7D3F901E002
:108B9000FAF782F9FBF77EFF48B1C098002818BFAA
:108BA000FBF77EFFBF98002818BFFBF7B2FFC39802
:108BB000002818BFFBF748FDB8F1000F0CBF0120DB
:108BC00000200DF54F7DBDE8F08F70B5FE4D1646C7
:108BD000D5F844231205120D1DD000281CBFC1F387
:108BE0000800FAF751FFD5F8480340F00100C5F836
:108BF0004803D5F8480320F00100C5F848030022D7
:108C0000341E23DDD5F8481340F2AF2011F0010FD8
:108C100008D1401E01D2002070BDD5F8481311F0D4
:108C2000010FF6D0D5F84403C0F30B000244D5F889
:108C3000480340F00100C5F84803D5F8480320F088
:108C40000100C5F84803641E002CDBDC1001B0FBFA
:108C5000F6F080B270BD2DE9F84F040016D0DB4865
:108C6000006CC0F30829FAF721FF49EA004200230B
:108C70007621072009F010F9D348D0F8401341F4C9
:108C80008031C0F84013322000900AE0FAF709FF63
:108C90000120BDE8F88F00BF00BF00BF00BF00BFCC
:108CA0000846411E0091F6D24FF0000840F2FF172F
:108CB000C246464608EB070000EBD0704510A9B24B
:108CC00064220120FFF781FFF0B1A04288BF6F1E30
:108CD00038BF05F101081ED1AA461FFA8AF14FF0EC
:108CE00064024FF00100FFF770FF04460023524674
:108CF0007721072009F0D0F8A4F5A8502C38A02837
:108D00009CBF0120BDE8F88FB9F1000F10D0484694
:108D1000FAF7BAFE0EE0011B48BF211A321B48BF0A
:108D2000A21B9142BCBFAA460646B845C2DDD4E7A5
:108D3000FAF7B7FE49F4803200237721072009F0C3
:108D4000ABF80020BDE8F88F2DE9F04FA04CADF650
:108D5000846D01262778FEF7E3FB012840F0B481FB
:108D600004F0A9FF9B480068B0F91E10B0F91C0080
:108D700005F0D9F917F0020F00F09D8101ADFEF763
:108D800041FF4FF00009A8B1B0E80E1001AC84E833
:108D90000E10B0E80E1005AC84E80E10B0E80E100E
:108DA00009AC84E80E1070E80C12806B0D91CDE9CF
:108DB0000E2022E0FF223C21284605F078F9864863
:108DC00001904FF4987002903C20CDE903095020A7
:108DD000CDE905094FF0FF30CDE908900A90ADF8D4
:108DE0003C900C908DF83E900B90CDF81C90CDF8F7
:108DF0003490CDF838908DF83F907848FAF784FF9A
:108E00000698401C0690F9F72DFF41F27C50FFF7C1
:108E100022FF6F49C860F9F7D4FF40F233380025CC
:108E2000CDF800909FE0284606F0F3F800287DD0AA
:108E3000008900EA080434F0CC0077D040F20F310A
:108E40002846FEF727FD002870D0FAF711F80099A0
:108E500000296CD1F9F7DCFE24F0EE0030F47E40FE
:108E60003CD01F20FFF7E4FA0090F9F715FE0098B8
:108E7000002875D1A6B314F0010F13D0FEF7DAFC69
:108E8000824605200DF1400BCDF8800E5846FAF7CA
:108E900024FB9AF925104FF464635A46DDF8800EDE
:108EA00006F0FDF814F0100F18D0FEF7C3FC824650
:108EB00007200DF1400BA890F9F7DAFF10F0300F02
:108EC0000CBF0220012010A9FAF757FB9AF92710CE
:108ED0004FF418735A46A89806F0E1F8009830BB92
:108EE00014F0220F06D0FCF708FE0090F9F7D4FD2D
:108EF0000098E0B9DEB114F0020F16D0FCF70AFAC0
:108F00008346374801783748007848434FEA400A9B
:108F1000FEF790FC4FF0060C5FEA0B0205D090F9CB
:108F200026105346604606F0BAF801E01AE017E052
:108F300014F0200F14D0FCF784F904462A48017875
:108F40002A48007808444FEA400AFEF773FC0146BD
:108F50000820220004D091F92810534606F09FF80B
:108F6000FEF737FE6D1C06F050F8A842009803D9B2
:108F700000283FF458AF03E0002808BF012000D0CC
:108F8000002018B1FCF799FE012834D0089800237E
:108F9000401C0890502005901A462121072008F017
:108FA0007BFF00231A461946FE20CDF80090FCF7FF
:108FB0007AFF01AC06F001F890B381690991C169AB
:108FC0000A9141690B9113E000500040006000409D
:108FD00074850010BC8600105443524600EE030016
:108FE0005B8500105C8500105D8500105E850010BB
:108FF000C0680C9028E017F0080F14BFA220A12031
:10900000C5490590C86860B1C448006CC0F3082029
:10901000ADF83C009DF83E00401C8DF83E0007E096
:109020000CE0ADF83C909DF83F00401C8DF83F00EF
:10903000C1F80C900798401C0790BAE74FF0FF303A
:109040000C900B900A900990B54801904FF49870DD
:1090500002903C20CDE903090021A368224608467E
:1090600052F820C0401C6144B0EB930FF8D34D423E
:10907000FF224FF4007110A8E56005F018F8A2680F
:10908000F4E8040110AB83E827000FCC14AD85E8A9
:109090000F000FCC18AD85E80F00D4E90001A268DD
:1090A000A04CCDE91C011E922046FAF72DFE10A916
:1090B0002046FAF7CBFE0020FCF73FFC00233A469F
:1090C0004021072008F0E8FE0DF6846DBDE8F04F62
:1090D00003F05EBB904A022804BF1181704707DC91
:1090E000002804BF51807047012808BF9180704755
:1090F000112804BFD1807047122808BF51817047E2
:10910000014600200229844A04BFB2F908007047D2
:1091100009DC002904BFB2F902007047012908BF29
:10912000B2F904007047112904BFB2F90600704774
:10913000122908BFB2F90A00704770B50126FEF780
:1091400061FD20B10069A12818BFA22801D000202C
:1091500070BD002405F059FF002834D9204605F0E1
:1091600058FF00281EBF058925F0CC0030F47C4054
:1091700024D040F20F312046FEF78CFBF0B115F001
:10918000010F0AD0FAF7BEF938B944F4807200230F
:109190002021072008F080FE002615F0100F0BD0CC
:1091A0000120FAF706FA38B944F48052002320214E
:1091B000072008F071FE0026FEF70BFD641C05F089
:1091C00024FFA042CAD8304670BD0020704700205E
:1091D00070475148407870474F49002048707047A9
:1091E00070B5002105220846FFF7EFFC00234A4A2C
:1091F000002833D05178002908BF5361A0F5A85C3E
:10920000ACF1750CBCF10E0F28D9491CC9B25170D4
:10921000D2F814C00A296044506129D93F495370DB
:10922000096CC1F30824DCB14EF6E401884224BF86
:109230004EF6C471814213D34EF6544181422CBF85
:10924000651C651E2846FAF71FFC44EA0542002308
:109250007521072008F020FE012070BD537007E043
:1092600041F27C50FFF7F7FC00281CBF012070BDC5
:10927000002070BD10B5FEF7C5FC38B3284A016860
:10928000914223D14168B1F5987F1FD8D0F808C02A
:109290000146BCF5007F19D800220B461146B2EBFF
:1092A0009C0F07D253F82140491C2244B1EB9C0F7C
:1092B000F8D35AB9188F00281CBFA0F57F41B1F12F
:1092C000FF0103D0FAF7E0FB012010BD002010BD24
:1092D00010B5FEF797FCD8B1114A0168914217D139
:1092E0004168B1F5987F13D8D0F808C00146BCF5A5
:1092F000007F0DD800220B461146B2EB9C0F09D21D
:1093000053F82140491C2244B1EB9C0FF8D30AB119
:10931000002010BD188F10BD748500100060004043
:109320005443524600EE030070470020704710B5CA
:1093300003F00700042808BFFEF7B6F9002010BDAF
:1093400010B403F007020024FE4BDFF8FCC3012A2F
:1093500002D0022A17D013E005208CF80000FB4849
:10936000CCF80C4000681A68532111701A68452126
:1093700051701A68010A91701968C87018680471F0
:1093800010BC002070479CF80020052A14D1DCF89E
:109390000C20052A28BF104605D21B689B5C037071
:1093A000501CCCF80C00052806D10120CCF80C404C
:1093B000087003208CF8000010BC0120704770B5C5
:1093C00003F007020125DF4CDF4B4FF0000C012AB0
:1093D00002D0022A25D022E005201870DB48C3F80D
:1093E0000CC000682268AC2111702268010A51701B
:1093F000216888702068C570206880F804C005F076
:109400007DFD48B1D24D286804F08FFD20B1286859
:109410002168007E487102E02168FF204871002029
:1094200070BD1A78052A10D1DA68062A28BF1046BE
:1094300004D22468A45C0470501CD860062804D1AF
:10944000C3F80CC00D7003201870012070BD03F02C
:109450000702022A1CBF0020704720220270012050
:10946000087070472DE9F041B74F0D46064613F0DE
:10947000070F04D003F00700022808D004E012F020
:10948000040F1CBF0020B8700020BDE8F08103F07D
:1094900079F9002814BF0124002403F076F900288C
:1094A00014BF0222002242EA0403B878002814BF45
:1094B0000422002242EA0300307001202870BDE837
:1094C000F08170B503F0070C00269F4C9D4DBCF158
:1094D000010F0AD0204613F0070F00780DD0BCF121
:1094E000040F08BF062818D029E0E6602868067037
:1094F000286846700520207021E005281FD1E0680B
:10950000022803D22B681A54401CE060022816D1AE
:109510000120E6600870062010E0286800785528D1
:109520000BD128684078AC2818BFBC2805D1286822
:109530000122411C062003F00BF9032020700020BB
:1095400070BD70B503F0070200257E4C7E4B012AEA
:1095500002D0022A24D021E005201870DD6003F03B
:10956000C3F841F6E8710144B0F5783F10D8CA78E5
:10957000086862F31F60774A904208BF002007D155
:109580000A18236812791A54401C1428F8D305E0ED
:10959000002021680D54401C1428FAD3002070BD0F
:1095A0001A78052A13D1DA68142A28BF104607D280
:1095B000D4F800C01CF802C080F800C0501CD8606D
:1095C000142804D10120DD600870032018700120E8
:1095D00070BD70B503F0070200255A4C5A4B012AA2
:1095E00002D0022A3FD03CE005201870DD6003F075
:1095F0007BF841F6E8710144B0F5783F2BD8CA7882
:10960000086862F31F60534A904224D12268087CA4
:1096100010702268487C50702268887C90702068A6
:10962000CA7CC27020680A7A02712268487A507136
:109630002268887A90712268C87AD0712268087D81
:1096400010722268487D50722268887D9072C87DB1
:109650002168C87205E0002021680D54401C0C28C8
:10966000FAD3002070BD1A78052A13D1DA680C2AC3
:1096700028BF104607D2D4F800C01CF802C080F8FA
:1096800000C0501CD8600C2804D10120DD60087097
:1096900003201870012070BD70B503F0070200258B
:1096A000284C294E012A02D0022A36D033E005F098
:1096B00084FC40B3D0E906212368C0681A70D4F84E
:1096C00000C0130A8CF80130D4F800C0130C120E3D
:1096D0008CF802302368DA702268117123680A0A54
:1096E0005A7123680A0C090E9A712268D171216897
:1096F00008722268010A51722268010C9172010EEF
:109700002068C17204E021680D54401C0C28FAD373
:1097100005203070F560002070BD3278052A10D128
:10972000F2680C2A28BF104604D223689B5C0370A1
:10973000501CF0600C2804D10120F5600870032053
:10974000307009E0A468020094850010044C0040C9
:10975000BC86001034CD12AB012070BD70B503F093
:1097600007020024F94DFA4B012A02D0022A3ED00A
:109770003BE0052018700026DC6002F0B5FF00F524
:109780000051B0F5783F98BF11F0030F27D1F14A8F
:109790000868904204BF0022104620D151F82030C2
:1097A000401C1A440728F9D302B1C6B128680A7CC4
:1097B00002702A68487C50702A68887C90702A68F9
:1097C000C87CD0702A68087D10712A68487D507165
:1097D0002A68887D9071C87D2968C87105E00020DD
:1097E00029680C54401C0828FAD3002070BD1A7850
:1097F000052A13D1DA68082A28BF104607D2D5F8FF
:1098000000C01CF802C080F800C0501CD8600828B6
:1098100004D10120DC60087003201870012070BDA5
:109820002DE9F04103F0070C0027C94E4FF0050861
:10983000BCF1010F0DD013F0070F0FD03246BCF171
:10984000020F127810D0BCF1040F08BF062A26D0F0
:1098500058E086F800807770F76053E07270BE4879
:10986000F062062030704DE0052A15D1F268042A16
:1098700028BF104609D2C2F10303D6F82CC0DB0082
:109880002CFA03F30370501CF060042804D101206B
:10989000F7600870032030700120BDE8F081707817
:1098A0000125002410F0010F11D002F01DFFB0F5CA
:1098B000783F23D86A030021B1EB900F07D252F80A
:1098C000043B491C1C44B1EB900FF8D3B5B1707840
:1098D00010F0020F0ED005F070FB78B18268002105
:1098E000B1EB920F06D250F8043B491C1C44B1EB7B
:1098F000920FF8D3002D18BFF46200D1F762777091
:1099000086F800800020BDE8F081F0B503F0070C78
:1099100000268E4D8E4C83B0BCF1010F0ED013F09B
:10992000070F1DD0224603271278BCF1020F26D064
:10993000BCF1040F08BF062A36D03CE002AA01A9F8
:10994000684603F084FB05202070296801980870A0
:10995000296800984870296802988870E6602AE0B3
:10996000E068032803D229680A54401CE0600228FA
:1099700021D306212170032808BFE6601BE0052AD9
:109980000FD1E268032A28BF104604D22B689B5CE3
:109990000370501CE060032803D10120E6600870CA
:1099A000277003B00120F0BD2868827801784078E4
:1099B00003F040FB277003B00020F0BD08B503F0B2
:1099C000070001280AD105F099FA38B101208DF875
:1099D0000000024669460D2002F0BAFE002008BDD4
:1099E00008B503F0070001280AD105F087FA38B15D
:1099F00000208DF80000012269460D2002F0A8FE2B
:109A0000002008BD08B503F00700012809D105F0C2
:109A100075FA30B103208DF800000122694602F08A
:109A200097FE002008BD0020704708B503F007002E
:109A300001280AD105F062FA38B10B208DF8000038
:109A400001226946032002F083FE002008BD1FB5F5
:109A500013F0070F0ED105F051FA58B19DF8080028
:109A6000F0280AD005F04AFA20B1012202A9092003
:109A700002F06EFE04B0002010BDFEF7E9F8F9E731
:109A80000020704770B503F00700304C304D0128BE
:109A900008D013F0070F12D0042804BF2878062836
:109AA00016D01FE00020E860216808702168487027
:109AB000216888702168C8700520287012E0E86865
:109AC00004280FD221680A54401CE860062008E0F0
:109AD00005F014FA30B104221046216802F038FE75
:109AE00003202870002070BD10B503F00700012886
:109AF00004D104F0E0F8164900200871002010BDE0
:109B000010B503F0070C124CBCF1010F06D013F096
:109B1000070F09D0BCF1020F20D015E00020E06053
:109B200008F0B1F9E0610FE0E068002804BF10021E
:109B3000E06106D0012804D1E0691043E06108F03B
:109B4000A1F9E068401CE060002010BDA46802009C
:109B50009485001054464953EFBEADDEE26812B161
:109B6000012A04D007E0A18B090A017003E0237FDA
:109B7000037001200870501CE0600120E5E710B57B
:109B800003F0070CFE4CBCF1010F06D013F0070FD9
:109B900009D0BCF1020F18D015E00020E06008F0F9
:109BA00075F9E0610FE0E068002804BF1002E06191
:109BB00006D0012804D1E0691043E06108F069F99A
:109BC000E068401CE060002010BDE26812B1012A8C
:109BD00004D007E0A18B090A017003E0237F037022
:109BE00001200870501CE060012010BD70B503F02A
:109BF000070CE34D0E460446BCF1010F06D013F0EE
:109C0000070F07D0BCF1020F18D015E00020E86064
:109C1000286111E0E868002804BF1002E86108D05C
:109C2000012806D1E869104381B2E861E88811F0A3
:109C3000C5FDE868401CE860002070BD2869022866
:109C40000ED2E88811F0C0FD2B6982B2002B04BF50
:109C5000100A207004D0012B02D122700120307034
:109C60002869401C2861012070BD10B403F0070C66
:109C7000C34CBCF1010F08BF00200BD013F0070F3D
:109C800003D0BCF1020F09D005E0E068002808BF4E
:109C9000E280401CE06010BC00207047E2681AB906
:109CA000A379037001200870501CE06010BC0120F3
:109CB00070472DE9F047064603F00700B04F89468C
:109CC000012808BF002037D0DFF8B882AE4D13F06E
:109CD000070F02D0022833D02FE0F868002808BF11
:109CE0007A7027D0012804BF1002F86122D0022820
:109CF00020D1F8691043F8617E7884B205F0FEF84F
:109D0000C0B1062E16D2DFE806F00306090C1013C8
:109D1000A8F80E400EE0A8F80C400BE028688483F9
:109D200008E02868A0F8144104E02868048601E0EF
:109D300028684486F868401CF8600020BDE8F08779
:109D4000386902282AD297F801A0002405F0D6F835
:109D5000C8B1BAF1060F16D2DFE80AF00306090C03
:109D60001013B8F80E400EE0B8F80C400BE028686D
:109D7000848B08E02868B0F8144104E02868048E59
:109D800001E02868448E3869002804BF200A30703A
:109D900004D0012802D1347089F800003869401CD1
:109DA00038610120BDE8F0872DE9F0411C461546D9
:109DB0000E46074605F0A2F888B1724814F0070F66
:109DC00004D004F0070102290CD008E0002D1ABFCE
:109DD00090F80801C0084FF0FF300CF0D1FE0020D1
:109DE000BDE8F08190F80801C0083870012030709B
:109DF000BDE8F0812DE9F0411C4615460F460646A8
:109E000013F0070F08D105F079F828B1022D3CBFF7
:109E100028460AF046FA03E004F00700022802D0C0
:109E20000020BDE8F0810AF035FA3070012038706A
:109E3000BDE8F08170B503F007020026534C504D89
:109E4000012A02D0022A15D012E009F0F5F92168A2
:109E50000870FDF765FB2168487004F0B5FD2168C6
:109E60008870FDF763FB2168C87005202870EE60DC
:109E7000002070BD2A78052A10D1EA68042A28BF7C
:109E8000104604D223689B5C0370501CE8600428D1
:109E900004D10120EE60087003202870012070BDFD
:109EA00070B503F0070C394C0026354DBCF1010F9D
:109EB00008D013F0070F08BF6A716DD0BCF1020F14
:109EC0006CD069E0FDF79EFE697901293AD00A213C
:109ED000696100283ED04169FF292CBFFF21C9B22A
:109EE000226811708169FF2934BFC9B2FF2122683D
:109EF0005170C169FF2934BFC9B2FF212268917036
:109F00002268017CD170226890F820101171018CB8
:109F10002268090A5171016A2268090C9171016A6B
:109F20000A0E2168CA71016BFF2934BFC9B2FF2133
:109F300022681172406BFF2834BFC0B2FF20216835
:109F4000487228E0112001466861FF22206804F071
:109F5000AEF820E0206806702068467020688670A1
:109F600021685020C8702168FF200871216848715D
:109F7000216888712168C87120680672206809E02C
:109F800094850010442E0110BC860010A4680200C5
:109F900002E003E04672EE60002070BD6B69EA6883
:109FA0009A4228BF104607D2D4F800C01CF802C05D
:109FB00080F800C0501CE860984206D10120EE6095
:109FC00008706879002818BF6E71012070BD03F019
:109FD0000702FF4B4FF0000C012A08BFC3F80CC06A
:109FE00001D0022A01D000207047DA68022A3DBF62
:109FF00080F800C0501CD8601046022803D1012010
:10A00000C3F80CC00870012070472DE9F0470646E0
:10A0100003F00700EE4F8A464FF00008012808BF02
:10A02000C7F80C8001D0022802D00020BDE8F087DC
:10A03000F868A0BB0024254602F056FB014600F557
:10A04000005018384FF400524FF04009B1F5783FF6
:10A0500020D890F803C003686CF31F63DFF874C363
:10A06000634517D1091FB4EB910F06D252F8043B98
:10A07000641C5D40B4EB910FF8D3C17D406961F37E
:10A080001F60A84206D104F039FF012804BF8020D8
:10A09000307001D086F80090F868401CF860012804
:10A0A00003D1C7F80C808AF800000120BDE8F087D2
:10A0B0002DE9F04103F007020026C74CC44D012AE8
:10A0C00002D0022A5CD058E0C448006805202870FD
:10A0D00004F014FF00284FD0C14F386803F025FF6B
:10A0E000002849D011F04BFB804611F04CFB396839
:10A0F0000A7E12F0040F11D0C98A2268090A117071
:10A1000039682268897D517039682268898A090A0C
:10A11000917039682268097DD17010E0898A2268BF
:10A12000090A117039682268097D517039682268FE
:10A13000C98A090A917039682268897DD1702268BC
:10A140004FEA18211171216881F805802268010AFF
:10A1500091712168C87138682268817C1172226807
:10A16000017C5172018B2268090A91722268817CFC
:10A17000D1722168007C0873EE600020BDE8F08198
:10A180002A78052A10D1EA680D2A28BF104604D281
:10A1900023689B5C0370501CE8600D2804D10120EB
:10A1A000EE600870032028700120BDE8F0812DE9E1
:10A1B000F04703F007020025874C854B012A02D0A7
:10A1C000022A5CD058E0052018700026DD6002F0FD
:10A1D0008BFA00F50053B0F5783F98BF13F0030FEA
:10A1E00044D1804A1968914204BF0022114608D127
:10A1F00053F821C0491C62440729F9D3002A08BF3B
:10A2000001269F7C93F813807EB3002241F6E8710B
:10A210000144B0F5783F07D8CB78086863F31F6036
:10A220006C4B984208BF01228E7C91F81390002A53
:10A2300008BF002013D004F0C0FE216880690E70B2
:10A24000216881F801902268010C000E917021684C
:10A25000C87020680771206880F805800CE02168CC
:10A260000D54401C0628FAD306E0FFE700202168C1
:10A270000D54401C0628FAD30020BDE8F0871A7858
:10A28000052A13D1DA68072A28BF104607D2D4F866
:10A2900000C01CF802C080F800C0501CD86007281D
:10A2A00004D10120DD600870032018700120BDE892
:10A2B000F08770B5054603F007000C46022829D147
:10A2C00004F01CFE30B3464800220068037EC3F34E
:10A2D00080008000C3F3400100EB410003F0010166
:10A2E0000844082812D2DFE800F00406080A0C0E21
:10A2F000111004220AE0052208E0062206E00722E7
:10A3000004E0022202E0032200E001222A70012080
:10A31000207070BD002070BD10B503F0070C2C4CF0
:10A32000BCF1010F06D013F0070F0AD0BCF1020FE9
:10A330001AD017E00020E060206111F0A1FAE0617E
:10A3400010E0E068002804BF1002E06107D0012897
:10A3500005D1E0691043E06180B211F08EFAE06847
:10A36000401CE060002010BD2269022A0BD212B10D
:10A37000012A04D007E0A18B090A017003E0237FC2
:10A38000037001200870501C2061012010BD70B5C1
:10A3900003F0070100260E4D0446012908BF2E6375
:10A3A00001D0022901D0002070BD286B002804BF15
:10A3B0000D4803F0BDFE296B102928BF267002D27C
:10A3C0000948405C2070481C2863012070BD0000D3
:10A3D0009485001034CD12ABA4680200044C0040F8
:10A3E000BC8600105446495340A900102DE9F041A5
:10A3F00003F007010026F84D0746012908BF2E6328
:10A4000001D0022902D00020BDE8F08195F830008B
:10A4100000F00F042879204304D1F04803F088FEAF
:10A4200001202871052C28BF2E71EC48005D387082
:10A43000286B401C28630120BDE8F08170B50446FC
:10A4400003F007000D4602281CBF002070BD03F07A
:10A4500074FE20700120287070BD2DE9F04103F0DA
:10A4600007020026DE4DDC4C012A02D0022A1FD052
:10A470001BE005202070002211461046E66002F025
:10A48000E6FD4FF6FF7101EA40006061297822295C
:10A4900004BF0C306061FDF743F8032803BF287840
:10A4A0002028D04802F0E6FDA0620020BDE8F0813F
:10A4B0002278052A1DD1D4F814C0E268624528BF6D
:10A4C000104607D212F0010F1CBF6378037013D03F
:10A4D000501CE06060450CD10120E660087003204C
:10A4E0002070FDF71DF8032806BF2878202802F009
:10A4F000CEFD0120BDE8F081A76A22F00103FB5ADE
:10A500001F0A07706370E3E770B503F007020025C8
:10A51000B14C012A02D0022A11D00EE0B248052225
:10A520000068B0F91210B0F9100022700844400021
:10A53000E560606103F032F8A062002070BD22780F
:10A54000052A17D1D4F814C0E268624528BF104626
:10A5500007D212F0010F1CBF637803700CD0501C9F
:10A56000E060604506D10120E5600870032020709E
:10A5700003F022F8012070BDA66A22F00103F35A0D
:10A580001E0A06706370EAE70020704770B50D463A
:10A59000044613F0070F04D003F00700022805D08B
:10A5A00002E01046FCF7B0FF002070BDFCF7AFFFE3
:10A5B00020700120287070BD70B503F007020325DC
:10A5C000854C012A02D0022A17D014E004F096FD2F
:10A5D0000646FCF79CFF0146304605F007F820626E
:10A5E00000281ABF052020702570304604F0E5FFD2
:10A5F00060620020E060002070BD2278052A0BD147
:10A60000236AE2689B5C0370501CE060626A9042BF
:10A6100002D3012008702570012070BD0020704712
:10A62000002070477FB51C460E46054613F0070F05
:10A6300008D104F063FC28B1012202A9272002F00E
:10A6400087F803E004F00700022802D004B00020DD
:10A6500070BD02F0D8FD28700120307004B070BDCC
:10A660002DE9F04103F0070200275B4E88460546BE
:10A67000012A02D0022A0BD007E0052030701220F8
:10A68000F760706102F0F6FCB0620020BDE8F08176
:10A690003078052819D1F2687069824228BF1046C7
:10A6A00008D212F0010F1CBF7078287010D0F0682B
:10A6B000401CF0607169884207D10120F76088F87A
:10A6C00000000320307002F0E2FC0120BDE8F081C0
:10A6D000002402F098FD012804D1F068B16A20F04E
:10A6E00001000C5A200A28707470E0E770B50D461E
:10A6F000044613F0070F04D003F00700022805D02A
:10A7000002E0104604F0F7FC002070BD04F0F6FCF7
:10A7100020700120287070BD7FB51C460E4605468E
:10A7200013F0070F08D104F0E9FB28B1012202A9B8
:10A73000212002F00DF803E004F00700022802D007
:10A7400004B0002070BD08F007FF287001203070B1
:10A7500004B070BD7FB51C460E46054613F0070FCA
:10A7600008D104F0CBFB28B1012202A9222001F07C
:10A77000EFFF03E004F00700022802D004B000203D
:10A7800070BD08F0EFFE28700120307004B070BD7D
:10A790007FB51C460D46064613F0070F08D104F09E
:10A7A000ADFB28B1012202A91D2001F0D1FF03E079
:10A7B00004F00700022802D004B0002070BDFCF7AE
:10A7C000E7FF0446FCF7D0FF44EA40003070012068
:10A7D000287004B070BD00009485001040A90010DE
:10A7E000DD85001064260110BC8600107FB51C4674
:10A7F0000E46054613F0070F08D104F07FFB28B181
:10A80000012202A90C2001F0A3FF03E004F00700DD
:10A81000022802D004B0002070BD08F00DFD2870A1
:10A820000120307004B070BD7FB51C460E46054651
:10A8300013F0070F08D104F061FB28B1012202A92F
:10A840000F2001F085FF03E004F00700022802D08A
:10A8500004B0002070BD10F081FA00F00F0040F04D
:10A86000100028700120307004B070BD2DE9F04157
:10A8700003F0070CFD4D0E460746BCF1010F07D053
:10A88000FB4C13F0070F07D0BCF1020F1BD017E0F1
:10A890000020E860286113E0E86804283CBF2168D4
:10A8A0000A54032809D1206821680068C97800BAD1
:10A8B00020F0FF000843FBF76DFDE868401CE860EE
:10A8C0000020BDE8F081286970B9FBF768FD2168B8
:10A8D00020F07E42100E08702168100C487021682C
:10A8E000100A88702068C2702A69042A06D220687B
:10A8F000032A805C387004BF01203070501C28612E
:10A900000120BDE8F0817FB51C460D46064613F0D8
:10A91000070F08D104F0F2FA28B1012202A9102091
:10A9200001F016FF03E004F00700022802D004B093
:10A93000002070BD10F016FA00F00F0410F00EFAAF
:10A9400064F31F1030700120287004B070BD70B522
:10A95000C64D144613F0070F04D003F00702022A75
:10A9600006D003E01046F5F728FD6C63002070BDAB
:10A9700095F8342002700120087070BD70B514463F
:10A980000E46054613F0070F04D003F00700022817
:10A9900008D005E01046FBF7E1FC60B203F0D2FB03
:10A9A000002070BDFBF7E3FC28700120307070BD03
:10A9B0002DE9F04103F0070CAD4DAC4C4FF0000811
:10A9C000BCF1010F0DD013F0070F1AD02246A94E8B
:10A9D00003271278BCF1040F1DD0BCF1020F3DD04B
:10A9E0002FE0C4F80C80286880F80080286880F880
:10A9F0000180286880F80280286880F8038005209C
:10AA000007E0E06804281CD229680A54401CE06072
:10AA10000620207015E0062A13D104F06FFA80B1E9
:10AA20002868007810B101280ED009E02868407825
:10AA30000028706814BF40F0800020F08000706033
:10AA400027700020BDE8F0812868407800287068F1
:10AA500014BF40F4007020F40070F0E7052A0FD115
:10AA600072687368C2F3C01203F4007342EA5312AF
:10AA70002B681A7002700120C4F80C8008702770CF
:10AA80000120BDE8F08110B503F00702774C012AE0
:10AA900002D0022A0DD00AE004F0FEFD002120625F
:10AAA00000281ABF4FF4056060626162E160002017
:10AAB00010BD636AE2689A4228BF104607D2D4F8F4
:10AAC00020C01CF802C080F800C0501CE060984212
:10AAD00004BF01200870012010BD10B4DFF898C138
:10AAE00013F0070F04D003F00702022A13D00FE07F
:10AAF000012A04BFDCF8000040F0010006D0002A63
:10AB000004BFDCF8000020F0010001D1CCF8000007
:10AB100010BC00207047DCF80030002213F0010F59
:10AB200018BF0122534BD3F804C0544B1B68B3F831
:10AB3000F030C3F30334012303FA04F41CEA040FD6
:10AB400018BF42F0020202700B7010BC0120704767
:10AB500070B514460E46054613F0070F04D003F0F7
:10AB6000070002280ED00BE0002C14BF01200020AB
:10AB700003F080F824B13F48016821F4405101609E
:10AB8000002070BD03F07DF8002814BF01220022D0
:10AB90002A700120307070BD2DE9F04103F0070CE0
:10ABA000324C0F468046BCF1010F12D0314E13F0EB
:10ABB000070F4FF0030510D02046BCF1020F0278BA
:10ABC00026D0BCF1040F02BFE0680128062A33D06A
:10ABD00036E005202070002018E0E06810B1012860
:10ABE00004D011E06270062020700DE0716860787A
:10ABF00000EA020319437160716820EA020291437E
:10AC00007160F9F7EDF92570E068401CE06017E02D
:10AC1000E068012808BF062A03D16078F9F7F6F941
:10AC20002570706888F8000001203870E068401CCA
:10AC3000E0600120BDE8F0816078F9F7E7F9257060
:10AC40000020BDE8F08170B5044603F007000D4612
:10AC500002281CBF002070BDFCF756FD002814BF61
:10AC60000122002222700120287070BD94850010FE
:10AC7000A468020000100040144C0040BC86001084
:10AC800070B50D46044613F0070F04D003F007001B
:10AC9000022805D002E0104608F0ECF9002070BD53
:10ACA00008F0EBF920700120287070BD70B50D46DA
:10ACB000044613F0070F04D003F00700022805D064
:10ACC00002E01046F6F77BF9002070BDF6F77AF93E
:10ACD00020700120287070BD70B503F00702DFF806
:10ACE00050C40C460546012A08BF05200DD013F0BC
:10ACF000070F08BF062008D0022A09D0042A04BF83
:10AD00009CF80000062809D00EE08CF800000BE04B
:10AD1000FCF74CFD28700120207070BD03208CF8DA
:10AD200000000120FCF745FD002070BD70B503F068
:10AD30000702FF4D0E460446012A04BF0020E860CA
:10AD400001D0022A01D0002070BD11F035FDEA6863
:10AD5000002A04BF000A207004D0012A02D120700A
:10AD600001203070501CE860012070BD03F0070224
:10AD700010B4EF4B012A04BF0020D86001D0022A92
:10AD800002D010BC00207047DA68022A0CD24FF0C3
:10AD9000010C002A08BF80F800C005D0012A03D1A9
:10ADA0004024047081F800C0501CD86010BC012001
:10ADB000704770B5044603F007000D46022807D01F
:10ADC00013F0070F04BF1046FCF798FB002070BD7E
:10ADD000FCF797FB20700120287070BD70B503F060
:10ADE000070C0026D34DD24C82B0BCF1010F06D027
:10ADF00013F0070F1FD0BCF1020F2DD029E06846D9
:10AE00000EF086FBBDF80000296800090870BDF847
:10AE10000200C0F30321BDF8000041EA00102968D8
:10AE200048702968BDF80200887028689DF80410F1
:10AE3000C170E6600DE0E06804283CBF29680A5450
:10AE4000401CE060042804D104221420296801F089
:10AE50007FFC02B0002070BDE268042A02D22B6899
:10AE60009B5C0370501CE060042804D10120E66064
:10AE700008700320207002B0012070BD70B503F08F
:10AE8000070C0026AB4DAA4CBCF1010F06D013F005
:10AE9000070F0CD0BCF1020F19D016E00EF02BFBFF
:10AEA0002A68010A117029684870E6600DE0E068C0
:10AEB00002283CBF29680A54401CE060022804D1E3
:10AEC00002221520296801F043FC002070BDE268D1
:10AED000022A02D22B689B5C0370501CE06002289F
:10AEE00004D10120E660087003202070012070BDAD
:10AEF00070B503F0070C00268E4D8D4CBCF1010F90
:10AF000006D013F0070F12D0BCF1020F1FD01CE0C7
:10AF10000EF0D9FA2A68010E11702A68010C5170DE
:10AF20002A68010A91702968C870E6600DE0E0683F
:10AF300004283CBF29680A54401CE060042804D15E
:10AF400004221620296801F003FC002070BDE2688D
:10AF5000042A02D22B689B5C0370501CE06004281A
:10AF600004D10120E660087003202070012070BD2C
:10AF70002DE9F04703F0070C6E4C00276C4EBCF136
:10AF8000010F0FD013F0070F4FF0010833D0032546
:10AF9000BCF1020F56D0BCF1040F04BF3078062874
:10AFA00061D087E00EF0DFFA05460EF0EDFA80463C
:10AFB0000EF0D3FA81460EF0E1FA0146206880F8DF
:10AFC0000090226808095070C5F3032040EA011080
:10AFD000216888702168280CCD702168087121686B
:10AFE000280E487121684FEA182081F806802168F0
:10AFF000C871F7605EE0F068002804BF23681A702B
:10B0000023681B78012B01D03BB110E0002818BF4A
:10B0100008283CBF23681A5409E02068077120689B
:10B020004771206887712068C7710720F060F06859
:10B03000401CF06008283DD1F76081F800800620B0
:10B04000307037E0F268082A02D223689B5C0370F4
:10B05000501CF060082803D1F76081F8008035703B
:10B060000120BDE8F087206800780EF079FA2068AA
:10B07000216840788978000140EA11100EF081FAC9
:10B080002168206822688978407901F00F0140EA40
:10B09000016021681279C978090441EA0221084354
:10B0A0000EF065FA2068C08840BA0EF070FA0EF013
:10B0B00073FA35700020BDE8F08770B503F0070C17
:10B0C00000261C4D1A4CBCF1010F06D013F0070FDF
:10B0D0000CD0BCF1020F19D016E00EF0EFF92A687F
:10B0E000010A117029684870E6600DE0E0680228E6
:10B0F0003CBF29680A54401CE060022804D128683B
:10B10000008840BA0EF0D6F9002070BDE268022A2D
:10B1100002D22B689B5C0370501CE060022804D1B3
:10B120000120E660087003202070012070BD00003F
:10B1300094850010A468020010B503F00702FE4CCD
:10B14000012A02D0022A27D024E004F0A5FA002325
:10B15000002804BF236263621BD000F1500121620A
:10B160004168B1F5887F90F820100CD390F8212029
:10B1700001EB020C01FB02C190F8222090F82300A1
:10B180001044084404E090F822000A1801FB002053
:10B190006062E360002010BD636AE2689A4228BFE3
:10B1A000104607D2D4F820C01CF802C080F800C0B6
:10B1B000501CE060984204BF01200870012010BDBF
:10B1C00003F00702012A02D0022A05D002E0DA4980
:10B1D0000020C86000207047012202700A701046EB
:10B1E000704710B513F0070F04D003F00702022ACE
:10B1F00005D002E0104601F057FF002010BDCF4AF5
:10B20000127802700120087010BD10B513F0070FFE
:10B2100004D003F00702022A05D002E0104602F033
:10B22000D8F9002010BDC64A1278027001200870BB
:10B2300010BD0020704703F00702BF4B012A04BF76
:10B240000020D86001D0022A01D000207047DA68BF
:10B250004FF0010C002A08BF80F800C0501CD860D5
:10B26000012808BF81F800C0012070471FB513F006
:10B27000070F07D103F042FE20B1012202A90B20E3
:10B2800001F066FA04B0002010BD70B503F00700AD
:10B29000A94C1546012804BF0020E06024D013F01B
:10B2A000070F21D103F02AFEF0B1E068A54E032874
:10B2B0003CBF31680D54401CE060032814D1F7F7FF
:10B2C000D1FC3068B0F8010045BAF7F7E3FB0400A1
:10B2D00018BFF7F74AFE306829460078F6F747FAB4
:10B2E000002C18BFF7F744FE002070BD70B503F0C6
:10B2F0000700914D1446012804BF0020E86020D0CB
:10B3000013F0070F1DD103F0F9FDD0B1E8688D4EA1
:10B3100002283CBF31680C54401CE860022810D160
:10B32000F7F7A0FCF7F7B6FB040018BFF7F71DFE10
:10B33000306841780078F6F7FDFA002C18BFF7F76F
:10B3400017FE002070BD70B50D46044613F0070FC0
:10B3500004D003F00700022805D002E01046F7F7FA
:10B3600024FE002070BDF7F723FE20700120287016
:10B3700070BD7FB51C460E46054613F0070F08D179
:10B3800003F0BCFD28B1012202A9182001F0E0F968
:10B3900003E004F00700022802D004B0002070BDD2
:10B3A00007F025FF002814BF012200222A70012087
:10B3B000307004B070BD7FB51C460E46054613F0D4
:10B3C000070F08D103F09AFD28B1012202A9192024
:10B3D00001F0BEF903E004F00700022802D004B037
:10B3E000002070BD07F0F0FE28700120307004B01E
:10B3F00070BD2DE9F04103F0070C4F4C0E46074697
:10B40000BCF1010F07D04F4D13F0070F07D0BCF16F
:10B41000020F19D015E00020E060206111E0E06823
:10B4200003283CBF29680A54401CE060032808D167
:10B430002868B0F8010040BA01B228680078FDF72A
:10B4400049FE0020BDE8F0812269022A12D242B9E9
:10B4500028680078FDF754FE2A68010A51702968AF
:10B460008870286822691044012A4078387004BF27
:10B47000012030702069401C20610120BDE8F0816E
:10B4800010B503F007002C49012808BF00200CD09C
:10B4900013F0070F2B4B02D0042808D018E0C8681F
:10B4A00004283CBF1B681A54401CC86010E0C868E0
:10B4B00004280DD31868196840788978000440EA98
:10B4C00001201968C978014318680078F8F7D2F8A4
:10B4D000002010BD2DE9F05F03F00705194E164F4F
:10B4E0001C469346894682464FF00008012D4ED1F6
:10B4F00002F01EFF3268017C11703268417C51708D
:10B5000001683268090E917001683268090CD170C7
:10B5100001883268090A11713268017851714168F5
:10B520003268090E917141683268090CD1718188C5
:10B530003268090A117207E094850010DD85001059
:10B54000E3850010A46802003268017951728168B5
:10B550003268090E917281683268090CD1720189D2
:10B560003268090A11733268017A5173C16832680E
:10B57000090E9173C1683268090CD17381893268F0
:10B58000090A11743168007B4874C7F80C8014F004
:10B59000070F4FF0010102D0022D10D00CE03268ED
:10B5A0000420107030684170584602F083FE022279
:10B5B0000720316801F0CCF80020BDE8F09FF86862
:10B5C000122805D23268125C8AF80020401CF8600C
:10B5D000122804BFC7F80C8089F800100120BDE8CC
:10B5E000F09F7FB50D46044613F0070F04D003F01B
:10B5F0000700022808D004E0012202A9122001F06D
:10B60000A7F804B0002070BD02F0F5FF2070012003
:10B61000287004B070BD10B503F00702FE4C012A7B
:10B6200002D0022A07D004E00020E060F9F7BBF85E
:10B63000E061002010BDE268042A07D2C2F10303D2
:10B64000D4F81CC0DB002CFA03F30370501CE0603C
:10B65000042804BF01200870012010BD10B503F0BC
:10B660000700012807D103F049FC20B10022114650
:10B670001E2001F06DF8002010BD2DE9F04103F00F
:10B680000705E54E174688460446012D04BF0020F5
:10B69000F0601BD013F0070F16D103F02FFC98B108
:10B6A000F068DE4B03283CBF19680F54401CF06063
:10B6B00003280BD1186890F9022090F9011090F935
:10B6C0000000FAF78CFC01E0022D02D00020BDE85A
:10B6D000F081F06830B1012809D002280CD003288D
:10B6E0000FD015E01420FAF721FB207010E0152090
:10B6F000FAF71CFB20700BE01620FAF717FB2070FE
:10B7000006E01720FAF712FB2070012088F80000ED
:10B71000F068401CF0600120BDE8F08170B50D4676
:10B72000044603F007000021BB4E012814BF13F0AC
:10B73000070FF16001D0022801D0002070BDF06831
:10B7400040B101280BD002280ED0032811D00428C4
:10B7500014D019E00120FAF7E9FA207014E0022071
:10B76000FAF7E4FA20700FE00320FAF7DFFA20700E
:10B770000AE00420FAF7DAFA207005E00520FAF76B
:10B78000D5FA207001202870F068401CF06001207C
:10B7900070BD70B503F0070C0026A04C9E4DBCF1A7
:10B7A000010F06D013F0070F0CD0BCF1020F1FD011
:10B7B0001CE007F0A6FEEE60216808702168000A10
:10B7C000487013E0E868022803D221680A54401C3C
:10B7D000E86002280AD1EE602068007810F0010FBE
:10B7E00004D002221A20216800F0B2FF002070BDB0
:10B7F000EA68022A28BF104604D223689B5C0370C3
:10B80000501CE860022804D10120EE60087003207B
:10B810002870012070BD7FB51C460E46054613F00A
:10B82000070F08D103F06AFB28B1012202A92520E5
:10B8300000F08EFF03E004F00700022802D004B0FD
:10B84000002070BD10F00BF828700120307004B09B
:10B8500070BD7FB51C460E46054613F0070F08D194
:10B8600003F04CFB28B1012202A9202000F070FF58
:10B8700003E004F00700022802D004B0002070BDED
:10B880000FF0F8FF28700120307004B070BD7FB554
:10B890001C460E46054613F0070F08D103F02EFB99
:10B8A00028B1012202A9242000F052FF03E004F095
:10B8B0000700022802D004B0002070BD13F0BAFACD
:10B8C00028700120307004B070BD7FB51C460E4654
:10B8D000054613F0070F11D103F010FB70B10FF004
:10B8E000D5FF01469DF8080081420BD00FF0CBFF39
:10B8F000012202A91F2000F02BFF03E004F0070043
:10B90000022802D004B0002070BD0FF0BFFF2870E5
:10B910000120307004B070BD2DE9FF413E4E1C4641
:10B920000F46054613F0070F1CD103F0E7FAC8B124
:10B930009DF80800002818BF012802D0022807D06F
:10B9400014E0F070012202A9082000F001FF0DE0D0
:10B95000F07004208DF80800012202A9082000F0F0
:10B96000F7FE03E004F00700022803D004B0002033
:10B97000BDE8F081F07828700120387004B0BDE88F
:10B98000F0817FB51C460D46064613F0070F08D11F
:10B9900003F0B4FA28B1012202A9082000F0D8FE71
:10B9A00003E004F00700022802D004B0002070BDBC
:10B9B000FBF7B6FD801E052813D2DFE800F0030771
:10B9C0000E05100000240DE001240BE0022406F017
:10B9D00060FB042808BF052404E0032402E00424DB
:10B9E00000E0FF2434700120287004B070BD2DE900
:10B9F000F0411C4617460E46054613F0070F0FD1BF
:10BA000003F07CFA60B1384607F02BFB00221146A8
:10BA1000012000F09DFE07E094850010A46802005C
:10BA200004F00700022802D00020BDE8F08107F0F2
:10BA30001BFB287001203070BDE8F08110B5104666
:10BA400013F0070F08BF07F0E5FB002010BD10B58D
:10BA5000104613F0070F08BF07F0E3FB002010BDEE
:10BA600070B5044603F007000D4602281CBF0020F5
:10BA700070BD07F0DEFB20700120287070BD03F060
:10BA8000070230B4FC4B4FF0000C012A05D0022A0B
:10BA900004BF1A78022A0BD01EE002201870F74863
:10BAA000C3F80CC06FF07F410068081AD86113E03A
:10BAB000DA68042A28BF104606D2DD69D40025FAC8
:10BAC00004F40470501CD860042805D10120C3F888
:10BAD0000CC008700320187030BC0120704713F0B0
:10BAE000070F04BFE64802700020704710B503F04E
:10BAF0000700E149012804BF0020C86013D013F0FB
:10BB0000070F10D1C868DF4B04283CBFD3F800C032
:10BB10000CF80020401CC860042804D10422132023
:10BB2000196800F015FE002010BD2DE9F0471646FB
:10BB300003F007020024D04F012A04BFFC603C61DF
:10BB400064D0DFF8448313F0070F07D0022A33D004
:10BB5000042A04BF387806284FD058E0FD68002D2D
:10BB600008BF3E6225D0012D06D0D7F81490AC1E38
:10BB70004C4516D284B908E0701C7861396A0844D3
:10BB8000B0F5007F88BF7C6113E04FF400724FF482
:10BB90007A31BE4802F068FABA49386A0968204426
:10BBA0000E54601C484504D1B848C0F8FC810620FA
:10BBB0003870681CF8602AE0FF2202707B69CBB104
:10BBC000D7F820C03A699444BCF5007F10D2B04D3C
:10BBD0002D68454518BF047005D10CF5783C9CF8DC
:10BBE00000C880F800C0501C984204BF01200870B3
:10BBF000501C38610120BDE8F0874FF47A30F8F727
:10BC000083F8A2494FF47A30F8F720F93C7000200D
:10BC1000BDE8F0872DE9F0478C4603F007010024CA
:10BC2000954F1646012904BFFC603C6162D013F0B9
:10BC3000070F984BDFF8608207D0022932D0042921
:10BC400004BF387806284DD055E0FD68002D08BFA8
:10BC50003E6224D0012D06D0D7F81490AC1E4C457E
:10BC600015D27CB908E0701C7861396A0844B0F5D7
:10BC7000007F88BF7C6112E04FF400721946834850
:10BC800002F0F2F97F49386A096820440E54601CBA
:10BC9000484504D17D48C0F8FC8106203870681CF6
:10BCA000F86028E0FF2101707B69C3B13A6A396905
:10BCB0000A44B2F5007F10D2784D2D68454518BF73
:10BCC000047004D102F5783292F800260270481C04
:10BCD000984204BF01208CF80000481C3861012004
:10BCE000BDE8F0871D461846F8F70EF86749284664
:10BCF000F8F7ACF83C700020BDE8F08770B503F0B1
:10BD000007005D4C1546012804BF0020E06014D0F8
:10BD100013F0070F11D103F0F1F870B1E068594941
:10BD200002283CBF0A681554401CE060022804D178
:10BD300002220968052000F00BFD002070BD2DE9EE
:10BD4000F041054603F007004E4C4B4E0F460128CC
:10BD50000AD013F0070F14D002281BD0042804BF08
:10BD60003078062834D03FE00020F0602168087069
:10BD700021684870216888702168C870052030707B
:10BD800032E0F06804282FD221680A54401CF06089
:10BD9000062028E0F06860B906F0A4F92168087070
:10BDA0002268010A51702268010C000E917021680E
:10BDB000C870F06804283ABF2168095CFF21297027
:10BDC00024BF01213970401CF0600120BDE8F081E2
:10BDD00003F094F840B12068C178006861F31F60F7
:10BDE00006F07BF9032030700020BDE8F0810020D0
:10BDF00070477FB51C460E46054613F0070F08D165
:10BE000003F07CF828B1012202A9282000F0A0FC50
:10BE100003E004F00700022802D004B0002070BD47
:10BE200007F02DFA28700120307004B070BD03F0C7
:10BE300007001149012808BF002009D013F0070F9F
:10BE400007D1C86818B9164B1B681A448A61401C90
:10BE5000C860002070472DE9F04103F00701064C4F
:10BE60001646054601291DD00D4F13F0070F3868FF
:10BE70001CD002292FD02BE094850010AC84001038
:10BE800035840010A4680200554E564D50A900108C
:10BE9000FCE9030000E60300324E564DFCE70300C8
:10BEA000E08600100020E060206111E0A56906F046
:10BEB00005F901280CD1A0693968884224BFF831FE
:10BEC000814205D9E068042838BF2E54401CE06048
:10BED0000020BDE8F081A66906F0F0F850B1A26933
:10BEE00039688A4224BF01F1F800904284BF20697A
:10BEF000305C00D8FF2028702069401C20610120A0
:10BF0000BDE8F0817FB51C460E46054613F0070FCD
:10BF100008D102F0F3FF28B1012202A91C2000F091
:10BF200017FC03E004F00700022802D004B0002050
:10BF300070BD07F08CF828700120307004B070BD1F
:10BF40007FB51C460E46054613F0070F08D102F0D8
:10BF5000D5FF28B1012202A9112000F0F9FB03E06E
:10BF600004F00700022802D004B0002070BD12F0D7
:10BF7000C6FD28700120307004B070BD00207047ED
:10BF80000020704770B50D46044613F0070F04D02B
:10BF900003F00700022805D002E010460AF075FA07
:10BFA000002070BD0AF07DFA20700120287070BD5D
:10BFB00010B503F00702F84CF84B4FF0000C012AC3
:10BFC00002D0022A34D031E0C3F80CC002F096FF50
:10BFD00000282BD0F24801F0B7FF38B3F1480068D1
:10BFE000007E10F0040FEE4810D0C18C2268090AC0
:10BFF0001170226890F826105170818C2268090A0D
:10C000009170216890F82400C8700FE0818C22683C
:10C01000090A1170226890F824105170C18C2268AE
:10C02000090A9170216890F82600C870002010BDA0
:10C03000DA68042A28BF104604D22468A45C04707D
:10C04000501CD860042803D10120C3F80CC008702C
:10C05000012010BD70B503F00701CF4DCF4C012971
:10C0600002D0022914D011E0012001F00FFD0020C0
:10C07000E06001F020FD2081296808702A68010A2B
:10C080000028517004BF002001F000FD002070BDA9
:10C09000E168022902D22A68525C0270481CE06002
:10C0A000012070BD2DE9F04103F007020026BB4DD1
:10C0B0000F460446012A02D0022A09D005E00520D5
:10C0C0002870EE602889400068610020BDE8F0819A
:10C0D0002878052817D1EA686869824205D212F0EB
:10C0E000010F1CBF6878207010D0E868401CE86021
:10C0F0006969884207D10120EE60387003202870FA
:10C10000002001F0C3FC0120BDE8F08101F0ECFC4F
:10C11000010A21706870E8E71FB513F0070F04D11A
:10C12000012202A91B2000F013FB04B0002010BD67
:10C13000002070470020704703F00700974901284E
:10C1400006D013F0070F04BF0878012806D014E0CA
:10C15000012008700020C86088610DE0C8680428CC
:10C1600005D28B69401C42EA03228A61C860042818
:10C1700003D103200870886908620020704703F02B
:10C180000700DFF818C2012807D013F0070F04BF1B
:10C190009CF80000022809D01EE002208CF8000064
:10C1A0000020CCF80C00CCF81C0015E0DCF80C00EA
:10C1B000022808D2DCF81C10401C42EA0121CCF80D
:10C1C0001C10CCF80C00022806D1DCF81C00CCF8BE
:10C1D000240003208CF800000020704770B403F0A6
:10C1E000070200256D4C012A02D0022A06D002E087
:10C1F00002202070E56070BC002070472278022A7F
:10C200001CD1D4F824C0E268624528BF10460ED283
:10C2100012F0030F04D1236A53F8046BC4E90763D7
:10C22000237F0370E069000AE061501CE060604514
:10C2300004D10120E56008700320207070BC01204B
:10C24000704770B503F007000025544C0E460128D6
:10C2500006D013F0070F04BF2078022805D02BE08A
:10C2600002202070E560E56126E0616AE0688842AE
:10C2700019D2E169090A41EA0262401CE26110F048
:10C28000030FE0600FD1206AB0F5802F28BF026055
:10C2900006D2B0F5005F03D304224349F7F72AFE24
:10C2A000206A001D2062616AE068884204D1012092
:10C2B000E560307003202070002070BD70B503F081
:10C2C000070C0025354CBCF1010F08BFE5603AD0E2
:10C2D00013F0070F03D0BCF1020F36D033E0052A6C
:10C2E00008BF4FF47A302DD005DC16D2DFE802F01B
:10C2F000171A1D2022002B48202A006808BFF8309A
:10C3000020D006DC102A1DD0112A08BF244819D0DD
:10C3100003E0302A11D0312A12D0A56113E04FF486
:10C3200000500FE04FF47F300CE04FF4483009E04C
:10C330001E4807E04FF47C3004E001F031FD01E0DD
:10C3400011F031FFA061002070BDE268042A07D21D
:10C35000C2F10303D4F818C0DB002CFA03F3037016
:10C36000501CE060042824BF01200870012070BD2B
:10C3700070B403F0070C094DBCF1010F07D0064C57
:10C3800013F0070F14D0BCF1020F2ED02AE00020CA
:10C39000E860286126E00000A4680200948500108F
:10C3A000442E0110BC860010B085001000EE030082
:10C3B000E86805283CBF21680A54042810D1236886
:10C3C0002268D4F800C0D3F80130A96912781BBAEA
:10C3D0009CF804C023F0FF0343EA0C0341F8223029
:10C3E000401CE86070BC002070472B6973B1042BBF
:10C3F00007D22268032B1A445278027004BF01202E
:10C400000870581C286170BC012070472268D5F85C
:10C4100018C012785CF8222026684FEA126C86F861
:10C4200001C026684FEA124C86F802C026684FEA1F
:10C43000122C86F803C0D4F800C08CF80420D8E78A
:10C4400010B503F00700012804D1002211460E2088
:10C4500000F07EF9002010BD2DE9F04103F0070443
:10C46000A94E174688460546012C04BF0020F060FF
:10C4700017D013F0070F12D102F040FD78B1F06829
:10C48000A24902283CBF0A681754401CF0600228E9
:10C4900007D102220968072000F05AF901E0022CB6
:10C4A00002D00020BDE8F081F26812B1012A04D068
:10C4B00009E0FBF735F8287005E0FBF737F828703E
:10C4C000012088F80000F068401CF0600120BDE801
:10C4D000F08170B503F0070000258B4C012808D0CF
:10C4E00013F0070F0BD0042804BF2078062825D0AE
:10C4F0002DE0A561E5616570E560257027E0E068E5
:10C50000022807D2A16942EA0121A16161781144A0
:10C51000617010E0042807D2E16942EA0121E1617B
:10C5200061781144617006E0052804D261788A427E
:10C5300004BF06212170401CE06008E0D4E9060138
:10C5400001F082FE002804BF0120A07025700020A9
:10C5500070BD10B56C4C13F0070F07D003F0070047
:10C56000042804BF2078062822D02BE0E0680228A7
:10C5700007D2A16942EA0121A16161781144617089
:10C5800013E06349091808D260490968014401F8B9
:10C59000022C61781144617007E05E49091804D2E9
:10C5A00061788A4204BF06212170401CE06009E0E6
:10C5B0005949A06901F06AFE002804BF0120A0705B
:10C5C00000202070002010BD03F0070CBCF1010F0B
:10C5D00000D0BEE74C49002088614870C8600870F0
:10C5E000704730B403F007050024DFF81CC1012DAB
:10C5F00007D013F0070F0DD0022D3CD0042D54D0DE
:10C600006FE0CCF81840CCF81C40CCF80C408CF80B
:10C61000004066E0DCF80C0002280BD2DCF81810B1
:10C6200042EA0121CCF818109CF8011011448CF852
:10C63000011019E0042817D2DCF81C10032842EA84
:10C640000121CCF81C109CF801301A448CF8012010
:10C650000AD106228CF80020DCF81820114304BF10
:10C660004FF40071CCF81C102C49401CCCF82C1055
:10C67000CCF80C0035E0DCF80C20042A28BF10466A
:10C680000AD2C2F10303DCF82C50DB0025FA03F3D5
:10C690000370501CCCF80C00042803D10120CCF806
:10C6A0000C40087030BC012070479CF80000062840
:10C6B00015D1DCF8180000224102DCF81C0043020E
:10C6C0001046B2EB930F06D251F8045B401C2A448B
:10C6D000B0EB930FF8D3CCF82C208CF80040CCF8BA
:10C6E0000C4030BC002070474FF47F300168880A4E
:10C6F000424211EB822218BF401C404201EB8000F5
:10C70000C01C20F00300704794850010A46802004C
:10C71000FEFDFFFFFDFDFFFF50A90010EFBEADDEE7
:10C72000F948002202704270827002714271C27038
:10C73000DFF8D8C3114601EB410300200CEB4303A3
:10C740001A54401C0628FBD3491C2029F3D37047F8
:10C7500001F0FDBC2DE9F04115460E460746F7F7FE
:10C7600037FF00F008040820F7F72DFF2A4631466E
:10C77000384601F0ECFC05462046F7F71FFF284637
:10C78000BDE8F081E04880787047DF484078704726
:10C79000DD49002048707047DB49CA681043C86013
:10C7A000704710B518B3FAF7BBFE0446F8F746FB1E
:10C7B0000220F8F7E3FB052C11D07820F4F713FCE6
:10C7C0003C20F6F70DFC0520F8F725FBD048F8F7DC
:10C7D00057FCF8F73AFCBDE81040F8F7BDBB3C2029
:10C7E000F4F701FC1E20F6F7FBFB0320ECE7F8F75B
:10C7F000BCFBF8F737FC0020F8F742FCBDE810401E
:10C80000F8F7FEBAC04AD179814218BFD07170479B
:10C8100010B5FAF779FF01280EBF0020BA48C07999
:10C8200010BD10B5F4F7C8FB10F0010F08BF10BD24
:10C83000FAF776FE052818BF10BDF4F7E0FB3C2898
:10C8400004D0BDE810400220F8F798BBFAF76EFE5E
:10C85000022804D0BDE810400020F8F78FBBBDE8E7
:10C8600010400120F8F78ABB10B50024F4F7A4FBB0
:10C8700010F0010F2ED0FAF753FE02282AD1F6F756
:10C88000ACFB38B3F6F7AFFB3C2802D01E2811D022
:10C890001CE0002360229421072005F0FDFA01200E
:10C8A000F9F74BF8FAF742FE02281CBF022006F007
:10C8B000A3FC0BE0002330229421072005F0ECFAC2
:10C8C000914A0121D079012818BFD1710020F6F7D3
:10C8D00081FB0124204610BD8B4910B508208871CA
:10C8E000FAF71EFE022818BF012811D0032818BF2E
:10C8F00005280DD00020F6F7B6FAF8F736FBF8F762
:10C90000B1FB0020F8F7BCFBBDE81040F8F778BA9F
:10C91000AFF27110BDE81040F6F7A5BA2DE9F04767
:10C920004FF00008F6F7A7FADFF8DCA10446DAF8C2
:10C930000C00C14640B1DAF80C0010F0400F18BFEF
:10C9400044F00404CAF80C9014F00F066CD00127D0
:10C95000FAF7E6FD05463046F6F790FA012E1DD0AF
:10C96000FAF7E4FD44EA006400232246032107208D
:10C9700005F092FA14F0050F14BF00200120F3F720
:10C98000FCFC14F0060F4FD04FF00108FAF7CEFD73
:10C990000646022D2CD0052D0AD03DE09AF806005F
:10C9A000854208BF00278AF80650002FD8D1E8E753
:10C9B00014F0020F13D0F3F761FFF8B1F3F76DFF36
:10C9C000040AF3F76AFFC0B244EA002200236C2194
:10C9D000022005F061FA0020F3F74AFF0EE04D4C0B
:10C9E000206858B10120F8F7A8FFC4F8009005E0CE
:10C9F00014F0020F1CBF0120F8F79FFF01F0DCFDCF
:10CA0000002818BF01F0DFFD022E05D0022D4FF0E7
:10CA100002000CD001F0ACFD02F060FB00281CBF4E
:10CA20004FF0805002F05DFB4046BDE8F08706F015
:10CA3000E3FBF1E72DE9F84F0026F8F784FBFAF75E
:10CA40006FFD022804D102F015FA002818BF012654
:10CA5000FFF764FF002818BF0126FFF705FF002835
:10CA600018BF0126DFF8A09099F80200002800F016
:10CA70009982D9F808006D464FF0FF34002740B185
:10CA8000D9F8082000230121084605F005FAC9F865
:10CA90000870F7F79DFD00F0080A0820F7F793FDEE
:10CAA00099F80300DFF864B000B399F8050000EBD3
:10CAB0004001401CC0B20BEB410189F80500202861
:10CAC00028BF89F8057099F80300401E89F8030013
:10CAD0004C7891F800800020002C05DD0A1892782F
:10CAE0002A54401C8442F9DC0F704F705046F7F70F
:10CAF00065FD002CC0F2468208F0FF0000242928C2
:10CB000080F0FD8108E00000CC85001050AB0010E3
:10CB100049E700003C860010DFE800F0CE3B15221C
:10CB20002D3E194BFD50CE8C92DAFC97A1B3CFFB72
:10CB3000FAF9F8CEF7F6F5F4ADF3F2CEF1F0EFCE68
:10CB4000EEEDCEECA7000020F8F7F7FE21E09DF80F
:10CB50000000AC280CBF01200220FAF7ADFD18E060
:10CB60009DF800100120FAF7F6FC012089F8010079
:10CB7000044600F0C4B99DF80310009861F31F60EB
:10CB800002F0A9FA01210320FAF7E5FC012089F857
:10CB90000100012400F0B3B9BDF8000040BA05F06F
:10CBA000A4FA02210320FAF7D6FC012089F801003B
:10CBB000EFE79DF801109DF80000EDE04FF0010A4D
:10CBC00089F801A099F8000080BBF6F744F968B332
:10CBD0009DF8005089F800A0FAF7A2FC012808BFD0
:10CBE000002515F0040F18BFFCF7EFFA15F0020F3F
:10CBF00006D01F20FBF71CFCF8F77FFF45F001056E
:10CC000015F0010F10D0FAF78BFC022802D106F0C4
:10CC10003FFA48B1FAF784FC052802D101F0B7FCCD
:10CC200010B10020F8F756FF89F8007089F80170FC
:10CC300000F065B99DF80000401E01F04FFFA8E725
:10CC40009DF8000006F0FBFAA3E79DF8000010F045
:10CC50000F0018BF01200EF095F800F050B99DF8B4
:10CC600000000EF085F800F04AB99DF8000006F0CB
:10CC7000FAFA00F044B99DF8000006F0DFF900F080
:10CC80003EB99DF8000018B101280CD000F037B96A
:10CC9000002011F031FF022011F037FA032011F0CB
:10CCA00053FA00F02CB9012011F026FF022011F0F8
:10CCB0001DFA032011F039FA21E19DF8000001F07E
:10CCC00097FC9DF8000000284FF00100E7D0F1E745
:10CCD0009DF80000002808BF00215CD0FAF720FC76
:10CCE000052841D0022818BF012406F08DFA01461C
:10CCF000022011E0FFE0F7E0F1E0A3E09DE0B8E002
:10CD00007CE0A4E024E01EE018E008E08BE084E092
:10CD100077E068E02EE042E0FAF71DFCEFE09DF8D6
:10CD20000000002818BF012006F057FA9DF8000007
:10CD3000002818BF012001F011FCE0E09DF8000080
:10CD400006F037FADBE0BDF8000006F040FB20E714
:10CD50009DF8000020B1012806D0022805D0CEE0C1
:10CD60004FF47F30F6F7D0FFC9E002F01FF9002141
:10CD7000042011E0F7F72CFC00F008040820F7F776
:10CD800022FC99F80300002808BF89F802702046A9
:10CD9000F7F714FC01210620FAF7DDFBF9E69DF810
:10CDA0000000062804D2DFE800F003061315181B64
:10CDB0000221084601E002210520FAF7CCFB02F02F
:10CDC0008DF900281CBF4FF0005002F08AF9E0E610
:10CDD000002106E000210420EFE700210620ECE717
:10CDE00004210320E9E79DF80300009A002360F383
:10CDF0001F626221072005F04FF880E0F9F783F900
:10CE0000C7E600989DF8031000BA20F0FF00084321
:10CE10000CF085FB0CF0C0FB71E0BDF8000040BADF
:10CE20000CF06CFB6BE000989DF8031000BA20F04A
:10CE3000FF0008430CF04BFB61E09DF8000006F09A
:10CE400086FBA6E69DF8000006F089FBA1E69DF8AA
:10CE5000000000F00100FAF795FC9DF800000028A2
:10CE60004FF0000002D011F060F992E611F06CF979
:10CE70008FE60EF0FFFC9DF8004006F042FB0546F1
:10CE800006F03BFA012808D1042C06D00EF032FC43
:10CE900018B1FAF745FB02281AD0012C08BF284622
:10CEA0001AD0022C08BF45F0805015D0042C18BFB2
:10CEB000082C7FF46EAE45F0005006F02DFA042CDD
:10CEC00018BF082C7FF465AE20460EF0CEFC60E65D
:10CED000204606F0D7F95CE606F01EFAF4E79DF866
:10CEE000000011F0AAFF0AE09DF800000EF0B4FC6B
:10CEF00006F007F903E09DF8000000F075F90CB1A9
:10CF000001263FE0D9F808006D464FF0FF3440B1EC
:10CF1000D9F8082000230121084604F0BDFFC9F814
:10CF20000870F7F755FB00F0080A0820F7F74BFBED
:10CF300099F8030000B399F8050000EB4001401C8C
:10CF4000C0B20BEB410189F80500202828BF89F801
:10CF5000057099F80300401E89F803004C7891F899
:10CF600000800020002C05DD0A1892782A54401C0D
:10CF70008442F9DC0F704F705046F7F71FFB002C0E
:10CF8000BFF6BAADF7F724FB00F008040820F7F766
:10CF90001AFB99F80310002908BF89F8027020468F
:10CFA000F7F70CFB002E04BF0020BDE8F88F02F05D
:10CFB00095F800281CBF4FF0804002F092F8012045
:10CFC000BDE8F88F02460020022928BF704752B101
:10CFD000012A18BF704701EB4100C0EB4110FD4929
:10CFE00001EB8000704740F2DB104843FA49F7E755
:10CFF00070B5F7F7EDFA00F008060820F7F7E3FA46
:10D00000F64C00256078FF2806D240F6D861F24839
:10D0100001F02FF8E5702571E079FF2805D2E821AD
:10D02000EC4801F026F8257265723046BDE8704084
:10D03000F7F7C4BADFF8A8C300FB01F31CEB030C3D
:10D0400088BF7047E54B1A62C3E906017047DFF8F5
:10D050008CC30028DCF8183018BF0360DF480029B3
:10D06000C06918BF0860002A1CBFDCF820101160DE
:10D0700058437047D94801214171007840F2DB11D3
:10D0800080F001004843D44901EB80007047D34849
:10D09000C278002132B1027922B9027882F001020D
:10D0A0000270C17041717047CC491E284A7848709F
:10D0B00008BF002003D01F2808BF012000D108703E
:10D0C00010467047C548007840F2DB1180F001003F
:10D0D0004843C14901EB800070472DE9F007BF4F7D
:10D0E00097F800C040F2DB140CFB04FCBA4CBE699C
:10D0F00004EB8C0C03FB06F40CEB440C8E4234BFA7
:10D1000035460D46FC69E31A934238BF1A46BB7890
:10D11000012B16BF052B6C0800244FF00008002AD5
:10D120009CBFBDE8F00770472346AC420FD297F88A
:10D130000290B9F1050F30F8139006BFA3EB040A73
:10D140002CF81A902CF813905B1CAB42EFD308F12B
:10D1500001080CEB460C00EB41009045E4D3BDE820
:10D16000F00770472DE9F0419C4F14468C4601466C
:10D170007A7806981D468A4218BFBDE8F0810121E1
:10D180003971012802D0022824D029E0387840F2F1
:10D19000DB1148439049BE6901EB8001A64234BFD0
:10D1A00032462246F869A84238BF05460023002DC2
:10D1B00016D90020002A06D91CF8007021F810703A
:10D1C000401C8242F8D85B1C01EB4601A444AB42F0
:10D1D000EFD305E000232A4621466046FFF77DFF96
:10D1E000BDE8F04100F0CDBC7C4A01281146D07268
:10D1F000497808BF242004D0002806BF2429FF2036
:10D200007047507070477548C07A704770B4DFF847
:10D21000D4C1DCF800C0DCF818C01CF0040F1ABF41
:10D22000012424EA0C060CF0010605680C68002EA7
:10D230001CBF1B1B5C1E1CF0020F1CBF521B551E8B
:10D240001CF0040F19BF04600D6005600C6070BC19
:10D250007047002808BF70476049634B4A786349AC
:10D260001B78002A097818BF022A05D0042A18BFA3
:10D27000092A01D0012230E75D4A1278012A84BFD1
:10D280005C4A1378012200F096BC2DE9F04FDFF8DC
:10D290004C9193B0012189F804105749544C554ED4
:10D2A0000D785149DFF830B10F7899F80110112944
:10D2B00033D00CDC042920D004DC002918BF02295B
:10D2C00011D11AE0092918D0102926D00BE0212904
:10D2D0007ED004DC122918BF132904D11DE02229B5
:10D2E00076D0242975D0002800F0538100233A46D7
:10D2F0002946FFF7F2FE00F04CB92178012902D946
:10D300003E4937780D78002800F0438100233A46E3
:10D31000294600F050FC00F03CB9F5F7A3FCF5F706
:10D32000B9FB0090002818BFF5F71FFE20780128F0
:10D3300088BF3778F5F79CFD10F0020F18BF7F1CEF
:10D34000DFF8BC8099F8016099F8000040F2DB1129
:10D350004143D9F818000BEB8104A84238BF0546B9
:10D36000D9F81C00B84238BF0746F5F7C4FE019053
:10D370000020F6F705FA4FF0000A002F4EDD4FF0BF
:10D380000009002DC4BF0AEB4A0000EB0A1B3DDD7B
:10D39000019810F90900262824BF002024F819005C
:10D3A00015D200F0010108EB813100EBD07001EBE8
:10D3B0008B014010102E51F8200035D0112E3AD09C
:10D3C000122E0CBFC0B2F6F7E1F924F8190019E0EB
:10D3D00037E03EE0E8BA001010AC0010DC85001029
:10D3E0004AFCFFFFBC860010598500105F850010C5
:10D3F0005A8500105C850010588500105B85001070
:10D400000000013009F10109A945C1DBF7480AF123
:10D41000010ABA45806904EB4004B0DB009800289B
:10D4200018BFF5F7A5FDB4E010F4003FC0F342309B
:10D43000CBD04042C9E710F4803FC0F30420F8D1BC
:10D44000C3E700287DD00023BA1C2946FFF745FE1C
:10D450009FE0002875D00646E5480068007E10F081
:10D46000040F07BF2C46BA463C46AA460323009346
:10D470004FEA5A0261080993201F0A930B930C92FA
:10D48000CDE901100D920E92CDE90331AAF104020B
:10D490000F921092CDE905031192CDE90710534682
:10D4A000224609A96846FFF7B1FE5346224609AF56
:10D4B0000AA9E84601A8FFF7A9FE5346224607F14C
:10D4C000080108F10800FFF7A1FE5346224607F1C4
:10D4D0000C0108F10C00FFF799FE5346224607F1B4
:10D4E000100108F11000FFF791FE5346224607F1A4
:10D4F000140108F11400FFF789FE5346224607F194
:10D50000180108F11800FFF781FE5346224607F183
:10D510001C0108F11C00FFF779FE5346224607F173
:10D52000200108F12000FFF771FE99F8000040F299
:10D53000DB11414300220BEB8100914620F8129051
:10D5400000E026E058F82210A1F1010C491C6145C9
:10D550001CD357F822104B1E491C99420FD303FBD2
:10D5600005C136F9114030F912108C42C8BF20F8BD
:10D57000124057F822105B1C491C9942EFD258F810
:10D5800022100CF1010C491C6145E2D2521C092AFF
:10D59000D4D313B0BDE8F04F00F0F3BA93480121A3
:10D5A0008172807980F0010000EB4001C1EB4010F6
:10D5B000904901EB800070478C48027A002132B11B
:10D5C000427A22B9827982F00102827101728172FB
:10D5D000704786491E28CA79C87108BF002003D049
:10D5E0001F2808BF012000D18871104670477F486E
:10D5F000807980F0010000EB4001C1EB40107D49D3
:10D6000001EB800070472DE9F04F7B49DFF8DC81AA
:10D6100085B00F7879490E78012188F8091098F8BB
:10D620000710744C4FF00009102918BF11293AD087
:10D63000122918BF132936D0F0B198F8061001EB63
:10D640004102C2EB411104EB8102002116EB070CF1
:10D6500018BF674C10D02368002E5B8A03BF30F8D8
:10D6600011500B4422F8135030F8113018BF22F833
:10D670001130491C8C45EED8F6F7AAFF00F00804DB
:10D680000820F6F7A0FF98F80A0000281CBF012127
:10D6900088F808107CD02046F6F790FF88F80990AB
:10D6A00005B0BDE8F08FF5F7DDFAF5F7F3F9029074
:10D6B000002818BFF5F759FC98F80750D8F824004F
:10D6C000009098F8060000EB4001C1EB401004EB1D
:10D6D000800BF4F76BFA00286AD01120F3F713FAE5
:10D6E00000280CBF1220112060F3070A0120F3F775
:10D6F0000AFA002814BF0120022060F30F2A0AF062
:10D70000FF000190F6F73CF8F5F7F3FC00240390D6
:10D71000002E1FD903980257142AA8BF143A02DA20
:10D720000A2AA8BF1232262A28BF2BF814900ED23C
:10D73000DDE90010F5F733F8102D4AD0112D4FD048
:10D74000122D0CBFC0B2F6F721F82BF81400641CA0
:10D75000B442DFD30BEB4606CAF3072B5846F6F765
:10D760000FF8F5F7C8FC00248246002F1AD91AF9E1
:10D770000420262A28BF26F8149010D25846009973
:10D78000F5F70DF8102D3BD0112D40D0122D00E0F3
:10D7900043E00CBFC0B2F5F7F9FF26F81400641C93
:10D7A000BC42E4D30298002818BFF5F7E1FB63E719
:10D7B0000120F3F7A8F9002814BF0120022060F32C
:10D7C000070A1120F3F79FF9002814BF1120122037
:10D7D00093E710F4003FC0F34230B6D04042B4E7C4
:10D7E00010F4803FC0F30420F8D1AEE7DC850010D0
:10D7F000BC860010E8BA00105D8500105E85001040
:10D8000010F4003FC0F34230C7D04042C5E710F4E7
:10D81000803FC0F30420F8D1BFE798F8060080F0FD
:10D82000010088F8060088F8089034E7FE48704741
:10D83000FE490A7840F2DB135A43FD4B896903EB3A
:10D840008202484303F5406102EB4000D1F8C03347
:10D85000D1F8C423D1F8C8130360426081607047D7
:10D860002DE9F041F14E0D4601213171F1490F785A
:10D87000F1490C78717821291EBF22292329BDE89E
:10D88000F081002818BF002D25D0002322463946FC
:10D89000FFF723FC631C012221462846FFF71DFCED
:10D8A00005EB4400A31C01223946FFF716FC317832
:10D8B000E01C40F2DB125143DD4A02EB8101B26908
:10D8C000504301EB4000DD49D1E9F023D1F8C81302
:10D8D000026043608160BDE8F04100F052B970B56C
:10D8E0000446C068D14D68B1697859B9D4490978FE
:10D8F00001298CBFD349D0490B78D349012209783B
:10D9000000F059F9A06820B16978002908BFFFF735
:10D91000BCFC6878102804BF0020FFF7B6FC6878CC
:10D92000112804BF0020FFF7B0FC6878122804BF5C
:10D930000020FFF7AAFC6878132804BF0020FFF737
:10D94000A4FC206920B1E979002908BFFFF75BFE3C
:10D95000E879102804BF0020FFF755FEE879112868
:10D9600004BF0020FFF74FFEE879122804BF002013
:10D97000FFF749FEE879132818BF70BD0020BDE805
:10D98000704040E62DE9F74F8046AA480D46002634
:10D9900090F800A0A848A549344690F80090BAFB3A
:10D9A000F5F000FB09F701200871487B0978DFF8E2
:10D9B00080B288420ED09D4A40F2DB1148430BEB07
:10D9C0008001107840F2DB1250430BEB8000920094
:10D9D00000F059FB0298002888BFDFF850B22DD91B
:10D9E0009BF80EC00022BCFBF9F009FB10C101FB43
:10D9F0000AF100FB0510002D12D938F814309BF8FD
:10DA0000001040F2DB1E01FB0EFE8949641C01EB95
:10DA10008E0100EB020E521C21F81E309542ECD80C
:10DA20000CF10100C0B28BF80E00B84224BF0020F8
:10DA30008BF80E00761C02988642D1D37B49887BF6
:10DA4000401EC0B2887387429CBF781E88730878D6
:10DA5000487303B0BDE8F04F00F093B87348017805
:10DA600000F1280281F0010132F81110002918BFDD
:10DA70007047017881F00101017000210182037873
:10DA800022F81310714A00781154704767490873DF
:10DA900070476648007B704770B5644C0025257060
:10DAA00025732582658240F6D861614800F0E1FA6D
:10DAB000A562A58270BD5D49087800224A8280F087
:10DAC00001001431095C69B140F2DB11584A41434D
:10DAD00032F82110A1F55062B63A02BF5C4931F824
:10DAE0001000704700207047504B187803F1140C59
:10DAF00080F001014FF6FF701CF80120012A18BFC9
:10DB0000704740F2DB104843494A02EB80005A8AD2
:10DB100030F81200521C5A824D4B33F81120521E1D
:10DB20001204120C23F8112004BF00220CF801206B
:10DB300070474749A1F12802137801EB43010B8894
:10DB400003440B8092F800C0012102F1140303F892
:10DB50000C10118A084410827047344A138A03EB70
:10DB600050003C4B01445B1824BF002070471178E3
:10DB700040F2DB1251432E4A02EB810101EB4000DF
:10DB8000704770B5F6F724FD00F008060820F6F798
:10DB90001AFD264C60790025002801BF207880F00E
:10DBA00001002070E5701CBF0120E0703046F6F7E0
:10DBB00005FD257170BD2DE9F047994616460D46C5
:10DBC0000446F5F79DFA5FEA000C1CD01749087867
:10DBD00040F2DB125043164AD1F8188002EB800065
:10DBE00009FB08F200EB4200454594BF2F4647462B
:10DBF000C969A1EB0901B14238BF0E460021002ED0
:10DC000009D8BDE8F0874B46324629462046BDE894
:10DC1000F047FFF762BA0023002F22D91CF9032036
:10DC200034F8122018E00000D0BB0010DC85001092
:10DC300010AC0010588500105985001010B8001065
:10DC40005A8500105C8500105F850010F08500107B
:10DC5000048600104AFCFFFF20F813205B1C9F4243
:10DC6000DCD8491C00EB480004EB4504B142D2D398
:10DC7000BDE8F0874149002814BF0020012008704A
:10DC800070473E48007800280CBF012000207047F4
:10DC900001203A49487070473848002141700178A6
:10DCA00000291ABF4068002870473548016821F0F4
:10DCB0000101016070473148017821B130490A689B
:10DCC00042F001020A60002141608160C16001618F
:10DCD00070472A48017821B129490A6842F00102B7
:10DCE0000A60002141608160C1600161704700B538
:10DCF0000178427885B0890141EA82018DF80010EF
:10DD0000418809098DF80110818809098DF80210F0
:10DD1000817801F00F02017962F31F118DF8031071
:10DD2000017A8DF80410417A8DF805108179C27955
:10DD300001F03F0102F00C0241EA02118DF80610D9
:10DD4000C179827A890102F0010241EA42118DF81B
:10DD50000710C17B8DF80810017C8DF80910407CFC
:10DD600000F00F008DF80A0000208DF80B000390E2
:10DD7000684600F0F1F905B000BD0000088600100B
:10DD8000144C0040002818BF474848498863704732
:10DD90004648806B444988420CBF012000207047F0
:10DDA00042487047424B4FF0000C1C681B1F1D6817
:10DDB0003E4B19605A603F49D963DC6214F0804FD2
:10DDC00022D0290C5985290A83F8291083F8285074
:10DDD000598D19B1598D012242EA014C93F829104D
:10DDE00039B193F82910022242EA014C32490C68F9
:10DDF0001C6393F8281039B193F82810032242EAE3
:10DE0000014C2E490C685C632D490C60091DC1F85A
:10DE100000C02C4A81691160B0E816109960DA6080
:10DE20001C61C3F814C090E807109861D9611A62A8
:10DE3000C3F824C0986B1C49884202D12349224868
:10DE40000860FEE72249012804BF096070470228E4
:10DE500018BF704708471548D0F8EC201C498A4283
:10DE600004BFD0F8F0208A4208D1D0F8F4208A42CA
:10DE700001BFD0F8F8208A4201207047C0F8EC10AA
:10DE8000C0F8F010C0F8F410C0F8F8100020704787
:10DE900006480F49C0F8EC10C0F8F010C0F8F410B4
:10DEA000C0F8F81070470000504D5544005F011055
:10DEB0002CED00E0544C414638ED00E034ED00E03C
:10DEC000344C00403C4C0040AD2007B0304C00408A
:10DED000ADDEADDE7047002808BF704780220146E6
:10DEE000014800F0C1B87047F0C3001010B501F050
:10DEF00012F8B0B101F005F801464FF4C4721748AA
:10DF000000F0B2F801F002F8154C01464FF4E87247
:10DF1000206800F0A9F82068C06BBDE8104005F04B
:10DF200006B90220F9F7C8FBE1E758B10D4A0168CC
:10DF3000914207D1406820F00F00B0F5407F04BF48
:10DF4000012070470020704730B1006820F00F00BA
:10DF5000802804BF0120704700207047442E011024
:10DF6000BC8600104150535230B4029C40B101288D
:10DF70000AD002280FD1C8B230BC114611F0BCBC87
:10DF800030BCC8B211F0EDBBC8B2D1B21A46A3B2D0
:10DF900030BC11F01DBC30BC704708A0704710B5F4
:10DFA000F2F7DBFC4169BDE8104004A008473E20C1
:10DFB00070470320704700F005B800004D3531353B
:10DFC00000000000024870474FF480607047000076
:10DFD0000080001030B41446012806D0022809D170
:10DFE00030BC1946104612F04CBB204630BC1A46D5
:10DFF00012F0F4BA30BC704700487047DC7202007F
:10E0000010B5431C02E010F8011B71B18107FAD171
:10E010004FF0013202C88C1A8C4314EAC211F9D0B5
:10E02000C01A0A0603D0C01E10BDC01A10BD0A04D3
:10E0300001D0801E10BD0902FCD0401E10BD01B5EC
:10E0400000F021F801BD70470021016001717047A7
:10E050000B54584541F6734CC1F2000C604743F233
:10E06000015CC1F2000C604742F28D7CC1F2000CF1
:10E07000604742F6450CC1F2000C604743F2C30C06
:10E08000C1F2000C604742F2037CC1F2000C604711
:10E0900042F2BB6CC1F2000C604745F21B6CC1F24E
:10E0A000000C604743F6413CC1F2000C604742F26D
:10E0B000F17CC1F2000C604740F2D32CC1F2000C9D
:10E0C000604740F2C11CC1F2000C604740F2ED2CE9
:10E0D000C1F2000C604741F6996CC1F2000C604738
:10E0E00040F6C93CC1F2000C604743F2F12CC1F28A
:10E0F000000C604744F2FD6CC1F2000C604743F233
:10E10000711CC1F2000C604743F2E91CC1F2000C23
:10E11000604740F2130CC1F2000C604740F22B1C28
:10E12000C1F2000C604740F2B31CC1F2000C604722
:10E1300043F2275CC1F2000C604743F21B6CC1F252
:10E14000000C604740F2010CC1F2000C604743F242
:10E15000993CC1F2000C604743F2214CC1F2000C23
:10E16000604742F2B92CC1F2000C604742F2A92C80
:10E17000C1F2000C604742F2E52CC1F2000C60478E
:10E1800043F6AF0CC1F2000C604741F67B4CC1F284
:10E19000000C604744F2673CC1F2000C604740F25B
:10E1A000931CC1F2000C604742F6010CC1F2000C56
:10E1B000604740F2C95CC1F2000C604745F27D5CEB
:10E1C000C1F2000C604740F6D75CC1F2000C60471A
:10E1D00045F6AD4CC1F2000C604741F6A16CC1F2AE
:10E1E000000C604742F2B12CC1F2000C604745F2CE
:10E1F000D15CC1F2000C604743F61F6CC1F2000C09
:10E20000604740F2B91CC1F2000C604740F2332C69
:10E21000C1F2000C604745F66D5CC1F2000C60472E
:10E2200045F6B50CC1F2000C604742F6050CC1F290
:10E23000000C604740F2070CC1F2000C604740F24E
:10E240000F0CC1F2000C604770B50E460446F9F79A
:10E2500067F9042811D1A4F5C07080280DD2A01947
:10E26000A0F28110802808D265020024002E04D973
:10E270002846F5F749FD012801D0002070BD641C37
:10E2800005F50075B442F3D3012070BD70B50D469D
:10E290000446F9F745F904280AD1A4F5C07080288E
:10E2A00006D260022946F5F7D1FD012808BF70BDEE
:10E2B000002070BD9C49087070479B4800787047EB
:10E2C0009A4B10B49A494FF0010C83F810C00A68B9
:10E2D000091D1A600968596096490968964C091920
:10E2E00012D0B1F5803F14D0A1F18051B1F57E017B
:10E2F00004BF83F811C04FF0805011D0A1F1CE714E
:10E30000B1F1C05F09D00BE0042058744FF04050C9
:10E3100006E008205874894802E0022058748848B2
:10E32000101A0CEB90009860C043D86010BC704786
:10E330007E4870472DE9F04F82488DB004ACB0E8BC
:10E340000E108DE80E10B0E80E1084E80E100FC805
:10E3500008AC84E80F0072B67B48016841F0010107
:10E360000160734E00253560371D3D6007F10408DC
:10E37000C8F80050DFF8B0912C464FF0402A6846AC
:10E3800000EB041C0121DCF8000099F8002081401A
:10E3900011424FD0022818BF032811D1DAF810001B
:10E3A00040F00400CAF81000DAF8100040F0010054
:10E3B000CAF81000DAF8100040F00300CAF81000A4
:10E3C000DCE9011082084FF001034FF0000005D096
:10E3D00041F82030401C5B1C8242F9D80123002008
:10E3E000002A0BD951F820B09B4511D16FEA030BDD
:10E3F00041F820B0401C5B1C9042F3D30123002065
:10E40000002A0CD951F820E06FEA030BDE4502D058
:10E4100001EB800004E0401C5B1C9042F2D32846D4
:10E4200040B1306000683860DCF80C00C8F80000CB
:10E43000F9F73AF9641C032CA1D399F8000010F005
:10E44000020F4FD06A460023A2F18050B0F5C030D1
:10E450000DD03E48C2F5C0333D4903F18053904290
:10E4600005D950F804C941F804C99042F9D8C3F558
:10E47000004000F1805080F30888314901234FF4B7
:10E480008042002041F82030401C5B1C8242F9D8B9
:10E4900001230020002A0BD951F820C09C4511D13E
:10E4A0006FEA030C41F820C0401C5B1C9042F3D380
:10E4B00001230020002A0CD951F820406FEA030CF8
:10E4C000644502D001EB800503E0401C5B1C9042D8
:10E4D000F2D33DB13560286838601E48C8F80000A6
:10E4E000F9F7E2F8F9F7E0F80DB0BDE8F08F0E4962
:10E4F000487070470C484078704770B500250A4C4A
:10E50000154EFEF797FA012808BF70BD6078012804
:10E5100004BF6570FFF70EFF3068FFF706FD0028A7
:10E5200018BFF9F763F8ECE71C860010DCC3001095
:10E53000344C00403C4C00405DA71F5000000430AC
:10E5400000800010A8680200144C0040FC7F0110FD
:10E55000FC7F0010A3587ADABC860010FD4A002820
:10E56000516814BF41F0010021F001005060704774
:10E57000F84B59680A0E120721F07F4142EA006207
:10E5800011435960022818BF7047F2F76AB9F14881
:10E590004068C0F303607047EE484068000F704762
:10E5A000EC483221C0684843EB49A1FB00108008C9
:10E5B0007047E84800697047E648006A7047E549D7
:10E5C000012008627047E349002008627047E14873
:10E5D00000787047002818BF0120DE490870704796
:10E5E000DC48406A7047DB48002141620170704797
:10E5F000D84988627047D748806A70472DE9F04350
:10E6000087B040F20F31F9F745F9002804BF07B091
:10E61000BDE8F083FFF7A5FDFFF7A8FDF7F735F993
:10E620005FEA00097ED1F2F79AFFCC48F4F77DFA51
:10E630000120F4F76DFAF2F7BFFCC94DC54EC94F82
:10E6400010F0010FC84615D00020F2F7BEFCFEF70F
:10E65000E8F8C5F800802020F5F7B5FAC248F5F7CC
:10E66000B8FA2020F5F7A1FA33202860386890F82E
:10E670001F012BE0F5F7CEFFBC48F6F780F8F6F760
:10E6800067F8F6F790F841003868B0F80E21B1FB52
:10E69000F2F1491CC1F34F01718090F8100110F0A4
:10E6A000FF0070700AD0F6F77EF839684000B1F8C4
:10E6B0000C11B0FBF1F0401CC0F34F010846F5F718
:10E6C000E2FF17202860386890F81E01B060F4F768
:10E6D000C9FAF4F7DFF9002808BFF4F72BFC7078CB
:10E6E00038B1401E10F0FF00707004BF7088F5F75D
:10E6F000CAFF7068C0F3036421460520F1F7F2FDFC
:10E70000FEF798F9012807D07068C0F30360A042B3
:10E7100008BFB9F1000F27D0F4F7DBFEC5F8008081
:10E72000202000E017E0F5F74EFA0020F5F751FA47
:10E73000F5F7F9FF40B1F5F7DEFFF6F714F8002022
:10E74000F6F71DF8F5F773FFF4F78CFAF4F7A4F970
:10E750000020F4F7EAF9FFF709FDFFF70CFDF9F7E0
:10E7600038FA07B0BDE8F0836846F4F766FE98B162
:10E770006846FFF7B4F8F8F7D3FE2146009A07F091
:10E78000A3FD6846FFF7FCFC814607F013FEF4F793
:10E79000A0FEF8F741FFB3E73868D0F8B00010F0FA
:10E7A000704F02D0F8F722FFAAE7F8F73CFFA7E77F
:10E7B0006F4A014602EB01110020CA6865498B6B64
:10E7C0009A4208BF70470120C86370472DE9F0479F
:10E7D000DFF8909180005F4FD9F8001000242646A2
:10E7E000D1F8001121FA00F000F00F00C1F303216D
:10E7F000C7E90B01884218BFBDE8F0870020DFF8A9
:10E800007081F863D9F80000D0F8001108EB04100B
:10E8100002799200D14001F00F050F2D04D08168DC
:10E8200020468847012805D0641CEBD0F86B0128EE
:10E830000AD102E02646FD62F8E708EB0610C06840
:10E84000B8630020F7F779F8796BF86A814207D04E
:10E8500040EA0022786300238921072003F01CFB93
:10E86000F86ABDE8F0872DE9F0413E480068B0F94C
:10E870001611B0F91401FFF756FCF1F7F2FF354D10
:10E880000120E861F7F759F800200CF0FCFF10F0C8
:10E89000C1FA0420FFF79AFFF7F734F8002004F0DC
:10E8A000B4FE00262E616E61AE6104F0CAFF022044
:10E8B0000FF03BFC00200FF057FCFFF766FC002038
:10E8C000EE60F8F7E4F8F8F72BFE052831D1686818
:10E8D000010FC0F30364A14202D02E616E61AE61EC
:10E8E0002046FFF773FF074604F0D5FF21460520B9
:10E8F00003F096FBF4B3022C44D0042C4AD0686891
:10E900000E2C4FEA106120F07F404FEA017104BFE6
:10E910000843686005D041F0007108436860F1F772
:10E92000A0FFFEF787F8012803D0F8F7F9FD0528C6
:10E93000CDD010F006F90020F8F797F80020F1F795
:10E940005DFD0020F7F7F4FFF6F7F6FF10F069FA27
:10E95000022010E020860010ABAAAAAA17430010DC
:10E9600010480040BC860010CD3A0010073B001054
:10E97000608600100AE00FF0E7FBBDE8F0410020E0
:10E980000FF001BC3846FFF739FECAE73846FFF7FB
:10E9900001FCC6E7384604F0F3FFC2E770470528DC
:10E9A0003CBFFE49087070470020FC498860486001
:10E9B000FB48006890F8CD00052838BF0870704704
:10E9C0000020F64948607047F4480078704770B5F9
:10E9D000F34D0024286890F8B80010F0020F0BD017
:10E9E000F8F79EFD022807D1EC482968007801EB72
:10E9F0008000B0F8D00084B2204670BD70B5E84DFC
:10EA00004FF48054286890F8B80010F0020F0DD031
:10EA1000F8F786FD022809D1E0482968007801EB63
:10EA20008000D0F8D000000CC0F31304204670BD65
:10EA3000DA488078002818BF012070472DE9F0419E
:10EA4000F8F76EFD022803D104F022FB022803D060
:10EA50004FF48050BDE8F0814FF480552E4604F00D
:10EA6000EBFBDFF83C830446CC4FD8F8000090F86D
:10EA7000B81011F0010F0CD0B0F8C200B9684042D4
:10EA8000814206DC2CB10020641EB860204604F0F0
:10EA9000D6FBD8F8001091F8B80010F0040F18BF9A
:10EAA000002C0AD0B1F8C800621E9040B1F8CA200C
:10EAB000824238BF1046C0F31306D1F8F00010F0C0
:10EAC000020F1CBFB978002902D0000CC0F3130557
:10EAD000B54298BF35462846BDE8F0812DE9F04F94
:10EAE000DFF8BCA287B0DAF8001091F8B82012F075
:10EAF000020F0DD0A94A91F8CC90DFF8A8B2177890
:10EB0000002809DB484503D2B84218BF064643D166
:10EB100007B00020BDE8F08F3E464FF0FF38F3F716
:10EB2000BBFFF4F7BEFE0025B9F1000F34D9DAF8C7
:10EB30000000002400EB8500B0F8D00081B2204630
:10EB4000F2F715FEF4F7F6F96846F4F776FC0028BC
:10EB500066D0029878B1014693489BF8002000786F
:10EB60005043421E07D331F9020B0028B8BF404280
:10EB70000444521EF7D2F4F7ACFCF3F78DFF0023E8
:10EB800022469221072003F087F9A04584BF2E4634
:10EB9000A0466D1C4D45CAD3B74244D0052E3CBF9C
:10EBA0007E490E70DAF80000B0F8CE1039B300EBF1
:10EBB000870200EB8600B2F8D020B0F8D00092B205
:10EBC00080B2801A484340F30F34F6F73DFB774B91
:10EBD0009BF80020002193F800C002FB0CF2002AF1
:10EBE0000DD930F81120224420F811209BF8002084
:10EBF00093F800C0491C02FB0CF28A42F1D84FF492
:10EC0000800004F0B5FCDAF80000002300EB860079
:10EC10008021B0F8D00082B2072003F03DF909E06E
:10EC2000F8F7E4FC90E704F007FB03283CBF401C26
:10EC300004F005FB012007B0BDE8F08F58485749A4
:10EC40000068B0F8C200424288688242BCBF401EE1
:10EC5000886070472DE9F04F93B093460E46044606
:10EC60004FF0000A04F0E8FADFF834814B4F05005A
:10EC7000D14610D1FFF793FAD8F80010B1F8C410BC
:10EC8000884208D30120C7F8089004F0D8FA13B0DE
:10EC90000120BDE8F08F002E1FDDB8680028B8BF46
:10ECA000C7F8089007DBD8F80010B1F8C010884208
:10ECB000BCBF401CB860D8F80000B968B0F8C0000C
:10ECC000884215DC032D13D2681CC7F8089004F0A5
:10ECD000B6FA13B00120BDE8F08F09D1D8F80000D2
:10ECE000B0F8C2004142B8688842C4BF401EB86054
:10ECF000B87850B1D8F8000090F8F00010F0040F88
:10ED00001EBF002013B0BDE8F08FD8F80000B0F9A6
:10ED1000BE108C420EDD796821447960B0F8BA00EB
:10ED2000884210DC4FF0FF30C7F80490FFF7D6FEA2
:10ED3000824608E07868002805DD002CD4BF012158
:10ED40002146401A7860DFF8689099F8000007289B
:10ED50003BD118485946007842006846FFF793F9BE
:10ED6000ADF80040ADF80260ADF804503889ADF858
:10ED70000600B888ADF80800D8F80000B0F8BE105A
:10ED8000ADF80A10B0F8C010ADF80C10B0F8BA1019
:10ED9000ADF80E10B0F8C2000EE00000A48600101E
:10EDA000BC860010588500105C8500105985001045
:10EDB000DD8500105F850010ADF8100099F80000A7
:10EDC000072804BF6846FEF744FA504613B0BDE872
:10EDD000F08F474810B50068D0F8F00010F4807F3D
:10EDE00006D0C0F30330012101FA00F0F5F70EF967
:10EDF000404900204870887010BD70B53D4D00241A
:10EE0000A878002814BF01260026687828B904F0E5
:10EE100022FA002808BF002100D001218E4227D00D
:10EE20000A1C18BF0122AA7031480068D0F8F030DF
:10EE300013F0040F0ED021B1C3F30310052808D23C
:10EE400006E00021A960696090F8CD00052800D295
:10EE50002870012413F0020F18BF0124002A18BFE4
:10EE6000012200238221072003F016F8F1F76AFA45
:10EE7000204670BD2DE9F0411D4800270068D0F8FC
:10EE8000F01011F4807F30D01A4E7078051C18BF36
:10EE90000125C1F30330184A5268012303FA00F038
:10EEA000024011F4007F0AD052B10CF0E3FC0428B8
:10EEB00018BF08280FD002200CF0D7FC0BE022B1BD
:10EEC000002401200CF0D1FC06E00CF0D3FC042857
:10EED00018BF0828EFD10124A54206D0201C18BF76
:10EEE00001207070FFF789FF07463846BDE8F081C2
:10EEF000BC860010A4860010001000407148007805
:10EF000070477048406800F5407070476D48406831
:10EF100000F58070704770B56A4C4FF448306A4A0B
:10EF200060600168914204BF4168B1F50C7F3BD13C
:10EF30008168B1F5464F37D8644AC568954223D0F9
:10EF40004FF0000C03466246BCEB910F0AD253F817
:10EF5000046B521C86EA0C0CB2EB910FF7D3BCF198
:10EF6000000F21D1026A7AB14FF0000C03466246CD
:10EF7000BCEB910F06D253F8046B521CB444B2EBB5
:10EF8000910FF8D365450FD1012500F58070FEF78C
:10EF9000CCFF48B1606800F54070FEF7D5FF00284F
:10EFA0001EBF2570012070BD002070BD45490020A6
:10EFB00008704FF44830F4F7A7BE4248017841B1D9
:10EFC0004068414A0168914202BF4168B1F50C7F37
:10EFD0007047002070473B4B5B6803F58073184413
:10EFE000F4F788BF374B5B6803F540731844F4F7B8
:10EFF00081BF3448406800F5A0607047314B5B68C2
:10F0000003F5A0631844F4F775BF2E484068006903
:10F0100070472C4949680A6982429CBF00207047AA
:10F0200000EB400001EB001000F5C0607047254A7E
:10F03000526802EB8000436A406E1A4400FB0120D4
:10F0400070472049886070471E48806870472DE9E6
:10F05000F0011C4B00220127D3E90146904683189A
:10F0600093F92030002B12DB07FA02FC1CEA060F92
:10F070000DD002F0FF0C04EB8C0CDCF82450DCF813
:10F0800064C0254403FB0C5341F8223001E041F8F1
:10F090002280521C102AE2D3BDE8F00170470029FB
:10F0A000B8BF704730B49446064A526802EB8000FD
:10F0B000446A406E224401FB002030BC1A4661467F
:10F0C000F4F718BFB086001054465053EFBEADDEC3
:10F0D000FB4840687047FA4948607047F8488068C4
:10F0E0007047F74AD16811F0405F12BF10F0804FAF
:10F0F0000843D0607047F24988707047F0488078C4
:10F1000070470200EF484FF008010068438A008A08
:10F1100003FB00101CBFC01C20F0030070472DE94A
:10F12000F04104460D460846F8F7F4F978B1012697
:10F1300006FA04F010F0CA0F18BF002C07D0032CF9
:10F1400005D8E0494FF4403201200B6802E000206E
:10F15000BDE8F081A04213D006FA00F111F0CA0F09
:10F160000BD0598A1F8A4FF0080C01FB07C1C91C3C
:10F1700021F0030C0CEB4C010A44401C0328E9D994
:10F180000120A8420CD0B3F812C01C8A08210CFB45
:10F190000411C91C21F00301401C0A440328F0D9C2
:10F1A0001046BDE8F0812DE9F04F0E4690F821A001
:10F1B00090F8209000F15005ADF20C4D1746012457
:10F1C00011463046FFF7ABFFA11E012E08BFBE4916
:10F1D00006D0022E08BFBD4902D0032E08BFBC498D
:10F1E0004FF0000830B102688A4204BF4068CDE9A0
:10F1F000002001D0CDE90018B648022E01680CBFEE
:10F20000B1F98A00B1F93A0086460CBFB1F98820FD
:10F21000B1F93820934600230AFB09FCBCF1000F2A
:10F220000ED935F913107145D8BF8B4505DC9142D5
:10F23000C8BF0A468142B8BF08465B1C9C45F0D84F
:10F24000104400EBD07042100023BCF1000F88BFC7
:10F25000E94616D935F91300801A00EBD070411039
:10F260007F29C8BF7F2105DC11F1800FB8BF6FF087
:10F270007F0100DA002409EB03005B1C01729C454E
:10F28000E8D88DF804409DF80500FF283CBF401CDD
:10F290008DF80500ADF806206C4639463046FFF77C
:10F2A0003EFF78B18749082209684B8A098A03FB27
:10F2B00001222146F4F71EFE01280CBF4FF0010881
:10F2C0004FF0000840460DF20C4DBDE8F08F2DE9DF
:10F2D000F047984615460E468146F8F718F9F8F7B4
:10F2E00019F9002808BFBDE8F087754F7A4C3878C7
:10F2F000814588BFBDE8F0870CD287F800904FF0B9
:10F300000000F8704FF0FF024FF014017248FEF752
:10F31000CEFE19E097F803C0BCF1050F28BFBDE889
:10F32000F087BCF1000F18BF00200DDD14F820108D
:10F33000B14206D104EB80014978A94208BFBDE87B
:10F34000F087401C6045F1DBF87804EB800104F89D
:10F3500020604D70A1F80280401CF870BDE8F08775
:10F3600070B5054616460C460846F8F7D3F800284F
:10F370001CBF681E032832BF022E002070BD04EBA4
:10F38000C400400105EB450100EB411006EB4601CE
:10F3900000EB011000F5403000F5686070BD2DE90C
:10F3A000F04F97B04FF0000816460D460746CDF8CF
:10F3B0003080FF2230216846CDF83480FEF777FE9A
:10F3C000DFF818A14FF47F30CDF800A00168880A5B
:10F3D000424211EB822218BF401C404201EB8000E8
:10F3E000C01C20F0030000F500503D49428A437CD8
:10F3F00052BA007C63F31F4242EA00600190088821
:10F40000A1F1040940BAADF80A003869039099F8EF
:10F4100000008DF81800002231462846FFF7A0FFB3
:10F420000446012231462846FFF79AFF4FF0010CAF
:10F43000012D04D0022D18BF032D53D081E00022EE
:10F44000114624B32368534521D1237A647A28B125
:10F45000D0F800B0D34504BF027A417A181902EB04
:10F46000010A504583BFADF830C0ADF83430ADF877
:10F470003640ADF830809CBFADF83420ADF8361082
:10F48000BDF83400BDF836100844ADF83200BDF8C0
:10F490003400BDF836109DF81820C0B28DF8080071
:10F4A000C9B20CFA02F28DF8091012F00E0F19BF52
:10F4B000401C8DF80800481C8DF8090041E0000050
:10F4C000C0860010BC8600104654525946544D3236
:10F4D00046544D33E0860010B4EB001046464853C6
:10F4E000C4860010002194B1226852450FD1227ABF
:10F4F00018B10368534508BF017A8A4287BFADF847
:10F5000030C0ADF83220ADF83080ADF83210022DA9
:10F5100018BF032D15D1387C10F0300004BF17B090
:10F52000BDE8F08FBDF832003146401C8DF8080070
:10F530002846FFF7F4FD00280CBF404640798DF8BF
:10F540000900FF480DF1380A6B46B0E816108AE84A
:10F55000161090E8071012AC84E807109DF8180008
:10F56000082813D20EA951F82000B0F1FF3F0DD0AA
:10F5700007EBC000D0E90A10CDE9041099F80300A8
:10F58000F049820003F11C00FEF77DFDBDF830104C
:10F590006C46CAB231462846FFF7E2FE48B1302237
:10F5A0002146F4F7A7FC01280CBF4FF001084FF0EB
:10F5B0000008404617B0BDE8F08F012200218240CC
:10F5C00012F0CA0F10D001281CBF0228032804D053
:10F5D000072808BF4FF4907106E0DB480821006857
:10F5E000428A008A02FB001108467047012310B5C9
:10F5F0000022834013F0CA0F0FD001281CBF02283D
:10F60000032802D0072803D007E0FFF788FD03E0B6
:10F6100000220120FFF7A4FE0246104610BD2DE98E
:10F62000F04106460127F7F772FF8046F7F772FFB1
:10F63000002808BFBDE8F081C44D686810F4807FE1
:10F6400018BF02240DD00120A04010F0CA0F05D031
:10F65000424621463046FFF7A6FD0746306978B995
:10F660000BE010F4007F18BF0324ECD110F007006A
:10F6700018BF0124E7D1BDE8F0812878112805D210
:10F68000424621463046FFF78AFE07463846BDE827
:10F69000F081AE4908617047AC4810B40069002899
:10F6A00008BF4FF47C30AA4A016891421CD14168DE
:10F6B000B1F5007F18D3836800228446B3F5056F47
:10F6C00088BF4FF405630021B1EB930F24BF10BC3A
:10F6D00070475CF82140491C2244B1EB930FF8D3EA
:10F6E000002A04BF10BC7047002010BC704770B5E2
:10F6F0000022C260D0F808C0012113460446BCF5C0
:10F70000056F88BF4FF4056C0022B2EB9C0F06D248
:10F7100054F82250521C2B44B2EB9C0FF8D35A429F
:10F72000C2608A4A127912F0800F07D14FF47C3000
:10F730004FF405622146F4F7DDFB014601290CBFB9
:10F740000120002070BDFF2270B500250446056130
:10F750004FF400615030FEF7AAFCA584E584E56211
:10F76000A56265632563E563A56365642564E56457
:10F770000120A56470BD2DE9F0414FF47C310446B1
:10F78000734E0868B04218D14868B0F5007F14D3B2
:10F790008A6800230D46B2F5056F94BF94464FF476
:10F7A000056C0020B0EB9C0F26D255F82070401C51
:10F7B0003B44B0EB9C0FF8D3F3B1FF224FF405614B
:10F7C0002046FEF774FC4FF40870C4E900604FF463
:10F7D0000560A0600020E06084F8200084F821002B
:10F7E00084F8220084F8230020616061A061E06158
:10F7F0002046FFF7A8FF07E0B2F5056F88BF4FF47A
:10F8000005622046FEF730FC0120BDE8F08170B4AF
:10F8100002684FF408715160016801F1500291F8DB
:10F8200021C091F820300CFB03F102EB41010022D2
:10F83000BCF1000F08D900EB4204521CB4F8DE40C2
:10F8400021F8024B9445F6D80022002B08D900EB92
:10F850004204521CB4F8064121F8024B9342F6D8F8
:10F860000022BCF1000F08D900EB4204521CB4F88E
:10F87000644021F8024B9445F6D80022002B08D9A9
:10F8800000EB4204521CB4F88C4021F8024B934226
:10F89000F6D8B0F8DA2021F8022BB0F8DC2021F8F5
:10F8A000022BB0F8D82021F8022B00240022BCF152
:10F8B000000F0ED904EB440505EB041500EB85059C
:10F8C00005EB4206521CB6F8526121F8026B624504
:10F8D000F6D30022002B0ED904EB440505EB0415EA
:10F8E00000EB850505EB4206521CB6F8826221F852
:10F8F000026B9A42F6D3641C042CD7D370BC7047B9
:10F900002DE9F74F88B000250A992C462E46096844
:10F91000049101F150030999002984BF0D49D1F8E0
:10F92000008029D90022002888BFB8F93A701AD976
:10F9300033F9021B0029B4BFC1F1000C8C460BE067
:10F94000EC6D0200B4EB0010BC860010C086001005
:10F9500053454C46E0860010BC45BCBF0D44641CBA
:10F96000521C8242E4D30999761C8E42DAD3002CD1
:10F97000C8BF95FBF4FA08DC4908414301EB50028B
:10F98000049901EB4201B1F950A0002102910191CB
:10F99000049950310091002103910999002969D9F6
:10F9A000FF49009E069609684FF0000B4FF00109D1
:10F9B000B1F81CE091F824105F46D846CDF814B099
:10F9C0000791002829D9B6F900204FF0000C0699BC
:10F9D0009344634600280DD9B1F90040A51A48BFE9
:10F9E000151B7545B8BF0CF1010C01EB49015B1CFF
:10F9F0008342F1D307998C4503D305997F1C1144A9
:10FA0000059108F1010806EB49068045DBD3002F7C
:10FA1000C4BF059991FBF7F101DC9BFBF0F1039B5F
:10FA20000A9A09B202EB4302A2F86410DC4A126897
:10FA3000538BAAEB0303994209DD128B52448A428D
:10FA400005DD019A114401910299491C0291009926
:10FA5000099A01EB400100910399491C03919142DD
:10FA60009ED30299002905DDDDE9011291FBF2F137
:10FA7000019102E05146CDF804A00A9AA2F8DA10EA
:10FA800000210291039104995031009100210491C9
:10FA9000002865D9C249009F069709684FF0000BFE
:10FAA000099EB1F820E091F82510D846D946CDF846
:10FAB00014B00791002E2BD9B7F900204FF0000C9D
:10FAC000069993446346002E0DD9B1F90040A51A5A
:10FAD00048BF151B7545B8BF0CF1010C01EB400187
:10FAE0005B1CB342F1D307998C4504D3059908F107
:10FAF00001081144059109F1010907EB4007B145DF
:10FB0000DAD3B8F1000FC4BF059991FBF8F101DC1D
:10FB10009BFBF6F1049B0A9A09B202EB4302A2F89E
:10FB20008C109F4A1268538BAAEB0303994209DD9C
:10FB3000128B52448A4205DD039A114403910299C3
:10FB4000491C02910099891C00910499491C049157
:10FB500081429FD302980028C4BF039991FBF0FA19
:10FB60000A98A0F8DCA001980A99504400B200EB72
:10FB7000D0704010A1F8D8000BB0BDE8F08F2DE98F
:10FB8000F04F146887B015460E468046A1F1200953
:10FB9000202928BF4FF0FF3B05D24FF0010000FAAB
:10FBA00006F0A0F1010B31BF0020012000FA09F09E
:10FBB000401E0290B8F1200F3DBF012000FA08F06E
:10FBC000401E4FF0FF3038BF002207D3A8F12002BB
:10FBD0004FF0010101FA02F1A1F10102C6F1200A80
:10FBE000202E34BF20FA0AF100FA09F1B240114385
:10FBF000B040CDE90001206920F4FE602061694831
:10FC0000406810F0010F79D010F4807F05D02A46AB
:10FC10003146404601F088FA8AE010F4007F2A4617
:10FC20003146404602D001F097FC81E001F057F9DF
:10FC30000020A86107466861B8F1000F22D905EBE2
:10FC40004700B0F98C000028B8BF404200B25449C8
:10FC50000968B1F93810814211DD7A0905EB820C8F
:10FC600007F01F0301219940DCF8142083B21143EF
:10FC7000CCF81410FAB2FF210420FFF728FB7F1CF8
:10FC80004745DCD30027B8F1010F1CBFA8F10100E4
:10FC900003904DD005EB4700B0F98E30B0F98C20C1
:10FCA000991A48BFD11A09B2DFF8F4C0DCF800C0D5
:10FCB000BCF932C08C4537DAB5F9DC10B2EB010C77
:10FCC00048BFA1EB020C0FFA8CFC5A1A48BFCA1AA3
:10FCD00011B28C4513DB7A0905EB820107F01F0C8A
:10FCE00001224B6902FA0CF21A434A61B0F88C30D7
:10FCF000FAB2FF210420FFF7EAFA15E02BE0791CA5
:10FD00004B0905EB830E01F01F0C0122DEF81430C5
:10FD100002FA0CF21A43CEF81420B0F88E30CAB2B0
:10FD2000FF210420FFF7D3FA03987F1C8742B1D349
:10FD30006969E869B14008432063A969286AB1404C
:10FD4000084360636969202E34BF21FA0AF101FA81
:10FD500009F1084360631349087910F0040F00F0BB
:10FD6000078200202863E8620846407850BB0027DD
:10FD7000002E27D90A4905EB47000968B0F952015E
:10FD8000B1F95C20824203DCB1F95E10814216DADF
:10FD90007A0907F01F03012105EB820C994003E06B
:10FDA000E0860010C0860010DCF82C2083B21143DE
:10FDB000CCF82C10F9B2FF220220FFF788FA7F1C42
:10FDC000B742D7D30020A8626862FE48407830BBB3
:10FDD0000027B8F1000F22D9FB4905EB470009685D
:10FDE000B0F98202B1F95C20824203DCB1F95E1005
:10FDF000814211DA7A0905EB820C07F01F03012119
:10FE00009940DCF8242083B21143CCF82410FAB2D4
:10FE1000FF210220FFF75BFA7F1C4745DCD300205F
:10FE20002864E863E748407890BB0027002E2FD96C
:10FE3000E54905EB47000968B0F99E01B1F960207A
:10FE40008242DCBFB1F96220904210DD7A0905EBF5
:10FE5000820C07F01F0301219940DCF83C2083B29B
:10FE60001143CCF83C10FF22F9B201200BE0B1F9AC
:10FE70006C208242DCBFB1F96E10884205DD83B28E
:10FE8000F9B2FF221020FFF722FA7F1CB742CFD32E
:10FE90000020A8636863CB48407898BB0027B8F17E
:10FEA000000F2FD9C84905EB47000968B0F9CE0209
:10FEB000B1F960208242DCBFB1F96220904210DDCE
:10FEC0007A0905EB820C07F01F0301219940DCF849
:10FED000342083B21143CCF83410FF21FAB2012050
:10FEE0000BE0B1F96C208242DCBFB1F96E108842A0
:10FEF00005DD83B2FAB2FF211020FFF7E8F97F1C7D
:10FF00004745CFD300202865E864A8646864AD48FD
:10FF10004078E8BB0027002E22D9AB4905EB47000B
:10FF20000968B0F9EA01B1F96420824203DCB1F951
:10FF30006610814211DA7A0905EB820C07F01F0383
:10FF400001219940DCF84C2083B21143CCF84C10CD
:10FF5000F9B2FF220320FFF7BAF97F1CB742DCD3C6
:10FF60000027B8F1000F24D9974905EB470009682D
:10FF7000B0F91A03B1F96420824203DCB1F96610CA
:10FF8000814213DA7A0905EB820C07F01F0300E0C7
:10FF90000FE001219940DCF8442083B21143CCF8F2
:10FFA0004410FAB2FF210320FFF791F97F1C474567
:10FFB000DAD3696AE86AB14040EA010EC4F838E071
:10FFC000A96A286BB1400843E063696A202E34BFF8
:10FFD00021FA0AF101FA09F141EA0007E763696BC6
:10FFE000E86B01FA06F140EA01022264A96B286C71
:10FFF00001FA06F140EA01006064696B34BF21FA3E
:020000021000EC
:100000000AF101FA09F141EA000060646B6CE96CE5
:1000100003FA06F341EA0301A1640391AB6C296D75
:1000200003FA06F341EA0301E1646B6C34BF23FA7F
:100030000AF303FA09F343EA0101E164059132EAA4
:100040000E054EEA0501256420EA070C049147EAF3
:100050000C00C4F844C006EB0801069008BFBCF1D0
:10006000000F45D000231A461846002988BF4FF0DC
:1000700001083DD94FEA501904EB890900F01F0A25
:10008000D9F8409008FA0AFA19EA0A0F03D0864212
:1000900094BF521C5B1C401C8142EBD8012B10D139
:1000A00005EA0B0040EA0E00A06302980CEA00008B
:1000B0003843E06325EA0B00206402982CEA000034
:1000C0006064012A14D1206C009AA36B02401A4389
:1000D000A263626C019BD4F83CC0134043EA0C035A
:1000E000E363009B98432064019822EA0000606467
:1000F000DDE903208243A264049840EA020CDDE9B2
:10010000050320EA0300E064069B43EA000508BFFC
:10011000002821D000231A461846002988BF01274D
:1001200017D94FEA501804EB880800F01F09D8F8D7
:10013000488007FA09F918EA090F03D0864294BFEC
:10014000521C5B1C401C8142EBD8002B18BF002ABC
:1001500002D10020A064E0641A48007910F0010F79
:1001600006D0206B20EA0C002063606BA84360631C
:10017000206B0099084203D1626B01990A4203D0B7
:10018000216941F01001216110EA0B0F03D1616B6D
:100190000298014203D0206940F020002061A06B4A
:1001A0000099084203D1E26B01990A4203D0216908
:1001B00041F04001216110EA0B0F08D1E16B029878
:1001C000014203E0C0860010E086001003D02069E1
:1001D00040F080002061206C0099084203D1626CDD
:1001E00001990A4203D0216941F48071216110EA2A
:1001F0000B0F03D1616C0298014203D0206940F4D7
:1002000000702061A06C002804BFE06C002803D0BF
:10021000206940F48060206107B00120BDE8F08FC4
:100220002DE9F04FCBB017460D460446F2F734FCEB
:100230000120F0F768FC06461120F0F764FC30431B
:1002400014BF012002208DF8180014BF11201220C5
:100250008DF81900F1F7AAFC38B19DF818009DF847
:1002600019108DF818108DF819009DF81800F0F786
:100270004AFC002818BF284604909DF81900F0F7A2
:1002800042FC002818BF20460590F2F732FF0022FA
:10029000002D88BF24A90BD98356142BA8BF143B6B
:1002A00002DA0A2BA8BF12338B54521CAA42F3D392
:1002B000F2F721FF0021002C88BF24AA07D9435C54
:1002C00002EB010C491C8CF826308C42F7D8F2F76F
:1002D000CFFD0390FE480DF1180A007910F0200FB1
:1002E00055D007F1DE00009028300025E9460DF1D9
:1002F000100B01905BF825601AF80500F3F740FA3F
:100300000024002E1AD905EB450000EB051024A9A6
:1003100001EB400818F90420262A28BF002006D245
:100320001AF805000021F2F73AFAF3F72FFA59F814
:10033000251021F81400641CB442EBD36D1C022D6F
:10034000D8D3E44C26781D2E21D100210A460DF188
:100350001C085BF822500020002D88BF59F822C0ED
:1003600007D93CF8103028F81130401C491C854250
:10037000F7D8521C022AECD31D2E08D14046FDF7B7
:1003800042F920781D2804BF07A8FDF73CF9D04D9D
:10039000287910F00C0F00F0B083039800F0F00003
:1003A000F2F736FC9DF81800F1F7CDF907909DF8AB
:1003B0001800F1F76EFA002437901AF80400F2F7EB
:1003C00031F944A941F824001AF80400F1F79EFA23
:1003D0000EA941F824001AF80400F1F7EAFB20A95D
:1003E00041F824001AF80400F1F71BFC22A941F897
:1003F00024001AF80400F0F7C5FB46A918AA41F832
:1004000024001CA81AA902EB840200EB840001EB73
:1004100084010092CDE9011016A800EB840314A812
:1004200000EB840212A800EB84011AF80400F1F733
:10043000D7FE1AF80400F2F706F81EA941F82400C6
:100440001AF80400F2F73EF910A941F82400641CE0
:10045000022CB2D3A04E3068B0F848109DF81800B6
:10046000F1F785F9002400211AF80400F2F7C0F82A
:10047000994E306890F84A101AF80400F1F75AFAC9
:100480001AF804000021F1F7AEFB1AF8040000216D
:10049000F1F7E1FB1AF804000121F0F759FB30688D
:1004A000B0F84C101AF80400F1F760FF1AF80400D5
:1004B0000021F2F7CFF8641C022CD4D384484FF00B
:1004C0000009007910F0040F00F0DE813446206846
:1004D00090F84B3090F85920B0F850100091CDE9C9
:1004E000012390F84F3090F84E2090F858109DF866
:1004F0001800F1F7BCFC206890F84B3090F85920B8
:10050000B0F850100091CDE9012390F84F3090F8E9
:100510004E2090F858109DF81900F1F7A8FC9DF8AE
:1005200018000021F2F796F89DF819000021F2F763
:1005300091F83AADF2F7FEFCFCF77CFA012806D000
:100540002846F2F77AFF00287DD0F2F7C2FFF2F7D3
:10055000A3FA3E99002204AD002055F82230002B6A
:100560000ED902EB420C0CEB021C07EB0C1C31F811
:10057000026B0CEB4008401CA8F852618342F6D88D
:10058000521C022AE8D35548D0E90010CDE90C10DE
:100590009DF81800F0F7B7FA48909DF81900F0F7A9
:1005A000B2FA49909DF8180040A9F1F760FA9DF859
:1005B000190042A9F1F75BFA9DF8180008A9F1F7B4
:1005C000D3FA9DF819000AA9F1F7CEFA424C206837
:1005D00090F84B3090F85920B0F852100091CDE9C6
:1005E000012390F84F3090F84E2090F858109DF865
:1005F0001800F1F73CFC206890F84B3090F8592037
:10060000B0F852100091CDE9012390F84F3090F8E6
:100610004E2090F858109DF81900F1F728FC9DF82D
:1006200018000CA9F1F77EFA9DF819000CA9F1F752
:1006300079FA00249DF818000021F2F70BF89DF8D4
:100640001900002100E017E0F2F704F89DF8180007
:100650000021F0F73EFA9DF819000021F0F739FA71
:100660001AF804000121F0F734FA1AF80400C0F374
:10067000011001280AD102E0F6F7B8FF5CE784F028
:10068000010001211AF80000F0F723FACDF8E090FC
:10069000CDF8E4909DF8180038A9F1F7C8F99DF855
:1006A000190038A9F1F7C3F904A8002150F82480F3
:1006B0001AF80400F2F719F900250190B8F1000FBB
:1006C00056D904EB440024A900EB041008E0000014
:1006D000C0860010E3850010E0860010D868020094
:1006E00001EB400107EB001B0091009838AA0021A4
:1006F0004657CDF8E090CDF8E4901AF80400F2F7F0
:100700000CF8202E06DBA6F1200101208840CDE95F
:10071000389003E00120B040CDE938091AF8040010
:1007200038A9F1F784F9389838AAC0433890399835
:100730000921C04339901AF80400F1F7EEFF3AAEF0
:10074000F2F7F8FBFCF776F9012806D03046F2F70D
:1007500074FE00287ED0F2F7BCFEF2F79DF90198F6
:1007600000880BEB45016D1CA1F89E014545BCD3EB
:10077000CDF8E090CDF8E4901AF8040038AA0021F2
:10078000F1F7CBFF641C022CFFF454AF9DF8180066
:1007900008A9F1F7C7F99DF819000AA9F1F7C2F9FC
:1007A0009DF818004899F0F794F99DF819004999B7
:1007B000F0F78FF99DF8180040A9F1F738F99DF886
:1007C000190042A9F1F733F9FE4C206890F84B303C
:1007D00090F85920B0F854100091CDE9012390F819
:1007E0004F3090F84E2090F858109DF81800F1F70F
:1007F0003EFB206890F84B3090F85920B0F8541028
:100800000091CDE9012390F84F3090F84E2090F8F8
:1008100058109DF81900F1F72AFB9DF818000121E6
:10082000F1F718FF9DF819000121F1F713FF3AAC19
:10083000F2F780FBFCF7FEF8012806D02046F2F71D
:10084000FCFD00287DD0F2F744FEF2F725F90022E6
:1008500004AC00E081E03E9954F822C00020BCF1D5
:10086000000F0ED902EB420303EB021307EB031355
:1008700031F8025B03EB4006401CA6F8EA518445C0
:10088000F6D8521C022AE7D3CF48007910F0080F9F
:100890007ED0CC4C206890F84B3090F85920B0F8BE
:1008A00056100091CDE9012390F84F3090F84E207A
:1008B00090F858109DF81800F1F7D9FA206890F8D0
:1008C0004B3090F85920B0F856100091CDE9012333
:1008D00090F84F3090F84E2090F858109DF819007D
:1008E000F1F7C5FA00210DF1100C00205CF8212071
:1008F000002A0CD901EB410303EB011307EB0313AF
:1009000003EB4005401CA5F836928242F8D8491CFA
:100910000229EAD32068002590F86800B5EB400F63
:1009200036DA206890F86800A842D4BF012100217F
:100930009DF81800F1F78EFE206890F86800A84234
:1009400000E00DE0D4BF012100219DF81900F1F76E
:1009500081FE3AAEF2F7EEFA05E0F6F747FEF1E671
:10096000F6F744FE66E7FCF765F8012805D0304647
:10097000F2F763FDD8B3F2F7ACFDF2F78DF83E99CC
:100980004FF0000904AB0022104653F8296000E044
:1009900058E0002E05D931F91030401C1A44864227
:1009A000F9D8B2FBF6F2701E3DD009EB490303EB18
:1009B000091307EB031B31F9103001EB400C3CF934
:1009C000028CB3EB080348BF5B4231F91080B8EBEF
:1009D000020831F910804CBFA2EB0808A8EB02080E
:1009E0003CF902EC3CF902CCBEEB020E00E00FE059
:1009F0004CBFA2EB0C0CACEB020CE0450BEB400C3B
:100A000009DDBCF936824345C8BFACF8363208E090
:100A1000F6F7ECFDA7E7BCF934829845B8BFACF80F
:100A20003432401EC7D109F1010901EB4601B9F189
:100A3000020FA7D320686D1C90F86800B5EB400F3B
:100A4000FFF66FAF9DF818000799F0F790FE9DF83C
:100A500018003799F0F72CFF00241CAD1EAE20AF14
:100A60000DF188080DF588790DF58C7B59F8241067
:100A70001AF80400F1F7BCFD0EA850F824101AF87B
:100A80000400F0F757FF57F824101AF80400F1F7A4
:100A9000AAF858F824101AF80400F1F7DCF85BF80B
:100AA00024101AF80400F0F753F81AA918A851F8FE
:100AB000241055F8242050F82400CDE9000116A890
:100AC000029250F8243014A850F8242012A850F8AC
:100AD00024101AF80400F1F7CAF956F824101AF88D
:100AE0000400F1F743FC10A850F824101AF8040091
:100AF000F1F7B0FD641C022CB8D30398F2F788F824
:100B00004BB0BDE8F08F30480121816000211122F7
:100B1000C1600270C170FDF7CEB82B49002088601B
:100B200070472DE9F04F284DADF56F7D4FF000086F
:100B30000127C5E902781120287085F80380FDF7A8
:100B4000BAF868684FF4407131EA000008BF002627
:100B500000F095811D20FCF7A7FAED901D20FCF711
:100B600038FDDFF864A0EE904FF46D716846DAF856
:100B70001040FDF77EFA0094BAF8040010F4804F9C
:100B80001CBF2046FEF7DFFD02F0B7FB30B10AF0D4
:100B900071FE082818BF8AF8017001D18AF8018017
:100BA00000986A4690F8203090F821C050300CFB35
:100BB00003F100EB41000021BCF1000F0DD930F82A
:100BC000025B03E0E0860010C086001002EB4106E5
:100BD000491CA6F8DE508C45F1D80021002B08D91D
:100BE00002EB410630F8025B491CA6F806518B4225
:100BF000F6D80021BCF1000F08D902EB410630F80D
:100C0000025B491CA6F864508C45F6D80021002BE5
:100C100008D902EB410630F8025B491CA6F88C505B
:100C20008B42F6D830F8021BA2F8DA1030F8021B1B
:100C3000A2F8DC1030F8021BA2F8D8100025002121
:100C4000BCF1000F0ED905EB450606EB051602EBCD
:100C5000860606EB410B30F8029B491CABF852911B
:100C60006145F6D30021002B0ED905EB450606EBB6
:100C7000051602EB860606EB410B30F8029B491C79
:100C8000ABF882929942F6D36D1C042DD7D36146FE
:100C90001846FEF735FEDAF804003E4610F4004F21
:100CA00003D1694600F024FF0646ED98FCF7FCF9F5
:100CB000EE98FCF78EFC94F8209094F82150002ECA
:100CC0001CBFB9F1000F002D00F0D9809AF8040084
:100CD00010F0020F04D06A462946484600F0A6FDEF
:100CE0009AF8040010F0050F04D06A4629464846D9
:100CF000FEF745FFFE48007910F0080F7CD0009AFF
:100D0000DFF8F0E36846116921F4C0511161F84938
:100D1000CDF86080CDF85C8091F801B0BBF1000F98
:100D20001CD10021002D19D9DEF800C000EB4103D1
:100D3000B3F93632BCF96AC09C450CDA4B0900EBBA
:100D4000830301F01F0AD3F85CC007FA0AFA4CEAE1
:100D50000A0CC3F85CC0491CA942E5D3C0F858800E
:100D6000C0F85480BBF1000F1ED10021B9F1000F73
:100D70001AD9DEF800C000EB4103B3F96633BCF9C1
:100D80006AC09C450DDA4FEA511C00EB8C0301F060
:100D90001F0AD3F854C007FA0AFA4CEA0A0CC3F83F
:100DA00054C0491C4945E4D3916BC36D1943436D4D
:100DB000AB4019439163D16B036E1943836DAB4014
:100DC0000B43D363416D202D39BFC5F1200C21FAAF
:100DD0000CF1A5F1200C01FA0CF11943D163416D1E
:100DE000002904BF816D002903D0116941F400611D
:100DF0001161C16D002900E007E004BF006E00280A
:100E000003D0106940F480501061B94D287910F07A
:100E1000400F0FD16069401C60612069002814BF39
:100E2000E069A06900F1010014BFE061A0616846BB
:100E3000FEF7EDFCC4F80C80A36800222146A4460E
:100E4000B3F5056F88BF4FF405630020B0EB930F37
:100E500006D25CF82090401C4A44B0EB930FF8D3C4
:100E60005042C860287910F0800F05D14FF47C30D3
:100E70004FF40562F3F73EF82046FEF7D0FB412021
:100E80008DF8B40316B3207C8DF8B503607C8DF823
:100E9000B603A07C8DF8B703E07C954C8DF8B803C1
:100EA000E06838B19DF8B813F02202EA10600843F8
:100EB0008DF8B80300230522EDA9072001F079F889
:100EC000C4F808800DF56F7DBDE8F08FFF208DF828
:100ED000B5038DF8B6038DF8B7030F20DDE72DE9D4
:100EE000F74F84B04FF0000AC2F820A00646C2F8BF
:100EF0001CA00598DFF8FC81174654464FF0010905
:100F0000002821D907EB4400B0F964000028B8BFDD
:100F1000404200B2D8F80010B1F9381081420FDD1C
:100F2000610907EB810104F01F03CA6909FA03F3A1
:100F30001A43CA6183B2E1B2FF220420FEF7C7F967
:100F40000598641C8442DDD3002401281CBF059849
:100F5000451E46D007EB4403B3F96620B3F964108D
:100F6000501A48BF881A00B2D8F800C0BCF930C087
:100F7000844533DAB7F9DA00B1EB000C48BFA0EBD7
:100F8000010C0FFA8CFC111A48BF811A08B2844573
:100F900011DB600907EB800004F01F02C16909FA48
:100FA00002F21143C161B3F86430E1B2FF220420C0
:100FB000FEF78DF912E0601C410907EB810100F09A
:100FC0001F0CCA6909FA0CFC42EA0C02CA61C1B2E0
:100FD000B3F86630FF220420FEF779F9641CAC42B6
:100FE000B8D3D8F8000090F8361000297ED090F8D9
:100FF00037003D68814288BF0846002405990029D2
:1010000084BF401C009071D94FF0010E00984FF042
:1010100000090121CA46012852D9364800680390C8
:10102000B0F93A3004FB066002900EFB06600190B6
:1010300004FB061005EB4000B0F950C0BCF1000FF6
:10104000B4BFCCF100006046834239DB0EFB0610D2
:1010500005EB4000B0F950000028B4BF4242024600
:1010600093422DDB029A521A05EB4202B2F94E80EE
:10107000B8F1000FB4BFC8F10002424693421FDB33
:10108000019A521A05EB4202B2F94E20002AB4BF6F
:10109000C2F1000B93469B4512DCA0EB0C0C0398AD
:1010A000B0F934006045B8BF09F10109A2EB0802AC
:1010B0008242C8BF0AF1010A491C00988142B7D395
:1010C000BAEB090048BFA9EB0A000A49096891F880
:1010D0003610884219DB600907EB800004F01F031B
:1010E0000121C26999401143C16105E018E0000087
:1010F000C0860010E086001007EB4400E1B2B0F8B3
:101100006430FF220420FEF7E2F80598641C844254
:1011100006D2002C18BFA4F1010E7FF477AF73E75D
:1011200007B00120BDE8F08F2DE9F74F064688B0E3
:10113000002017681062D06190615061FE480490F1
:101140000020009001900290824603900998154675
:1011500047F6FF7BA0F10109A6F10108002871D92B
:101160000024002E69D94FEAEA700AEBD06020F023
:101170001F01AAEB0101012202FA01F1401105EB66
:101180008000CDE906011C3005900AFB064007EB04
:101190004000BAF1000FB0F9500018BFCA450BD19A
:1011A000002C18BF444507D1E4490968B1F99220E1
:1011B000B1F99010B2B911E0E049049B0968984276
:1011C000B1F98A20B1F98810C4BF0294CDE903A017
:1011D0005845BCBF8346CDE9004AEBE7D74A1268C1
:1011E000B2F98A2019B9D5490968B1F98810904235
:1011F00001DC88421EDA06994FF0010CCA69079992
:101200000A4305990A60E11704EBD1614A1105EB25
:10121000820303F1140221F01F015B69611A0CFAC9
:1012200001F11943116083B2E2B20AF0FF01062016
:10123000FEF74DF8641CB442A7D309980AF1010ADD
:1012400082458DD3BD4C2068B0F88E00002846D072
:101250000499A1EB0B01814241DD039803994009F8
:1012600005EB800001F01F03C269012101FA03F3BD
:101270001A43C2610198019A400905EB800002F00F
:101280001F02C36901FA02F21A43C2610298029A6C
:10129000400905EB800002F01F02436901FA02F2E7
:1012A0001A4342610098009A400905EB800002F061
:1012B0001F024369914019434161049883B2029827
:1012C000C2B20398C1B20620FEF701F800981FFAD7
:1012D0008BF3C2B20198C1B20620FDF7F8FF974820
:1012E000006890F88C00002800F032814FF0000A6E
:1012F000002E7DD90998801E009007EB4A000999BD
:10130000B0F950000024012973D04FEAEA710AEBCA
:10131000D16121F01F02AAEB0202012303FA02F2BB
:10132000491105EB8101CDE9031214310291611CD1
:10133000019101FB06A107EB4101B1F950B0BBF1EE
:10134000000FC8BF00285EDDBBEB000148BFA0EB6B
:101350000B018345CCBF5A4602464FF448435943DC
:1013600091FBF2F101F2FF114A0A002C1CBF009917
:101370008C420AD1BAF1000F18BFC24504D16F499F
:10138000096891F88D100CE014B100998C4204D1D9
:101390006A49096891F8991003E06849096891F869
:1013A0008C1019B96549096891F88C108A422ADDB8
:1013B000E11704EBD1614A1105EB820221F01F0114
:1013C00002F11C03A4EB010CD269012101FA0CF11A
:1013D00011431960039983B206204A6904990A43AC
:1013E00002990A600AF0FF02E1B2FDF770FF01E026
:1013F00012E00CE001981FFA8BF3C1B20AF0FF0271
:101400000620FDF764FF641C58464C458FD30AF153
:10141000010AB245FFF471AF09984FF0000A0028A5
:1014200084BFB01E00907DD90AFB06F007EB400098
:101430000024B0F95000012E75D04FEAEA710AEB92
:10144000D16121F01F02AAEB0202012303FA02F28A
:10145000491105EB8101CDE902121C3101910AFB12
:10146000064107EB4101B1F952B0BBF1000FC8BF13
:1014700000285EDDBBEB000148BFA0EB0B018345FC
:10148000CCBF5A4602464FF44843594391FBF2F110
:1014900001F2FF114A0ABAF1000F18BFCA4509D17B
:1014A000002C1CBF00998C4205D12449096891F891
:1014B0008D100CE014B100998C4204D11F490968C9
:1014C00091F8981003E01D49096891F88C1019B93A
:1014D0001A49096891F88C108A422ADD02994FF066
:1014E000010CCA6903990A4301990A60E11704EBE8
:1014F000D1614A1105EB820303F1140221F01F01AF
:101500005B69611A0CFA01F11943116083B2E2B20E
:101510000AF0FF010620FDF7DAFE601C1FFA8BF3CC
:10152000C2B201E014E00DE00AF0FF010620FDF771
:10153000CEFE5846641C03E00080FFFFE0860010EA
:1015400044458CD309980AF1010A8245FFF46CAF37
:101550000BB00120BDE8F08F2DE9F74F06460020C3
:1015600084B017681062D06190610546506105989B
:101570009046002884BFA0F1010BA6F1010A7DD995
:101580000024002E7ED9E81705EBD06020F01F0163
:10159000691A012202FA01F1401108EB8000CDE93D
:1015A00001011C30009005FB064007EB4000082DB0
:1015B000B0F950000CD1002C0ADB012C08DCFF49EB
:1015C000002C096814BFB1F9BA90B1F9B8902CE0B9
:1015D000002D18BF5D451CD1002C18BF544519D1F2
:1015E00055EA040108BF40F2132925D0002D04BF9D
:1015F000544540F235291FD05D4504BF002C4FF4FF
:101600001F7919D05D4504BF54454FF4347913D088
:101610000BE00CB1544504D1E8490968B1F9B29026
:1016200003E0E6490968B1F9B090B9F1000F03D1C0
:10163000E2490968B1F9B09048451DDD01994FF0C4
:10164000010CCA6902990A4300990A60E11704EB88
:10165000D1614A1108EB820303F1140221F01F014A
:101660005B69611A0CFA01F11943116083B2E2B2AD
:10167000E9B20720FDF72BFE641C01E007E001E062
:10168000B44290D305986D1C8542FFF479AF0025D4
:1016900000287CD90024002E7AD9E81705EBD06009
:1016A00020F01F01691A012202FA01F1401108EB32
:1016B00080000391029005FB06F11C30CDE900107B
:1016C00005F1010AA5F1010905FB064007EB400BF6
:1016D0000598731EBBF95020A0F1010C00210846AB
:1016E00035B109FB064007EB40000121B0F950007D
:1016F000654507D00AFB064E07EB4E0E491CBEF9A6
:1017000050E070441CB1BBF94EE0491C70449C424F
:1017100003D0BBF952B0491C5844002C18BF654592
:1017200007D00AFB064B07EB4B0B491CBBF94EB02D
:1017300058449C4218BF654507D00AFB064C07EB8E
:101740004C0C491CBCF952C06044002C18BF002D41
:1017500007D009FB064C07EB4C0C491CBCF94EC0EA
:1017600060449C4218BF002D07D009FB064307EBDD
:101770004303491CB3F952301844002914BF002A0E
:10178000FF2016D06423584390FBF1F001E049E0BC
:1017900043E002EBC20101EB0211C0EB810000B299
:1017A0000028A7BF1044401E801A401C90FBF2F096
:1017B00000B2834B0099DFF80CC22344CB56A444FB
:1017C00011F90C1055EA040C08BF6FF09001984213
:1017D00001DC88421DDA02984FF0010CC1690398C0
:1017E000014301980160E01704EBD060411108EB60
:1017F000810101F1140320F01F004969201A0CFA3D
:1018000000F00843186093B2E2B2E9B20720FDF796
:101810005EFD641CB442FFF457AF05986D1C854211
:10182000FFF438AF07B00120BDE8F08F2DE9F04F8D
:10183000D2F80090804689B0D9F81000164620F002
:101840000F00C9F8100047F6FF7003906FEA000020
:1018500002904FF0FF00049005904FF000001061DF
:10186000F060B0605FEA010A09F1500B0546706054
:1018700067D005FB08F04FF0000E3BF91010CDE9E2
:10188000005E0A46012017467346B8F1010F19D9C8
:1018900005FB080C3BF91C408C42C4BF2146864620
:1018A000BC42BCBF27460190B4EB020C48BFA2EB80
:1018B000040C0FFA8CF29A42C8BF13462246401C11
:1018C0004045E5D30298814202DDCDE9045E0291F4
:1018D0000398874203DA0198039707950690C81B7F
:1018E00048BF781A02B235480068B0F91CC0944568
:1018F00003DBB0F91E00834220DDEA1705EBD2625C
:10190000531106EB830C22F01F020CF10C03AA1AF0
:101910000120DCF80CC090404CEA000018608BB24B
:101920000EF0FF02E9B20520FDF7D1FC0198BBB231
:10193000C2B20098C1B20520FDF7C9FC6D1C554527
:1019400097D30025B8F1000F5ED93BF915100020A0
:101950008646034600900A46012017460195BAF1D3
:10196000010F19D900FB085C3BF91C408C42C4BF35
:1019700021468646BC42BCBF27460090B4EB020C11
:1019800048BFA2EB040C0FFA8CF29A42C8BF134670
:101990002246401C5045E5D3C81B48BF781A02B206
:1019A00006480068B0F920C0944503DBB0F9220076
:1019B000834226DDEA1705EBD26205E0E0860010DF
:1019C000E0680200666B0200531106EB830322F00D
:1019D0001F0203F1040CAA1A01205B68904018430F
:1019E0008BB2CCF80000EAB20EF0FF010520FDF743
:1019F0006EFC0198BBB2C2B20098C1B20520FDF7DF
:101A000066FC6D1C4545A0D3F068002804BF306912
:101A1000002805D0D9F8100040F00800C9F81000DF
:101A20007068002804BFB068002805D0D9F81000FD
:101A300040F00400C9F810007168F06801FA0AF17A
:101A40000843C9F82800B168306901FA0AF108436F
:101A5000C9F82C007168BAF1200F39BFCAF1200211
:101A6000D140AAF1200291400843C9F82C00039804
:101A7000A9F824000298A9F82600B6F9D81002980F
:101A8000401A44BF0298081AF64C2168B1F91810A0
:101A900088420EDDD9F8100040F00200C9F81000AD
:101AA000029883B20598C2B20498C1B20520FDF72E
:101AB0000EFCB6F9D8100398081A44BF0398401AD0
:101AC0002168B1F91A1088420EDDD9F8100040F0F3
:101AD0000100C9F81000039883B20698C2B20798B3
:101AE000C1B20520FDF7F3FB09B00120BDE8F08F7E
:101AF0002DE9F04F0446DC4887B00F4600684FF0F0
:101B0000000890F8F80000F00F0500F0C8FA01286E
:101B10000BD040F20F312846F5F7BCFE012813D058
:101B2000002000F0B9FA00F099B900210846F1F759
:101B3000A5F8EFF741FA50B1CC48D0F8401341F482
:101B40008031C0F8401302E0012000F0A5FAC84837
:101B50000678C8480578002D18BF002E00F07C815B
:101B60003868002180F8206080F8215080F8221029
:101B700080F82310F1F769FEF1F77AF90090002060
:101B800014F0030F18BFBC4814F0200F1CBF40F026
:101B9000F00040F00050DFF8CC82002800F0DD803B
:101BA000009940F47F00084014F4407F18BF20F4EF
:101BB0007F00F1F72DF80020F7F7A2FA60F30F0984
:101BC000824600210846F7F785FA0220F7F798FACF
:101BD00060F31F4900210220F7F77CFA1220F7F783
:101BE0008FFA60F30F0B00211220F7F773FA14F449
:101BF000407F17D00020EFF7A6FD06900020EFF7FA
:101C000048FE05900020EFF781FE04900020EFF7DA
